:020000040800F2
:10000000A074002085050008E5050008E505000846
:10001000E5050008E5050008E5050008000000000A
:10002000000000000000000000000000E5050008DE
:10003000E505000800000000E50500087945000816
:10004000E5050008E5050008E5050008E5050008E8
:10005000E5050008E5050008E5050008E5050008D8
:10006000E5050008E5050008E5050008E5050008C8
:10007000E5050008E5050008E5050008E5050008B8
:10008000E5050008E5050008E5050008E5050008A8
:10009000E5050008E5050008E5050008E505000898
:1000A000E5050008E5050008C59C0008E505000811
:1000B000DD450008E5050008E5050008E505000840
:1000C000E5050008E5050008E5050008E505000868
:1000D000E5050008BD630008D1630008E56300087A
:1000E000E5050008E5050008E5050008E505000848
:1000F000E5050008E5050008E5050008E505000838
:10010000E5050008E5050008E5050008E505000827
:10011000F96300080D640008E5050008E50500081E
:10012000E5050008E5050008E5050008E505000807
:10013000E5050008E5050008E5050008E5050008F7
:10014000E5050008E5050008E5050008E5050008E7
:10015000E5050008E5050008E5050008216400083C
:10016000E5050008E5050008E5050008E5050008C7
:10017000E5050008E5050008E5050008E5050008B7
:10018000E5050008E505000880B582B000AF04F081
:100190006DFA02460B4613467B601B4B1B687A6860
:1001A000D21A1A4B1B689A422BD9194B1B68002B89
:1001B0000ED0184B1B685A00164B1A60154B1B6863
:1001C000B3F5006F11D9134B4FF480721A600CE035
:1001D000104B1B685A080F4B1A600E4B1B68FF2B05
:1001E00003D80C4B4FF400621A600B4B0A4A526959
:1001F00022F47061074A12680A435A61024B7A6816
:100200001A600837BD4680BDC80A0020D010002003
:10021000D00A0020000000200008024080B582B013
:1002200000AF04F023FA02460B4613467B60144BE2
:100230001B687A68D21A134B1B689A421DD9124B5D
:100240001B68002B14BF00230123DBB21A460E4BA0
:100250001A600D4B1B68002B06D00C4B0B4A5269E1
:1002600042F470625A6105E0084B084A526922F470
:1002700070625A61024B7A681A600837BD4680BDC9
:10028000E00A0020D0100020D40A0020000802401C
:1002900080B500AF044B1B68002B04D0012003493C
:1002A00001220DF0B9FE80BDD80A0020001E010811
:1002B00080B582B000AF09F05DFB78600837BD46BD
:1002C00080BD00BF80B500AFFFF7E2FFFFF7F0FF92
:1002D000064B1B68002B02D0012B03D005E0FFF773
:1002E00053FF02E0FFF79AFF00BF80BDDC0A002049
:1002F00080B500AF354809F077FE012034490AF097
:1003000045FD344B1B685A08334B1A6009F0A8FBB3
:100310000120012108F06AFDFFF7D4FF4FF480505F
:1003200009F02EFE0346002B13D02B4B1B68642BC9
:1003300005D9294B1B68A3F16402274B1A60274B90
:100340001B68002B14BF00230123DBB21A46234B8A
:100350001A604FF4005009F013FE0346002B0CD036
:100360001C4B1B685A001C4B1B689A4205D91A4B40
:100370001B6803F16402184B1A604FF4804009F0C7
:10038000FFFD0346002B09D0154B1B68002B14BF43
:1003900000230123DBB21A46114B1A604FF40040D0
:1003A00009F0EEFD0346002B0ED00E4B1B685A1CC5
:1003B0000C4B1A600B4B1A680B4B1B689A4203DDFF
:1003C000084B00221A60A7E7A6E700BF041E010839
:1003D000101E0108D8100020D0100020D80A0020DC
:1003E000D00A0020DC0A00200400002080B485B080
:1003F00000AF78600B4B1B68002B02D1094B0A4AF7
:100400001A60084B1B68FB60064B1A687B681A442D
:10041000044B1A60FB6818461437BD465DF8047B30
:10042000704700BFE40A0020A014002080B483B00D
:1004300000AF7860FEE700BF80B483B000AF7860A3
:100440003960054B16221A604FF0FF3318460C37FF
:10045000BD465DF8047B70479C14002080B400AF5B
:1004600001231846BD465DF8047B704780B483B015
:1004700000AF786039604FF0FF3318460C37BD4647
:100480005DF8047B704700BF80B582B000AF786034
:10049000786806F035FF034618460837BD4680BD2C
:1004A00080B586B000AFF860B9607A60F868B96866
:1004B00006F0C0FD78617B69002B01DB7B6904E0FD
:1004C000044B7A691A604FF0FF3318461837BD465F
:1004D00080BD00BF9C14002080B582B000AF786062
:1004E000786807F073F8034618460837BD4680BDA4
:1004F00080B584B000AFF860B9607A60F868B96818
:100500007A6806F047FF034618461037BD4680BD9F
:1005100080B584B000AFF860B9607A60F868B968F7
:100520007A6806F0A5FE034618461037BD4680BD22
:1005300080B584B000AFF860B9607A60F868B968D7
:100540007A6806F057FE034618461037BD4680BD50
:1005500080B400AFFEE700BF0EB480B585B000AF39
:10056000786007F12003BB607868F969BA6806F023
:10057000E1FFF860FB6818461437BD46BDE88040CF
:1005800003B0704780B582B000AF134B7B60134B54
:100590003B6007E03B681A1D3A607A68111D79607C
:1005A00012681A603A680E4B9A42F3D30F4810490A
:1005B0004FF000028842B8BF40F8042BFADBDFF8A6
:1005C0003400016841F47001016000F015F8FFF794
:1005D0008FFE0837BD4680BD742C01080000002046
:1005E000C40A002080B400AFFEE70000C80A002063
:1005F000A014002088ED00E080B400AF164B164A2E
:10060000D2F8882042F47002C3F88820134B134AB2
:10061000126842F001021A60104B00229A600F4AE1
:100620000E4B1B6823F0847323F4803313600B4B51
:100630000B4A5A60094B094A126822F480221A6058
:10064000064B0022DA60044B4FF000629A60BD4610
:100650005DF8047B704700BF00ED00E00038024009
:100660001030002480B487B000AF00233B6100232A
:100670007B610223FB600023BB6002237B60324B63
:100680009B6803F00C033B613B69042B07D0082BEC
:1006900009D0002B3FD12D4B2D4A1A603FE02B4B48
:1006A0002C4A1A603BE0284B5B6803F480039B0DE7
:1006B000BB60254B5B6803F03F037B60BB68002B8E
:1006C0000DD0244A7B68B2FBF3F21F4B596847F602
:1006D000C0730B409B0903FB02F37B610CE01C4AD7
:1006E0007B68B2FBF3F2184B596847F6C0730B40B6
:1006F0009B0903FB02F37B61134B5B6803F44033FC
:100700001B0C01335B00FB607A69FB68B2FBF3F200
:100710000E4B1A6003E00D4B0D4A1A6000BF0A4BE6
:100720009B6803F0F0031B090B4AD35CDBB23B610F
:10073000064B1A683B69DA40044B1A601C37BD4609
:100740005DF8047B704700BF0038024008000020BD
:100750000024F40000127A000C00002080B489B05C
:1007600000AF0723FB61C023BB6105237B6100232E
:100770007B6000233B6002233B610823FB604FF456
:10078000A873BB604B4B4C4A1A604C4B4B4A1268E7
:1007900042F480321A60494B1B6803F400333B601B
:1007A0007B6801337B603B68002B03D17B68B3F52A
:1007B000A04FF0D1414B1B6803F40033002B02D053
:1007C00001233B6001E000233B603B68012B50D1DB
:1007D0003A4B3A4A126C42F080521A64384B384A0B
:1007E000126842F440421A60344B344A92689A606C
:1007F000324B324A926842F400429A602F4B2F4AA1
:10080000926842F4A0529A602C4BBA689101FA683F
:1008100011433A695210013A12040A431146FA6927
:1008200012060A4342F480025A60244B234A12689B
:1008300042F080721A6000BF204B1B6803F0007307
:10084000002BF9D01F4B40F205621A601B4B1B4A6C
:10085000926822F003029A60184B184A926842F09C
:1008600002029A6000BF154B9B6803F00C03082B33
:10087000F9D1124B114A926822F400029A600F4B90
:10088000BA6991017A6912070A43C3F884200B4BB5
:100890000A4A126842F080621A6000BF074B1B6868
:1008A00003F00063002BF9D02437BD465DF8047BCC
:1008B000704700BF08000020007A030A0038024099
:1008C00000700040003C024080B485B000AF1023AF
:1008D000FB604FF4A873BB6004237B6007233B607D
:1008E0002B4B2C4A1A602C4B2B4A126C42F0805234
:1008F0001A642A4B294A126842F440421A60264B75
:10090000254A92689A60244B234A926842F4204216
:100910009A60214B204A926842F4A0529A601E4B82
:10092000BA689101FA6811437A685210013A1204C8
:100930000A4311463A6812060A435A60164B164A91
:10094000126842F080721A6000BF134B1B6803F0FC
:100950000073002BF9D0124B4FF4C1621A600E4B9A
:100960000D4A926822F003029A600B4B0A4A926881
:1009700042F002029A6000BF074B9B6803F00C0331
:10098000082BF9D11437BD465DF8047B704700BFD2
:100990000800002000BD0105003802400070004042
:1009A000003C024080B485B000AF1023FB60F02310
:1009B000BB6008237B6005233B60294B294A1A60F2
:1009C000294B294A126C42F080521A64274B274A5D
:1009D000126842F440421A60234B234A92689A609C
:1009E000214B214A92689A601F4B1F4A92689A6075
:1009F0001D4BBA689101FA6811437A685210013AA6
:100A000012040A4311463A6812060A435A60164B0A
:100A1000154A126842F080721A6000BF124B1B68C0
:100A200003F00073002BF9D0114B40F202621A6000
:100A30000D4B0D4A926822F003029A600A4B0A4A53
:100A4000926842F002029A6000BF074B9B6803F075
:100A50000C03082BF9D11437BD465DF8047B7047B1
:100A60000800002080C3C901003802400070004027
:100A7000003C024080B400AF114B124A1A60124B86
:100A8000114A126C42F080521A64104B0F4A1268DD
:100A900042F440421A600C4B0B4A92689A600A4B2F
:100AA000094A92689A60084B074A92689A60084B14
:100AB0004FF4C0621A60BD465DF8047B704700BF0A
:100AC000080000200024F4000038024000700040BC
:100AD000003C024080B483B000AF7860054A7B6878
:100AE00043F0BF6343F40033D3600C37BD465DF879
:100AF000047B704700ED00E080B485B000AF786003
:100B00000023FB730023BB730F237B737B68DB78AD
:100B1000002B37D0254BDB68DB4303F4E0631B0A73
:100B2000FB73FB7BC3F10403BB737A7BFB7B42FA51
:100B300003F37B737B685B781A46BB7B02FA03F393
:100B4000FB737B689A787B7B1340DAB2FB7B1343A1
:100B5000FB73FB7B1B01FB73154A7B681B781344FB
:100B6000FA7B83F80023124B7A6812785209D2B2CA
:100B70007968097801F01F01012000FA01F143F8BA
:100B800022100EE00A4B7A6812785209D2B27968C4
:100B9000097801F01F01012000FA01F1203243F829
:100BA00022101437BD465DF8047B704700ED00E06D
:100BB00000E100E080B483B000AF78603960074A9C
:100BC0003B6823F0604323F07F0379680B43936015
:100BD0000C37BD465DF8047B704700BF00ED00E0B8
:100BE00080B483B000AF02460B46FA71BB71BB798B
:100BF000002B06D0094B094A1169FA790A431A6198
:100C000006E0064B054A1169FA79D2430A401A6197
:100C10000C37BD465DF8047B704700BF00ED00E077
:100C200080B483B000AF78607B68042B06D1094B99
:100C3000084A126842F004021A6005E0054B054AB2
:100C4000126822F004021A600C37BD465DF8047B7E
:100C5000704700BF10E000E080B400AF094B0022F5
:100C60001A60084B00225A60064B00229A60054B1E
:100C70000022DA60034B044A5A61BD465DF8047BEA
:100C8000704700BF003C0140FFFF7F0080B485B08B
:100C900000AF78600023FB60324BFB607B689B7980
:100CA000002B4DD02F4B2F4A11687A681268D2431F
:100CB0000A401A602B4B2B4A51687A681268D2435B
:100CC0000A405A607B681B79FA681344FB60FB6832
:100CD000FA6811687A6812680A431A60214B214A3F
:100CE00091687A681268D2430A409A601D4B1D4A87
:100CF000D1687A681268D2430A40DA607B685B790F
:100D0000102B0ED1174B174A91687A6812680A4364
:100D10009A60144B134AD1687A6812680A43DA6001
:100D20001BE0104BFB607B685B79FA681344FB6047
:100D3000FB68FA6811687A6812680A431A600CE066
:100D40007B681B79FA681344FB60FB68FA681168DA
:100D50007A681268D2430A401A601437BD465DF8BB
:100D6000047B7047003C014080B483B000AF7860E2
:100D70007B6800221A607B6800221A717B680C2253
:100D80005A717B6800229A710C37BD465DF8047B6E
:100D9000704700BF80B483B000AF7860054B054A50
:100DA00011697A680A431A610C37BD465DF8047B05
:100DB000704700BF003C014080B485B000AF786050
:100DC0000023FB73084B5A697B681340002B02D049
:100DD0000123FB7301E00023FB73FB7B18461437F0
:100DE000BD465DF8047B7047003C014080B483B091
:100DF00000AF7860034B7A685A610C37BD465DF8E6
:100E0000047B7047003C014080B485B000AF78603F
:100E10000023FB73084B5A697B681340002B02D0F8
:100E20000123FB7301E00023FB73FB7B184614379F
:100E3000BD465DF8047B7047003C014080B483B040
:100E400000AF7860034B7A685A610C37BD465DF895
:100E5000047B7047003C014080B582B000AF7860F1
:100E60007A684B4B9A4208D10120012100F052FED2
:100E70000120002100F04EFE86E07A68454B9A4240
:100E800008D10220012100F045FE0220002100F0DF
:100E900041FE79E07A68404B9A4208D10420012152
:100EA00000F038FE0420002100F034FE6CE07A6887
:100EB0003A4B9A4208D10820012100F02BFE08206D
:100EC000002100F027FE5FE07A68354B9A4208D196
:100ED0001020012100F01EFE1020002100F01AFE5B
:100EE00052E07A682F4B9A4208D12020012100F06D
:100EF00011FE2020002100F00DFE45E07A682A4B0B
:100F00009A4208D14020012100F004FE4020002137
:100F100000F000FE38E07A68244B9A4208D1802025
:100F2000012100F0F7FD8020002100F0F3FD2BE00F
:100F30007A681F4B9A420AD14FF48070012100F069
:100F4000E9FD4FF48070002100F0E4FD1CE07A68B8
:100F5000184B9A420AD14FF40070012100F0DAFDDB
:100F60004FF40070002100F0D5FD0DE07A68124BBF
:100F70009A4209D14FF48060012100F0CBFD4FF47B
:100F80008060002100F0C6FD0837BD4680BD00BF6F
:100F9000000002400004024000080240000C024031
:100FA000001002400014024000180240001C0240E1
:100FB00000200240002402400028024080B487B094
:100FC00000AF7860396000237B6100233B61002320
:100FD000FB6000237B6176E07B69012202FA03F368
:100FE0003B613B681A683B691340FB60FA683B69E8
:100FF0009A4265D17B681A687B695B00032101FA1C
:1010000003F3DB431A407B681A607B681A683B680D
:101010001B7919467B695B0001FA03F31A437B686D
:101020001A603B681B79012B03D03B681B79022BAC
:101030002ED17B689A687B695B00032101FA03F378
:10104000DB431A407B689A607B689A683B685B79EF
:1010500019467B695B0001FA03F31A437B689A60C7
:101060007B685A687B699BB2012101FA03F3DB4379
:101070001A407B685A607B685A683B689B791946BE
:101080007B699BB201FA03F39BB21A437B685A60F7
:101090007B68DA687B699BB25B00032101FA03F38A
:1010A000DB431A407B68DA607B68DA683B68DB798F
:1010B00019467B695B0001FA03F31A437B68DA6027
:1010C0007B6901337B617B690F2B85D91C37BD465A
:1010D0005DF8047B704700BF80B483B000AF7860D8
:1010E0007B684FF6FF721A607B6800221A717B687A
:1010F00000225A717B6800229A717B680022DA71A3
:101100000C37BD465DF8047B704700BF80B485B0E6
:1011100000AF78600B467B804FF48033FB607A88A9
:10112000FB681343FB60FA687B68DA617A887B6846
:10113000DA61FA687B68DA617B68DB69FB607B688F
:10114000DB69FB601437BD465DF8047B704700BF68
:1011500080B485B000AF78600B467B800023FB73C2
:101160007B681A697B881340002B02D00123FB7334
:1011700001E00023FB73FB7B18461437BD465DF886
:10118000047B704780B483B000AF78607B681B69D4
:101190009BB218460C37BD465DF8047B704700BF14
:1011A00080B485B000AF78600B467B800023FB7372
:1011B0007B685A697B881340002B02D00123FB73A4
:1011C00001E00023FB73FB7B18461437BD465DF836
:1011D000047B704780B483B000AF78607B685B6944
:1011E0009BB218460C37BD465DF8047B704700BFC4
:1011F00080B483B000AF78600B467B807B687A88D0
:101200001A830C37BD465DF8047B704780B483B009
:1012100000AF78600B467B807B687A885A830C37F6
:10122000BD465DF8047B704780B483B000AF786042
:1012300013460A467A807B707B78002B03D07B684C
:101240007A881A8302E07B687A885A830C37BD4615
:101250005DF8047B704700BF80B483B000AF786056
:101260000B467B807A887B685A610C37BD465DF8F7
:10127000047B704780B483B000AF78600B467B80FE
:101280007B685A697B885A407B685A610C37BD4637
:101290005DF8047B704700BF80B485B000AF786014
:1012A00013460A467A807B700023FB600023BB60F4
:1012B0007A787B8803F007039B0002FA03F3FB6054
:1012C0007B88DB089BB21A467B88DB089BB21946F9
:1012D0007B68083153F821107B8803F007039B00DB
:1012E0000F2000FA03F3DB4319407B68083243F810
:1012F00022107B88DB089BB21A467B68083253F8C1
:101300002220FB681343BB607B88DB089BB21A4634
:101310007B680832B96843F822101437BD465DF87F
:10132000047B704780B400AF144B144A126842F03B
:1013300001021A60114B00229A60104A0F4B1B6881
:1013400023F0A85323F4102313600C4B0C4A5A606B
:101350000A4B0C4AC3F88420084B084A126822F44E
:1013600080221A60054B0022DA60044B0022C3F889
:101370008C20BD465DF8047B704700BF00380240FA
:10138000103000240030002080B483B000AF03464A
:10139000FB71054B00221A70034BFA791A700C3757
:1013A000BD465DF8047B70470238024080B582B0CC
:1013B00000AF00233B600023FB710023BB71312091
:1013C00000F0D8FC0346BB713B6801333B603B68CF
:1013D000B3F5A04F02D0BB79002BF0D0312000F044
:1013E000C9FC0346002B02D00123FB7101E000235E
:1013F000FB71FB7918460837BD4680BD80B485B0C7
:1014000000AF0346FB710023FB600A4B1B68FB60C7
:10141000FB6823F0F803FB60FB79DB00FA681343F9
:10142000FB60044BFA681A601437BD465DF8047B14
:10143000704700BF0038024080B483B000AF03465D
:10144000FB71044BFA791A600C37BD465DF8047BDA
:10145000704700BF0000474280B483B000AF03462E
:10146000FB710C4B00221A700A4B00221A70FB7998
:10147000012B02D0042B04D007E0064B01221A7086
:1014800003E0044B05221A7000BF0C37BD465DF81F
:10149000047B70477038024080B483B000AF0346CD
:1014A000FB71044BFA791A600C37BD465DF8047B7A
:1014B000704700BF800E474280B485B000AFF8602F
:1014C000B9607A603B600A4B7A689101BA6811434F
:1014D0003A685208013A12041143FA681143BA6992
:1014E00012060A435A601437BD465DF8047B704704
:1014F0000038024080B483B000AF0346FB71044B58
:10150000FA791A600C37BD465DF8047B704700BF5E
:101510006000474280B483B000AF78603960064B0A
:101520007A6891013A6812070A43C3F884200C379D
:10153000BD465DF8047B70470038024080B483B03C
:1015400000AF0346FB71044BFA791A600C37BD46B5
:101550005DF8047B704700BF6800474280B485B0E7
:1015600000AFF860B9607A60074BFA689101BA6819
:10157000120611437A6812070A43C3F88820143709
:10158000BD465DF8047B70470038024080B483B0EC
:1015900000AF0346FB71044BFA791A600C37BD4665
:1015A0005DF8047B704700BF7000474280B483B091
:1015B00000AF0346FB71044BFA791A600C37BD4645
:1015C0005DF8047B704700BF4C00474280B485B093
:1015D00000AF786039600023FB600A4B9B68FB60BA
:1015E000FB6823F0EC63FB607A683B681343FA689E
:1015F0001343FB60034BFA689A601437BD465DF8ED
:10160000047B70470038024080B485B000AF78603A
:1016100039600023FB600A4B9B68FB60FB6823F08A
:101620007843FB607A683B681343FA681343FB60B6
:10163000034BFA689A601437BD465DF8047B704727
:101640000038024080B485B000AF78600023FB60B2
:10165000094B9B68FB60FB6823F00303FB60FA689F
:101660007B681343FB60044BFA689A601437BD46ED
:101670005DF8047B704700BF0038024080B400AFC3
:10168000054B9B68DBB203F00C03DBB21846BD468A
:101690005DF8047B704700BF0038024080B485B01D
:1016A00000AF78600023FB60094B9B68FB60FB6820
:1016B00023F0F003FB60FA687B681343FB60044B84
:1016C000FA689A601437BD465DF8047B704700BF26
:1016D0000038024080B485B000AF78600023FB6022
:1016E000094B9B68FB60FB6823F4E053FB60FA68DE
:1016F0007B681343FB60044BFA689A601437BD465D
:101700005DF8047B704700BF0038024080B485B0AC
:1017100000AF78600023FB60094B9B68FB60FB68AF
:1017200023F46043FB607B68DB00FA681343FB60D3
:10173000034BFA689A601437BD465DF8047B704726
:101740000038024080B489B000AF78600023BB61EC
:1017500000237B610023FB6102233B610023FB60CC
:101760000223BB60484B9B6803F00C03BB61BB6961
:10177000042B07D0082B09D0002B3FD17B68434AAC
:101780001A603FE07B68424A1A603BE03E4B5B6870
:1017900003F480039B0DFB603B4B5B6803F03F034E
:1017A000BB60FB68002B0DD0394ABB68B2FBF3F27B
:1017B000354B596847F6C0730B409B0903FB02F396
:1017C000FB610CE0314ABB68B2FBF3F22E4B596867
:1017D00047F6C0730B409B0903FB02F3FB612A4BE6
:1017E0005B6803F440331B0C01335B003B61FA6917
:1017F0003B69B2FBF3F27B681A6003E07B68234A23
:101800001A6000BF204B9B6803F0F003BB61BB690B
:101810001B09BB611F4ABB6913441B78DBB27B61A8
:101820007B681A687B69DA407B685A60164B9B6854
:1018300003F4E053BB61BB699B0ABB61154ABB69FA
:1018400013441B78DBB27B617B685A687B69DA40A2
:101850007B689A600C4B9B6803F46043BB61BB6977
:101860005B0BBB610B4ABB6913441B78DBB27B612A
:101870007B685A687B69DA407B68DA602437BD464A
:101880005DF8047B704700BF003802400024F4007C
:1018900000127A001C00002080B485B000AF786090
:1018A0000023FB607B6803F44073B3F5407F11D1E4
:1018B0000F4B9B68FB60FB6823F4F813FB607B68AD
:1018C00023F0704323F44073FA681343FB60084B22
:1018D000FA689A60064B064A116F7A68C2F30B02E7
:1018E0000A431A671437BD465DF8047B704700BF92
:1018F0000038024080B483B000AF0346FB71044B54
:10190000FA791A600C37BD465DF8047B704700BF5A
:101910003C0E474280B483B000AF0346FB71044BDA
:10192000FA791A600C37BD465DF8047B704700BF3A
:10193000400E474280B483B000AF7860034B7A68B2
:101940001A600C37BD465DF8047B70475C01474266
:1019500080B485B000AF78600023FB600A4BD3F8F9
:101960008C30FB60FB6823F01F03FB607B68013B4E
:10197000FA681343FB60044BFA68C3F88C201437F1
:10198000BD465DF8047B70470038024080B485B0E6
:1019900000AF78600023FB600B4BD3F88C30FB600A
:1019A000FB6823F4F853FB607B68013B1B02FA6879
:1019B0001343FB60044BFA68C3F88C201437BD4610
:1019C0005DF8047B704700BF0038024080B485B0EA
:1019D00000AF78600023FB600A4BD3F88C30FB60CB
:1019E000FB6823F44033FB60FA687B681343FB60B9
:1019F000044BFA68C3F88C201437BD465DF8047BAD
:101A0000704700BF0038024080B483B000AF7860F8
:101A1000034B7A681A600C37BD465DF8047B70474B
:101A2000E011474280B483B000AF78600B46FB7092
:101A3000FB78002B06D0094B084A116B7A680A43E1
:101A40001A6306E0054B054A116B7A68D2430A40D7
:101A50001A630C37BD465DF8047B704700380240BE
:101A600080B483B000AF78600B46FB70FB78002B2E
:101A700006D0094B084A516B7A680A435A6306E05C
:101A8000054B054A516B7A68D2430A405A630C37BA
:101A9000BD465DF8047B70470038024080B483B0D7
:101AA00000AF78600B46FB70FB78002B06D0094B2B
:101AB000084A116C7A680A431A6406E0054B054A25
:101AC000116C7A68D2430A401A640C37BD465DF83F
:101AD000047B70470038024080B483B000AF786068
:101AE0000B46FB70FB78002B06D0094B084A516C63
:101AF0007A680A435A6406E0054B054A516C7A68D5
:101B0000D2430A405A640C37BD465DF8047B7047E7
:101B10000038024080B483B000AF78600B46FB70A1
:101B2000FB78002B06D0094B084A11697A680A43F2
:101B30001A6106E0054B054A11697A68D2430A40EA
:101B40001A610C37BD465DF8047B704700380240CF
:101B500080B483B000AF78600B46FB70FB78002B3D
:101B600006D0094B084A51697A680A435A6106E06F
:101B7000054B054A51697A68D2430A405A610C37CD
:101B8000BD465DF8047B70470038024080B483B0E6
:101B900000AF78600B46FB70FB78002B06D0094B3A
:101BA000084A116A7A680A431A6206E0054B054A38
:101BB000116A7A68D2430A401A620C37BD465DF852
:101BC000047B70470038024080B483B000AF786077
:101BD0000B46FB70FB78002B06D0094B084A516A74
:101BE0007A680A435A6206E0054B054A516A7A68E8
:101BF000D2430A405A620C37BD465DF8047B7047F9
:101C00000038024080B483B000AF78600B46FB70B0
:101C1000FB78002B06D0094B084A116D7A680A43FD
:101C20001A6506E0054B054A116D7A68D2430A40F1
:101C30001A650C37BD465DF8047B704700380240DA
:101C400080B483B000AF78600B46FB70FB78002B4C
:101C500006D0094B084A516D7A680A435A6506E076
:101C6000054B054A516D7A68D2430A405A650C37D4
:101C7000BD465DF8047B70470038024080B483B0F5
:101C800000AF78600B46FB70FB78002B06D0094B49
:101C9000084A116E7A680A431A6606E0054B054A3F
:101CA000116E7A68D2430A401A660C37BD465DF859
:101CB000047B70470038024080B483B000AF786086
:101CC0000B46FB70FB78002B06D0094B084A516E7F
:101CD0007A680A435A6606E0054B054A516E7A68EF
:101CE000D2430A405A660C37BD465DF8047B704704
:101CF0000038024080B483B000AF0346FB71FB792B
:101D0000012B06D1084B084A126F42F008021A67ED
:101D100005E0054B044A126F22F008021A670C37DF
:101D2000BD465DF8047B70470038024080B483B044
:101D300000AF02460B46FA71BB71BB79002B08D08D
:101D40000B4B0B4A1278D1B2FA790A43D2B21A700D
:101D500009E0074B064A1278D1B2FA79D243D2B2DF
:101D60000A40D2B21A700C37BD465DF8047B70474A
:101D70000D38024080B487B000AF0346FB710023EA
:101D8000FB6000237B610023FB74FB795B09DBB202
:101D9000FB60FB68012B03D1124B1B687B6109E0E0
:101DA000FB68022B03D10F4B1B6F7B6102E00D4BD5
:101DB0005B6F7B61FB7903F01F03FB60FB687A6953
:101DC00022FA03F303F00103002B02D00123FB747A
:101DD00001E00023FB74FB7C18461C37BD465DF810
:101DE000047B70470038024080B400AF044B044AC3
:101DF000526F42F080725A67BD465DF8047B7047AF
:101E00000038024080B485B000AF0346FB71002368
:101E1000FB73094BDA68FB791340002B02D00123D6
:101E2000FB7301E00023FB73FB7B18461437BD46B0
:101E30005DF8047B704700BF0038024080B483B077
:101E400000AF0346FB71044BFA791A700C37BD469C
:101E50005DF8047B704700BF0E38024080B500AFCC
:101E60004FF480400121FFF7AFFE4FF48040002186
:101E7000FFF7AAFE80BD00BF80B483B000AF034669
:101E8000FB71044BFA791A600C37BD465DF8047B90
:101E9000704700BF0038014080B483B000AF0346F4
:101EA000FB71044BFA791A600C37BD465DF8047B70
:101EB000704700BF2000274290B484B000AF0246B4
:101EC0000B46FA71BB710023FB60BB7903F003037F
:101ED0009B000F2202FA03F3FB60154BBA799208BC
:101EE000D2B21349B8798008C0B2023051F820004C
:101EF000F968C9430140023243F822100C4BBA7909
:101F00009208D2B20A49B8798008C0B2023051F8BA
:101F10002000FC79B97901F00301890004FA01F18C
:101F20000143023243F822101037BD4690BC70477F
:101F30000038014080B483B000AF7860034B7A680A
:101F40001A600C37BD465DF8047B7047DC00274201
:101F500080B483B000AF0346FB71044BFA791A607A
:101F60000C37BD465DF8047B704700BF0004274274
:101F700080B483B000AF0023FB71094B1B6A03F4EC
:101F80008073002B02D00123FB7101E00023FB7161
:101F9000FB7918460C37BD465DF8047B704700BFDF
:101FA0000038014080B582B000AF78607A685F4B3E
:101FB0009A4208D101200121FFF706FE01200021ED
:101FC000FFF702FEAFE07B68B3F1804F08D101203C
:101FD0000121FFF7DBFD01200021FFF7D7FDA2E083
:101FE0007A68534B9A4208D102200121FFF7CEFDB7
:101FF00002200021FFF7CAFD95E07A684D4B9A4216
:1020000008D104200121FFF7C1FD04200021FFF7C2
:10201000BDFD88E07A68484B9A4208D1082001212A
:10202000FFF7B4FD08200021FFF7B0FD7BE07A68E0
:10203000424B9A4208D110200121FFF7A7FD102042
:102040000021FFF7A3FD6EE07A683D4B9A4208D16C
:1020500020200121FFF79AFD20200021FFF796FDA7
:1020600061E07A68374B9A4208D102200121FFF7DC
:10207000ABFD02200021FFF7A7FD54E07A68324B48
:102080009A420AD14FF480300121FFF79DFD4FF4B1
:1020900080300021FFF798FD45E07A682B4B9A428B
:1020A0000AD14FF400300121FFF78EFD4FF40030CC
:1020B0000021FFF789FD36E07A68254B9A420AD164
:1020C0004FF480200121FFF77FFD4FF48020002195
:1020D000FFF77AFD27E07A681E4B9A4208D140202C
:1020E0000121FFF753FD40200021FFF74FFD1AE0CB
:1020F0007A68194B9A4208D180200121FFF746FDEA
:1021000080200021FFF742FD0DE07A68134B9A42D0
:1021100009D14FF480700121FFF738FD4FF4807032
:102120000021FFF733FD0837BD4680BD00000140A8
:102130000004004000080040000C00400010004077
:1021400000140040000401400040014000440140F0
:102150000048014000180040001C004000200040E2
:1021600080B485B000AF786039600023FB817B6864
:102170001B88FB817A68284B9A4213D07A68274BD8
:102180009A420FD07B68B3F1804F0BD07A68244B12
:102190009A4207D07A68234B9A4203D07A68224B3E
:1021A0009A4208D1FB8923F07003FB813B685A886F
:1021B000FB891343FB817A681C4B9A420CD07A68E6
:1021C0001B4B9A4208D0FB8923F44073FB813B6888
:1021D0001A89FB891343FB817B68FA891A803B6863
:1021E0005A687B68DA623B681A887B681A857A6865
:1021F000094B9A4203D07A68084B9A4204D13B6853
:102200009B7A1A467B681A867B6801229A82143769
:10221000BD465DF8047B70470000014000040140AA
:102220000004004000080040000C00400010004086
:102230000014004080B483B000AF78607B684FF03A
:10224000FF325A607B6800221A807B6800221A8164
:102250007B6800225A807B6800229A720C37BD4648
:102260005DF8047B704700BF80B483B000AF786036
:1022700013460A467A803B807B687A881A857B6899
:102280003A889A820C37BD465DF8047B704700BFE0
:1022900080B485B000AF78600B467B800023FB8163
:1022A0007B681B88FB81FB8923F07003FB81FA8923
:1022B0007B881343FB817B68FA891A801437BD46FB
:1022C0005DF8047B704700BF80B483B000AF7860D6
:1022D00039607B683A685A620C37BD465DF8047B0A
:1022E000704700BF80B483B000AF786039607B680E
:1022F0003A68DA620C37BD465DF8047B704700BF70
:1023000080B483B000AF78607B685B6A18460C3796
:10231000BD465DF8047B704780B483B000AF786041
:102320007B681B8D9BB218460C37BD465DF8047B5D
:10233000704700BF80B483B000AF78600B46FB707D
:10234000FB78002B08D07B681B889BB243F002030C
:102350009AB27B681A8007E07B681B889BB223F0E7
:1023600002039AB27B681A800C37BD465DF8047B85
:10237000704700BF80B483B000AF78600B467B80AD
:102380007B88002B08D07B681B889BB243F004033A
:102390009AB27B681A8007E07B681B889BB223F0A7
:1023A00004039AB27B681A800C37BD465DF8047B43
:1023B000704700BF80B483B000AF78600B46FB70FD
:1023C000FB78002B08D07B681B889BB243F080030E
:1023D0009AB27B681A8007E07B681B889BB223F067
:1023E00080039AB27B681A800C37BD465DF8047B87
:1023F000704700BF80B483B000AF78600B467B802D
:102400007B681B889BB223F008039AB27B681A8012
:102410007B681B889AB27B8813439AB27B681A80C8
:102420000C37BD465DF8047B704700BF80B483B0B5
:1024300000AF78600B467B807B681B889BB223F4DF
:1024400040739AB27B681A807B681B889AB27B883B
:1024500013439AB27B681A800C37BD465DF8047B43
:10246000704700BF80B483B000AF78600B46FB704C
:10247000FB78002B08D07B681B889BB243F00103DC
:102480009AB27B681A8007E07B681B889BB223F0B6
:1024900001039AB27B681A800C37BD465DF8047B55
:1024A000704700BF80B485B000AF7860396000230A
:1024B0007B810023FB810023BB817B681B8C9BB24B
:1024C00023F001039AB27B681A847B681B8CFB8122
:1024D0007B689B88BB817B681B8B7B817B8923F01E
:1024E00070037B817B8923F003037B813B681A881F
:1024F0007B8913437B81FB8923F00203FB813B68CB
:102500009A89FB891343FB813B685A88FB891343F3
:10251000FB817A681E4B9A4203D07A681D4B9A421F
:1025200023D1FB8923F00803FB813B68DA89FB890F
:102530001343FB81FB8923F00403FB813B689A88EA
:10254000FB891343FB81BB8923F48073BB81BB8967
:1025500023F40073BB813B681A8ABB891343BB8198
:102560003B685A8ABB891343BB817B68BA899A80CE
:102570007B687A891A833B689A687B685A637B68B0
:10258000FA891A841437BD465DF8047B704700BF92
:10259000000001400004014080B485B000AF7860C5
:1025A000396000237B810023FB810023BB817B6892
:1025B0001B8C9BB223F010039AB27B681A847B6851
:1025C0001B8CFB817B689B88BB817B681B8B7B8121
:1025D0007B8923F4E0437B817B8923F440737B81F7
:1025E0003B681B881B029AB27B8913437B81FB8962
:1025F00023F02003FB813B689B891B019AB2FB8976
:102600001343FB813B685B881B019AB2FB89134330
:10261000FB817A68224B9A4203D07A68214B9A4216
:102620002BD1FB8923F08003FB813B68DB891B01F5
:102630009AB2FB891343FB81FB8923F04003FB81A2
:102640003B689B881B019AB2FB891343FB81BB89C2
:1026500023F48063BB81BB8923F40063BB813B68A7
:102660001B8A9B009AB2BB891343BB813B685B8A80
:102670009B009AB2BB891343BB817B68BA899A805D
:102680007B687A891A833B689A687B689A637B685F
:10269000FA891A841437BD465DF8047B704700BF81
:1026A000000001400004014080B485B000AF7860B4
:1026B000396000237B810023FB810023BB817B6881
:1026C0001B8C9BB223F480739AB27B681A847B685C
:1026D0001B8CFB817B689B88BB817B689B8B7B8190
:1026E0007B8923F070037B817B8923F003037B814B
:1026F0003B681A887B8913437B81FB8923F4007331
:10270000FB813B689B891B029AB2FB891343FB81C7
:102710003B685B881B029AB2FB891343FB817A6892
:10272000224B9A4203D07A68214B9A422BD1FB89E3
:1027300023F40063FB813B68DB891B029AB2FB89AF
:102740001343FB81FB8923F48063FB813B689B88F7
:102750001B029AB2FB891343FB81BB8923F480538C
:10276000BB81BB8923F40053BB813B681B8A1B01DF
:102770009AB2BB891343BB813B685B8A1B019AB247
:10278000BB891343BB817B68BA899A807B687A894D
:102790009A833B689A687B68DA637B68FA891A8453
:1027A0001437BD465DF8047B704700BF0000014050
:1027B0000004014080B485B000AF78603960002328
:1027C000BB8100237B810023FB817B681B8C9BB238
:1027D00023F480539AB27B681A847B681B8C7B81BC
:1027E0007B689B88FB817B689B8BBB81BB8923F4C7
:1027F000E043BB81BB8923F44073BB813B681B88EA
:102800001B029AB2BB891343BB817B8923F400531B
:102810007B813B689B891B039AB27B8913437B8135
:102820003B685B881B039AB27B8913437B817A6880
:10283000114B9A4203D07A68104B9A420AD1FB8915
:1028400023F48043FB813B681B8A9B019AB2FB897E
:102850001343FB817B68FA899A807B68BA899A83E3
:102860003B689A687B681A647B687A891A84143793
:10287000BD465DF8047B7047000001400004014044
:1028800080B483B000AF78607B6800221A807B68D8
:1028900000225A807B6800229A807B6800229A601E
:1028A0007B6800229A817B680022DA817B680022A3
:1028B0001A827B6800225A820C37BD465DF8047B81
:1028C000704700BF80B485B000AF786013460A46F9
:1028D0007A803B800023FB6000237B817B68FB6068
:1028E000FB681833FB607B88012202FA03F37B81CB
:1028F0007B681B8C9AB27B89DB439BB213409AB2F4
:102900007B681A847B88002B02D07B88082B13D12C
:102910007B885B089BB2FA681344FB60FA68FB682B
:1029200019684FF68F730B401360FB68FA681168E3
:102930003A880A431A6016E07B88043B9BB25B0826
:102940009BB2FA681344FB60FA68FB68196848F6A2
:10295000FF730B401360FB68FA6811683A88120233
:1029600092B20A431A601437BD465DF8047B704783
:1029700080B483B000AF786039607B683A685A638E
:102980000C37BD465DF8047B704700BF80B483B050
:1029900000AF786039607B683A689A630C37BD464F
:1029A0005DF8047B704700BF80B483B000AF7860EF
:1029B00039607B683A68DA630C37BD465DF8047BA2
:1029C000704700BF80B483B000AF786039607B6827
:1029D0003A681A640C37BD465DF8047B704700BF47
:1029E00080B485B000AF78600B467B800023FB810C
:1029F0007B681B8BFB81FB8923F07003FB81FA89C9
:102A00007B881343FB817B68FA891A831437BD46A0
:102A10005DF8047B704700BF80B485B000AF78607C
:102A20000B467B800023FB817B681B8BFB81FB8932
:102A300023F4E043FB817B881B029AB2FB8913439A
:102A4000FB817B68FA891A831437BD465DF8047BE5
:102A5000704700BF80B485B000AF78600B467B80C4
:102A60000023FB817B689B8BFB81FB8923F0700338
:102A7000FB81FA897B881343FB817B68FA899A83FF
:102A80001437BD465DF8047B704700BF80B485B045
:102A900000AF78600B467B800023FB817B689B8BBB
:102AA000FB81FB8923F4E043FB817B881B029AB204
:102AB000FB891343FB817B68FA899A831437BD46EF
:102AC0005DF8047B704700BF80B485B000AF7860CC
:102AD0000B467B800023FB817B681B8BFB81FB8982
:102AE00023F00803FB81FA897B881343FB817B6811
:102AF000FA891A831437BD465DF8047B704700BF1E
:102B000080B485B000AF78600B467B800023FB81EA
:102B10007B681B8BFB81FB8923F40063FB817B8833
:102B20001B029AB2FB891343FB817B68FA891A83E3
:102B30001437BD465DF8047B704700BF80B485B094
:102B400000AF78600B467B800023FB817B689B8B0A
:102B5000FB81FB8923F00803FB81FA897B881343FF
:102B6000FB817B68FA899A831437BD465DF8047B44
:102B7000704700BF80B485B000AF78600B467B80A3
:102B80000023FB817B689B8BFB81FB8923F4006323
:102B9000FB817B881B029AB2FB891343FB817B6814
:102BA000FA899A831437BD465DF8047B704700BFED
:102BB00080B485B000AF78600B467B800023FB813A
:102BC0007B681B8BFB81FB8923F00403FB81FA8963
:102BD0007B881343FB817B68FA891A831437BD46CF
:102BE0005DF8047B704700BF80B485B000AF7860AB
:102BF0000B467B800023FB817B681B8BFB81FB8961
:102C000023F48063FB817B881B029AB2FB89134308
:102C1000FB817B68FA891A831437BD465DF8047B13
:102C2000704700BF80B485B000AF78600B467B80F2
:102C30000023FB817B689B8BFB81FB8923F00403D2
:102C4000FB81FA897B881343FB817B68FA899A832D
:102C50001437BD465DF8047B704700BF80B485B073
:102C600000AF78600B467B800023FB817B689B8BE9
:102C7000FB81FB8923F48063FB817B881B029AB272
:102C8000FB891343FB817B68FA899A831437BD461D
:102C90005DF8047B704700BF80B485B000AF7860FA
:102CA0000B467B800023FB817B681B8BFB81FB89B0
:102CB00023F08003FB81FA897B881343FB817B68C7
:102CC000FA891A831437BD465DF8047B704700BF4C
:102CD00080B485B000AF78600B467B800023FB8119
:102CE0007B681B8BFB81FB89C3F30E03FB817B8815
:102CF0001B029AB2FB891343FB817B68FA891A8312
:102D00001437BD465DF8047B704700BF80B485B0C2
:102D100000AF78600B467B800023FB817B689B8B38
:102D2000FB81FB8923F08003FB81FA897B881343B5
:102D3000FB817B68FA899A831437BD465DF8047B72
:102D4000704700BF80B485B000AF78600B467B80D1
:102D50000023FB817B689B8BFB81FB89C3F30E0304
:102D6000FB817B881B029AB2FB891343FB817B6842
:102D7000FA899A831437BD465DF8047B704700BF1B
:102D800080B485B000AF78600B467B800023FB8168
:102D90007B681B8CFB81FB8923F00203FB81FA8992
:102DA0007B881343FB817B68FA891A841437BD46FC
:102DB0005DF8047B704700BF80B485B000AF7860D9
:102DC0000B467B800023FB817B681B8CFB81FB898E
:102DD00023F00803FB81FA897B881343FB817B681E
:102DE000FA891A841437BD465DF8047B704700BF2A
:102DF00080B485B000AF78600B467B800023FB81F8
:102E00007B681B8CFB81FB8923F02003FB817B8883
:102E10001B019AB2FB891343FB817B68FA891A84F0
:102E20001437BD465DF8047B704700BF80B485B0A1
:102E300000AF78600B467B800023FB817B681B8C96
:102E4000FB81FB8923F08003FB817B881B019AB205
:102E5000FB891343FB817B68FA891A841437BD46CA
:102E60005DF8047B704700BF80B485B000AF786028
:102E70000B467B800023FB817B681B8CFB81FB89DD
:102E800023F40073FB817B881B029AB2FB891343F6
:102E9000FB817B68FA891A841437BD465DF8047B90
:102EA000704700BF80B485B000AF78600B467B8070
:102EB0000023FB817B681B8CFB81FB8923F400636F
:102EC000FB817B881B029AB2FB891343FB817B68E1
:102ED000FA891A841437BD465DF8047B704700BF39
:102EE00080B485B000AF78600B467B800023FB8107
:102EF0007B681B8CFB81FB8923F40053FB817B885F
:102F00001B039AB2FB891343FB817B68FA891A84FD
:102F10001437BD465DF8047B704700BF80B485B0B0
:102F200000AF786013460A467A803B800023FB811D
:102F30007B88012202FA03F3FB817B681B8C9AB227
:102F4000FB89DB439BB213409AB27B681A847B688F
:102F50001B8C9AB239887B8801FA03F39BB2134326
:102F60009AB27B681A841437BD465DF8047B7047BB
:102F700080B485B000AF786013460A467A803B8003
:102F80000023FB817B88042202FA03F3FB817B6828
:102F90001B8C9AB2FB89DB439BB213409AB27B68CD
:102FA0001A847B681B8C9AB239887B8801FA03F3F8
:102FB0009BB213439AB27B681A841437BD465DF8FE
:102FC000047B704780B582B000AF786039603B68A1
:102FD0001B88002B0FD13B6859883B689A883B6857
:102FE0001B89786800F092FC3B68DB88786819469A
:102FF00000F0E0F836E03B681B88042B0FD13B68FB
:1030000059883B689A883B681B89786800F0BAFC4D
:103010003B68DB887868194600F0E8F822E03B68F6
:103020001B88082B0FD13B6859883B689A883B68FE
:103030001B89786800F0ECFC3B68DB8878681946EF
:1030400000F0F2F80EE03B6859883B689A883B68CC
:103050001B89786800F01EFD3B68DB88786819469C
:1030600000F0FEF80837BD4680BD00BF80B483B0D5
:1030700000AF78607B6800221A807B6800225A804B
:103080007B6801229A807B680022DA807B680022BC
:103090001A810C37BD465DF8047B704780B584B05B
:1030A00000AF786039600023FB810123BB813B685E
:1030B0005B88002B02D10223FB8101E00023FB810E
:1030C0003B689B88012B02D10223BB8101E00123D5
:1030D000BB813B681B88002B1CD13B6859883B682F
:1030E0009A883B681B89786800F010FC3B68DB8895
:1030F0007868194600F05EF83B681B89F989BA893F
:10310000786800F03FFC3B68DB887868194600F07F
:103110006DF81BE03B6859883B689A883B681B89BF
:10312000786800F02FFC3B68DB887868194600F06F
:103130005DF83B681B89F989BA89786800F0E6FB7D
:103140003B68DB887868194600F034F81037BD46D4
:1031500080BD00BF80B483B000AF78607B685B6BDC
:1031600018460C37BD465DF8047B704780B483B0C9
:1031700000AF78607B689B6B18460C37BD465DF8E6
:10318000047B704780B483B000AF78607B68DB6BF2
:1031900018460C37BD465DF8047B704780B483B099
:1031A00000AF78607B681B6C18460C37BD465DF835
:1031B000047B704780B483B000AF78600B467B809F
:1031C0007B681B8B9BB223F00C039AB27B681A833B
:1031D0007B681B8B9AB27B8813439AB27B681A83F5
:1031E0000C37BD465DF8047B704700BF80B483B0E8
:1031F00000AF78600B467B807B681B8B9BB223F40F
:1032000040639AB27B681A837B681B8B9AB27B8877
:103210001B029BB213439AB27B681A830C37BD46DC
:103220005DF8047B704700BF80B483B000AF786066
:103230000B467B807B689B8B9BB223F00C039AB27E
:103240007B689A837B689B8B9AB27B8813439AB284
:103250007B689A830C37BD465DF8047B704700BFDE
:1032600080B483B000AF78600B467B807B689B8B1B
:103270009BB223F440639AB27B689A837B689B8BF2
:103280009AB27B881B029BB213439AB27B689A83E3
:103290000C37BD465DF8047B704700BF80B483B037
:1032A00000AF786039603B681A883B685B881343DD
:1032B0009AB23B689B8813439AB23B68DB881343FE
:1032C0009AB23B681B8913439AB23B685B891343EC
:1032D0009AB23B689B8913439AB27B68A3F8442057
:1032E0000C37BD465DF8047B704700BF80B483B0E7
:1032F00000AF78607B6800221A807B6800225A80C9
:103300007B6800229A807B680022DA807B6800223A
:103310001A817B6800225A817B6800229A810C37CF
:10332000BD465DF8047B704780B483B000AF786021
:103330000B46FB70FB78002B0CD07B68B3F8443055
:103340009BB26FEA43436FEA53439AB27B68A3F898
:10335000442009E07B68B3F844309BB2C3F30E030A
:103360009AB27B68A3F844200C37BD465DF8047B15
:10337000704700BF80B483B000AF78600B46FB702D
:10338000FB78002B08D07B689B889BB243F004033A
:103390009AB27B689A8007E07B689B889BB223F097
:1033A00004039AB27B689A800C37BD465DF8047BB3
:1033B000704700BF80B483B000AF78600B46FB70ED
:1033C000FB78002B08D07B689B889BB243F00103FD
:1033D0009AB27B689A8007E07B689B889BB223F057
:1033E00001039AB27B689A800C37BD465DF8047B76
:1033F000704700BF80B483B000AF786013460A46C0
:103400007A807B707B78002B08D07B689B899AB28E
:103410007B8813439AB27B689A8109E07B689B8919
:103420009AB27B88DB439BB213409AB27B689A8145
:103430000C37BD465DF8047B704700BF80B483B095
:1034400000AF78600B467B807B687A889A820C3765
:10345000BD465DF8047B704780B485B000AF7860EE
:103460000B467B800023FB737B681B8A9AB27B88A8
:1034700013409BB2002B02D00123FB7301E0002319
:10348000FB73FB7B18461437BD465DF8047B704721
:1034900080B483B000AF78600B467B807B88DB43D1
:1034A0009AB27B681A820C37BD465DF8047B704780
:1034B00080B485B000AF78600B467B800023FB733F
:1034C0000023BB8100237B817B681B8A9AB27B88A7
:1034D0001340BB817B689B899AB27B8813407B81B8
:1034E000BB89002B05D07B89002B02D00123FB7305
:1034F00001E00023FB73FB7B18461437BD465DF8E3
:10350000047B704780B483B000AF78600B467B804B
:103510007B88DB439AB27B681A820C37BD465DF824
:10352000047B704780B483B000AF786013460A46CE
:103530007A803B807A883B8813439AB27B68A3F8F1
:1035400048200C37BD465DF8047B704780B483B0DB
:1035500000AF786013460A467A807B707B78002B38
:1035600008D07B689B899AB27B8813439AB27B68A8
:103570009A8109E07B689B899AB27B88DB439BB286
:1035800013409AB27B689A810C37BD465DF8047B84
:10359000704700BF80B483B000AF78600B46FB700B
:1035A000FB78002B08D07B689B889BB243F0080314
:1035B0009AB27B689A8007E07B689B889BB223F075
:1035C00008039AB27B689A800C37BD465DF8047B8D
:1035D000704700BF80B483B000AF78607B681B8900
:1035E0009BB223F007039AB27B681A810C37BD4661
:1035F0005DF8047B704700BF80B582B000AF786093
:103600000B467B807B887868194600F075F87B68EC
:103610001B899BB243F007039AB27B681A81083773
:10362000BD4680BD80B584B000AFF86079813A8135
:10363000FB807B89602B07D13A89FB88F8681146AB
:10364000012200F09FF906E03A89FB88F8681146EC
:10365000012200F05BF97B89F868194600F04CF80C
:10366000FB681B899BB243F007039AB2FB681A817F
:103670001037BD4680BD00BF80B586B000AFF86092
:1036800079813A81FB800023FB8279893A89FB8822
:10369000F86800F0A1F8FB681B89FB82FB8A23F025
:1036A0000703FB82FB8A43F00703FB82FB8A23F0BC
:1036B0007003FB82FB8A43F07003FB82FB68FA8A8B
:1036C0001A811837BD4680BD80B584B000AFF86060
:1036D00079813A81FB8079893A89FB88F86800F022
:1036E0007BF8FB681B899BB243F480439AB2FB686A
:1036F0001A811037BD4680BD80B485B000AF7860B8
:103700000B467B800023FB817B681B89FB81FB8947
:1037100023F07003FB81FA897B881343FB817B686C
:10372000FA891A811437BD465DF8047B704700BFE3
:1037300080B483B000AF78600B467B807B689B8849
:103740009BB223F070039AB27B689A807B689B8857
:103750009AB27B8813439AB27B689A800C37BD4635
:103760005DF8047B704700BF80B483B000AF786021
:103770000B467B807B681B899BB223F007039AB2C0
:103780007B681A817B681B899AB27B8813439AB243
:103790007B681A810C37BD465DF8047B704700BF1B
:1037A00080B483B000AF78600B467B807B681B8958
:1037B0009BB223F080039AB27B681A817B681B89D5
:1037C0009AB27B8813439AB27B681A810C37BD4644
:1037D0005DF8047B704700BF80B487B000AFF8602D
:1037E00079813A81FB800023FB82FB681B89FB8285
:1037F000FB8ADBB2FB82FB881B029AB23B89134334
:103800009AB27B8913439AB2FB8A1343FB82FB680B
:10381000FA8A1A811C37BD465DF8047B704700BFE9
:1038200080B487B000AFF86079813A81FB800023D3
:10383000FB820023BB8200237B82FB681B89FB8207
:10384000FB681B8BBB82FB681B8C7B82FB8A23F093
:103850000703FB82FA8A7B891343FB82BB8A23F42A
:10386000407323F00303BB82BB8A43F4807343F0AD
:103870000103BB827B8A23F022037B82FB881B012E
:103880009AB23B8913439AB27B8A13437B82FB68CB
:10389000FA8A1A81FB68BA8A1A83FB687A8A1A84C0
:1038A0001C37BD465DF8047B704700BF80B483B011
:1038B00000AF78600B46FB70FB78002B08D07B686C
:1038C0009B889BB243F080039AB27B689A8007E0A2
:1038D0007B689B889BB223F080039AB27B689A80B6
:1038E0000C37BD465DF8047B704700BF80B483B0E1
:1038F00000AF78600B467B807B687A88A3F8502005
:103900000C37BD465DF8047B704700BF80B487B0BC
:1039100000AFF86079813A81FB800023FB820023AD
:10392000BB82FB681B8C9BB223F001039AB2FB683D
:103930001A84FB681B8BFB82FB681B8CBB82FB8A97
:1039400023F0F303FB82FB881B019AB23B891343EC
:103950009AB2FB8A1343FB82BB8A23F00A03BB8221
:103960007A89BB8A13439BB243F00103BB82FB6895
:10397000FA8A1A83FB68BA8A1A841C37BD465DF836
:10398000047B704780B487B000AFF86079813A81DA
:10399000FB800023FB820023BB8200237B82FB6829
:1039A0001B8C9BB223F010039AB2FB681A84FB684D
:1039B0001B8BFB82FB681B8CBB827B891B017B8280
:1039C000FB8A23F440731B051B0DFB82FB881B0342
:1039D0009AB2FB8A1343FB823B891B029AB2FB8A91
:1039E0001343FB82BB8A23F0A003BB827A8ABB8A83
:1039F00013439BB243F01003BB82FB68FA8A1A831D
:103A0000FB68BA8A1A841C37BD465DF8047B704790
:103A100080B487B000AFF86079813A81FB800023E1
:103A2000FB820023BB8200237B82FB681B8C9BB242
:103A300023F480739AB2FB681A84FB689B8BFB8229
:103A4000FB681B8CBB827B891B027B82FB8A23F079
:103A5000F303FB82FB881B019AB23B8913439AB2A2
:103A6000FB8A1343FB82BB8A23F42063BB827A8ADE
:103A7000BB8A13439BB243F48073BB82FB68FA8A10
:103A80009A83FB68BA8A1A841C37BD465DF8047BAA
:103A9000704700BF80B487B000AFF86079813A8189
:103AA000FB800023FB820023BB8200237B82FB6818
:103AB0001B8C9BB223F480539AB2FB681A84FB6878
:103AC0009B8BFB82FB681B8CBB827B891B037B82ED
:103AD000FB8A23F440731B051B0DFB823B891B02F1
:103AE0009AB2FB8A1343FB82FB881B039AB2FB8AC0
:103AF0001343FB82BB8A23F400535B045B0CBB8241
:103B00007A8ABB8A13439BB243F48053BB82FB681F
:103B1000FA8A9A83FB68BA8A1A841C37BD465DF814
:103B2000047B704780B582B000AF78607A683A4B0A
:103B30009A4208D110200121FEF746F810200021FA
:103B4000FEF742F865E07A68344B9A420AD14FF4A6
:103B500000300121FEF71AF84FF400300021FEF783
:103B600015F856E07A682E4B9A420AD14FF480201D
:103B70000121FEF70BF84FF480200021FEF706F834
:103B800047E07A68274B9A420AD14FF4002001217E
:103B9000FDF7FCFF4FF400200021FDF7F7FF38E0B0
:103BA0007A68214B9A420AD14FF480100121FDF727
:103BB000EDFF4FF480100021FDF7E8FF29E07A685F
:103BC0001A4B9A4208D120200121FDF7FDFF202049
:103BD0000021FDF7F9FF1CE07A68154B9A420AD1E3
:103BE0004FF080400121FDF7D1FF4FF080400021D0
:103BF000FDF7CCFF0DE07A680E4B9A4209D14FF0E9
:103C000000400121FDF7C2FF4FF000400021FDF709
:103C1000BDFF0837BD4680BD001001400044004094
:103C200000480040004C004000500040001401409B
:103C300000780040007C004080B58AB000AF78601A
:103C4000396000237B6200233B620023FB61002379
:103C5000BB617B681B8A9BB27B627B6A23F4405307
:103C60007B623B68DB887A6A13437B627B6A9AB229
:103C70007B681A827B689B899BB27B627B6A23F498
:103C8000B05323F00C037B623B689A883B681B8926
:103C900013439AB23B685B8913439BB27A6A13431E
:103CA0007B627B6A9AB27B689A817B689B8A9BB2B3
:103CB0007B627B6A23F440737B623B689B897A6AF0
:103CC00013437B627B6A9AB27B689A8207F108038E
:103CD0001846FDF737FD7A68314B9A4203D07A686F
:103CE000304B9A4202D17B693B6201E03B693B6207
:103CF0007B689B899BB29BB21BB2002B0CDA3A6AA1
:103D000013469B0013449A001A443B681B685B00EF
:103D1000B2FBF3F3FB610BE03A6A13469B001344DA
:103D20009A001A443B681B689B00B2FBF3F3FB61EB
:103D3000FA691D4BA3FB02135B091B017B627B6AC3
:103D40001B09642202FB03F3FA69D31ABB617B6887
:103D50009B899BB29BB21BB2002B0DDABB69DB00C7
:103D600003F13202104BA3FB02135B0903F00703BC
:103D70007A6A13437B620CE0BB691B0103F13202D8
:103D8000094BA3FB02135B0903F00F037A6A134389
:103D90007B627B6A9AB27B681A812837BD4680BDF8
:103DA00000100140001401401F85EB5180B483B026
:103DB00000AF78607B684FF416521A607B6800226F
:103DC0009A807B680022DA807B6800221A817B68F7
:103DD0000C225A817B6800229A810C37BD465DF81F
:103DE000047B704780B485B000AF786039600023F1
:103DF000FB607B681B8A9BB2FB60FB6823F47063EB
:103E0000FB603B681A883B685B8813439AB23B6847
:103E10009B8813439AB23B68DB8813439BB2FA68D2
:103E20001343FB60FB689AB27B681A821437BD4665
:103E30005DF8047B704700BF80B483B000AF78604A
:103E40007B6800221A807B6800225A807B680022EF
:103E50009A807B680022DA800C37BD465DF8047BCF
:103E6000704700BF80B483B000AF78600B46FB7032
:103E7000FB78002B08D07B689B899BB243F40053EE
:103E80009AB27B689A8107E07B689B899BB223F496
:103E900000539AB27B689A810C37BD465DF8047B6B
:103EA000704700BF80B483B000AF78600B46FB70F2
:103EB0007B681B8B9BB223F0FF039AB27B681A834B
:103EC0007B681B8B9AB2FB789BB213439AB27B68D8
:103ED0001A830C37BD465DF8047B704780B483B00D
:103EE00000AF78600B46FB70FB78002B0AD07B6834
:103EF0009B899BB26FEA43436FEA53439AB27B6854
:103F00009A8107E07B689B899BB2C3F30E039AB248
:103F10007B689A810C37BD465DF8047B704700BF13
:103F200080B483B000AF78600B46FB70FB78002B49
:103F300008D07B689B8A9BB243F400639AB27B688B
:103F40009A8207E07B689B8A9BB223F400639AB253
:103F50007B689A820C37BD465DF8047B704700BFD2
:103F600080B483B000AF78600B467B807B88C3F35E
:103F700008039AB27B689A800C37BD465DF8047BD3
:103F8000704700BF80B483B000AF78607B689B88C7
:103F90009BB2C3F308039BB218460C37BD465DF8CD
:103FA000047B704780B483B000AF78600B46FB7031
:103FB0007B681B8A9BB223F00F039AB27B681A823C
:103FC0007B681B8A9AB2FB789BB213439AB27B68D8
:103FD0001A820C37BD465DF8047B704780B483B00D
:103FE00000AF78600B46FB70FB78002B08D07B6835
:103FF0009B899BB243F002039AB27B689A8107E0E7
:104000007B689B899BB223F002039AB27B689A81FA
:104010000C37BD465DF8047B704700BF80B483B0A9
:1040200000AF78600B467B807B689B899BB223F452
:1040300000639AB27B689A817B689B899AB27B887D
:1040400013439AB27B689A810C37BD465DF8047BB6
:10405000704700BF80B483B000AF78600B467B80B0
:104060007B681B8A9BB223F020039AB27B681A827A
:104070007B681B8A9AB27B8813439AB27B681A8248
:104080000C37BD465DF8047B704700BF80B483B039
:1040900000AF78600B46FB70FB78002B08D07B6884
:1040A0001B8A9BB243F480439AB27B681A8207E072
:1040B0007B681B8A9BB223F480439AB27B681A8286
:1040C0000C37BD465DF8047B704700BF80B483B0F9
:1040D00000AF78607B689B899BB243F001039AB282
:1040E0007B689A810C37BD465DF8047B704700BF42
:1040F00080B483B000AF78600B46FB70FB78002B78
:1041000008D07B689B8A9BB243F008039AB27B6815
:104110009A8207E07B689B8A9BB223F008039AB2DD
:104120007B689A820C37BD465DF8047B704700BF00
:1041300080B483B000AF78600B46FB707B681B8B4C
:104140009BB2DBB29AB27B681A837B681B8B9AB2F4
:10415000FB789BB21B029BB213439AB27B681A8313
:104160000C37BD465DF8047B704700BF80B483B058
:1041700000AF78600B46FB70FB78002B08D07B68A3
:104180009B8A9BB243F020039AB27B689A8207E035
:104190007B689B8A9BB223F020039AB27B689A8249
:1041A0000C37BD465DF8047B704700BF80B483B018
:1041B00000AF78600B46FB70FB78002B08D07B6863
:1041C0009B8A9BB243F010039AB27B689A8207E005
:1041D0007B689B8A9BB223F010039AB27B689A8219
:1041E0000C37BD465DF8047B704700BF80B483B0D8
:1041F00000AF78600B467B807B689B8A9BB223F084
:1042000004039AB27B689A827B689B8A9AB27B8805
:1042100013439AB27B689A820C37BD465DF8047BE3
:10422000704700BF80B483B000AF78600B46FB706E
:10423000FB78002B08D07B689B8A9BB243F002037B
:104240009AB27B689A8207E07B689B8A9BB223F0D4
:1042500002039AB27B689A820C37BD465DF8047BF4
:10426000704700BF80B483B000AF786013460A4641
:104270007A807B707B78002B08D07B689B8A9AB20F
:104280007B8813439AB27B689A8209E07B689B8A99
:104290009AB27B88DB439BB213409AB27B689A82C6
:1042A0000C37BD465DF8047B704700BF80B487B013
:1042B00000AF786013460A467A807B7000233B612A
:1042C0000023FB600023BB6000237B617B687B6174
:1042D0007B88DBB25B09DBB23B617B8803F01F03A9
:1042E000FB60FB68012202FA03F3BB603B69012B10
:1042F00003D17B690C337B6109E03B69022B03D15D
:104300007B6910337B6102E07B6914337B617B78CE
:10431000002B06D07B697A691168BA680A431A6073
:1043200006E07B697A691168BA68D2430A401A606C
:104330001C37BD465DF8047B704700BF80B485B074
:1043400000AF78600B467B800023FB737B681B8883
:104350009AB27B8813409BB2002B02D00123FB73DF
:1043600001E00023FB73FB7B18461437BD465DF864
:10437000047B704780B483B000AF78600B467B80CD
:104380007B88DB439AB27B681A800C37BD465DF8A8
:10439000047B704780B487B000AF78600B467B80A9
:1043A0000023FB6000237B610023BB600023FB74C0
:1043B0007B88DBB25B09DBB2BB607B8803F01F0349
:1043C0007B617B69012202FA03F37B61BB68012BED
:1043D00006D17B689B899BB27A6913407B610FE0B1
:1043E000BB68022B06D17B681B8A9BB27A6913409B
:1043F0007B6105E07B689B8A9BB27A6913407B6195
:104400007B881B0A9BB2FB60FB68012202FA03F364
:10441000FB607B681B889BB2FA681340FB607B697A
:10442000002B05D0FB68002B02D00123FB7401E0B8
:104430000023FB74FB7C18461C37BD465DF8047BEB
:10444000704700BF80B485B000AF78600B467B80BA
:104450000023FB810023BB817B881B0AFB81FB8936
:10446000012202FA03F3BB81BB89DB439AB27B686A
:104470001A801437BD465DF8047B704780B483B062
:1044800000AF0346FB71084B97F907205209F979F1
:1044900001F01F01012000FA01F143F822100C374E
:1044A000BD465DF8047B704700E100E080B483B056
:1044B00000AF0346FB71094B97F907205209F979C0
:1044C00001F01F01012000FA01F1203243F822100F
:1044D0000C37BD465DF8047B704700BF00E100E08B
:1044E00080B483B000AF03463960FB7197F90730A1
:1044F000002B0BDA0D49FB7903F00F03043B3A68FC
:10450000D2B21201D2B20B441A7609E0084997F9E7
:1045100007303A68D2B21201D2B20B4483F80023BA
:104520000C37BD465DF8047B704700BF00ED00E02E
:1045300000E100E080B582B000AF78607B68013BAD
:10454000B3F1807F01D301230FE00A4B7A68013A6F
:104550005A604FF0FF300F21FFF7C2FF054B0022DA
:104560009A60044B07221A60002318460837BD469C
:1045700080BD00BF10E000E080B400AF064BD3E97F
:104580000023013243F100030349C1E90023BD4682
:104590005DF8047B704700BFF00A002080B586B04C
:1045A00000AF78600420FCF73BFB07F108031846D6
:1045B000FDF7C8F8FA687B68B2FBF3F31846FFF71B
:1045C000B9FF7A68034B1A60034B01221A7018373F
:1045D000BD4680BDD8100020E80A002080B400AF9E
:1045E0000B4BD3E90023013243F100030849C1E931
:1045F00000234FF080434FF08042128A92B222F0A3
:10460000010292B21A82BD465DF8047B704700BF7A
:10461000F00A002080B582B000AF7860064B02221D
:104620001A70022079681C2201F078F90246034BC7
:104630001A600837BD4680BDE80A0020D810002067
:1046400080B582B000AF78600220796801F0B4F8DC
:104650000246044B1A60044B03221A700837BD4609
:1046600080BD00BFD8100020E80A002080B586B0C9
:1046700000AF264B1B78032B3ED801A252F823F043
:10468000914600089B460008BB460008E346000828
:104690004FF000024FF0000332E04FF0FF30FFF721
:1046A00005FF1B4BD3E90023C7E904234FF0FF307C
:1046B000FFF7E4FED7E9042322E04FF08040012118
:1046C0000022FEF797FE124BD3E90023C7E902232D
:1046D0004FF0804001210122FEF78CFED7E9022332
:1046E0000EE04FF080435B6A1A464FF00003C7E9C3
:1046F0000023D7E9002303E04FF000024FF000034E
:10470000104619461837BD4680BD00BFE80A002094
:10471000F00A002080B582B000AF7860224B1B7891
:10472000032B3ED801A252F823F000BFA347000894
:104730003D4700085D470008854700084FF0FF30FF
:10474000FFF7B4FE7B681A464FF000031749C1E932
:1047500000234FF0FF30FFF791FE22E04FF0804042
:1047600001210022FEF746FE7B681A464FF0000347
:104770000E49C1E900234FF0804001210122FEF7DC
:1047800039FE0EE04FF080400021FDF76BFE4FF048
:1047900080437A685A624FF080400121FDF762FE43
:1047A00000BF0837BD4680BDE80A0020F00A00209F
:1047B00080B584B000AF7860FFF758FF02460B4623
:1047C0001346FB601B4B1B6806EE903AB8EE667A08
:1047D0007B6806EE903AF8EEE67A67EE277A17EEF7
:1047E000900A05F077FD02460B46104619464FF039
:1047F0000002114B05F0ECFE02460B46104619462E
:1048000005F0CEFF0346BB6000BFFFF72FFFFB683C
:104810001A464FF00003801A61EB0301BB681A4689
:104820004FF00003904271EB030CEEDB1037BD46F6
:1048300080BD00BFD810002000408F402DE9B04F50
:1048400086B000AF786039607B68002B4CD0FFF7F2
:104850000DFF02460B46C7E90423D7E904010246CF
:104860000B464FEA432B4BEAD25B4FEA422A5246B1
:104870005B465D0145EAD2655401A41A65EB030568
:10488000241845EB01054FEA851949EA94694FEA76
:104890008418B8EB040869EB050910EB080041EB3C
:1048A0000901144B1B681A464FF0000305F098FFEE
:1048B00002460B46C7E90223D7E9022310461946F0
:1048C0000D4A4FF0000305F08BFF02460B467B6854
:1048D0001A60D7E9022310461946074A4FF0000331
:1048E00005F07EFF7B685A60002318461837BD46E6
:1048F000BDE8B08FD810002040420F002DE9B04F26
:1049000086B000AF78603960796800294ED0796848
:1049100009688A464FEAEA7B504659464FEA4129E0
:1049200049EAD0594FEA4028404649464B0143EAFC
:10493000D0634201121A63EB010312EB0A0243EB4C
:104940000B039D0145EA92659401A41A65EB0305EA
:1049500014EB0A0045EB0B017B685B681A464FEAD3
:10496000E273121843EB0103C7E90423124B1B68DF
:104970001A464FF00003396903FB01F0796902FB25
:1049800001F101443869A0FB022319440B4610468B
:1049900019460A4A4FF0000305F022FF02460B4673
:1049A000C7E90223BB681846FFF7B4FE0023184688
:1049B0001837BD46BDE8B08FD810002040420F0028
:1049C00080B584B000AF78607B68082B02DC7B6820
:1049D000002B02DA4FF0FF3314E07B68DA000B4B58
:1049E0001344FB60FB681B68BB60BB68002B02D1F3
:1049F0006FF0010306E0FB685B6818460121FDF7D4
:104A000011F8002318461037BD4680BD201E01084E
:104A100080B584B000AF78607B68002B03D07B68E2
:104A20001B78002B01D1002345E0786807F0F8FCE3
:104A30000346032B01D800233DE07B681B78FB6015
:104A40001F4B1A68FB68013313441B7803F0030300
:104A5000022B02D1FB68203B00E0FB68413B0E2BA0
:104A600028D801A252F823F0B14A0008B54A00083C
:104A7000B54A0008B54A0008B54A0008AD4A000822
:104A8000B54A0008B54A0008A54A0008B54A00081A
:104A9000B54A0008B54A0008B54A0008B54A0008FA
:104AA000A94A0008002306E0012304E0022302E0F3
:104AB000032300E0002318461037BD4680BD00BF29
:104AC0002002002080B584B000AF78607B68002BA6
:104AD00003D07B681B78002B01D1012325E0786887
:104AE00007F09EFC0346032B01D801231DE07B68E1
:104AF00001331B78FB600F4B1A68FB6801331344CA
:104B00001B7803F00303022B02D1FB68203B00E07B
:104B1000FB684F2B06D0502B02D0442B02D003E071
:104B2000002302E0012300E0012318461037BD46B0
:104B300080BD00BF2002002080B584B000AF786047
:104B40007B68002B03D07B681B78002B01D10023EE
:104B500063E0786807F064FC0346032B01D8002368
:104B60005BE07B6802331B78FB602E4B1A68FB68A6
:104B7000013313441B7803F00303022B02D1FB68BB
:104B8000203B00E0FB68313B1C2B45D801A252F8CA
:104B900023F000BF154C0008094C0008194C000810
:104BA000194C0008114C0008194C0008194C000859
:104BB000194C0008194C0008194C0008194C000841
:104BC000194C0008194C0008194C0008194C000831
:104BD000194C0008194C0008194C0008194C000821
:104BE000194C0008194C0008114C0008194C000819
:104BF000154C0008194C0008194C0008194C000805
:104C0000094C00080D4C0008002306E0012304E0D5
:104C1000022302E0032300E0002318461037BD46BC
:104C200080BD00BF2002002080B584B000AF786056
:104C30007B68002B03D07B681B78002B01D10023FD
:104C400027E0786807F0ECFB0346032B01D800232C
:104C50001FE07B6803331B78FB60104B1A68FB680E
:104C6000013313441B7803F00303022B02D1FB68CA
:104C7000203B00E0FB684E2B04D0552B04D0442B86
:104C800004D005E0002304E0012302E0022300E059
:104C9000002318461037BD4680BD00BF200200200B
:104CA00080B487B000AF78607B68002B02D14FF0F2
:104CB000FF333FE07B681B78002B02D16FF00103CC
:104CC00038E07B681B787B611D4B1A687B69013378
:104CD00013441B7803F00303022B02D17B69203BB2
:104CE00000E07B69502B02D17B6801337B607B68DD
:104CF0001B783B61124B1A683B69013313441B78E4
:104D000003F00303022B02D13B69203B00E03B6927
:104D1000FB73FB7B002B02D16FF002030AE0FB7BED
:104D2000402B02D9FB7B4A2B02D96FF0030301E031
:104D3000FB7B413B18461C37BD465DF8047B704742
:104D40002002002080B584B000AF78607B68002B23
:104D500002D14FF0FF3344E07B681B78002B02D177
:104D60006FF001033DE07B681B78FB601F4B1A6806
:104D7000FB68013313441B7803F00303022B02D1B9
:104D8000FB68203B00E0FB68502B02D17B680133BD
:104D90007B607B681B78002B02D16FF0020320E060
:104DA0007B6801337B607B681B78002B02D16FF03E
:104DB000030316E00D4B1A687B681B78013313441C
:104DC0001B7803F00403002B02D16FF0040308E00A
:104DD000786800210A2207F069FE0346012202FAE0
:104DE00003F318461037BD4680BD00BF20020020E7
:104DF00080B584B000AF78607B68002B02D14FF0A3
:104E0000FF3341E07B681B78002B02D16FF0010378
:104E10003AE07B681B78FB601D4B1A68FB68013326
:104E200013441B7803F00303022B02D1FB68203BE1
:104E300000E0FB68502B02D17B6801337B607B680C
:104E40001B78002B02D16FF002031DE07B68013359
:104E50007B607B681B78002B02D16FF0030313E0AB
:104E60000B4B1A687B681B78013313441B7803F0E3
:104E70000403002B02D16FF0040305E078680021E1
:104E80000A2207F013FE034618461037BD4680BDC0
:104E90002002002080B588B000AFF860B960FA71D8
:104EA000BB71FB68082B02DCFB68002B02DA4FF0B9
:104EB000FF3329E0FB68DA00154B1344FB61FB6903
:104EC0001B68BB61BB69002B02D16FF001031BE0C3
:104ED000F868FFF775FD0346002B02DA6FF0020356
:104EE00012E0BB683B61FB793B7597F82830BB75D6
:104EF000BB797B7597F82C30FB7507F11003B86907
:104F00001946FCF75BF8002318462037BD4680BDE4
:104F1000201E0108F0B587B002AF7860396078686C
:104F2000FFF7BEFEF8607868FFF70CFFB860FB681B
:104F3000002B02DBBB68002B02DA4FF0FF3321E0CD
:104F40003868FFF765FD03461D463868FFF7F4FD36
:104F500003461C463868FFF7B5FD03461E46386811
:104F6000FFF762FE034600960193F868B9682A4687
:104F70002346FFF78FFF0346002B02DA6FF0010391
:104F800000E0002318461437BD46F0BD80B586B05A
:104F900002AF78607868FFF783FEF8607868FFF703
:104FA000D1FEB860FB68002B02DBBB68002B02DA85
:104FB0004FF0FF3310E00023009301230193F868C2
:104FC000B96800220023FFF765FF0346002B02DAD1
:104FD0006FF0010300E0002318461037BD4680BD86
:104FE00080B586B002AF78607868FFF759FEF86048
:104FF0007868FFF7A7FEB860FB68002B02DBBB6890
:10500000002B02DA4FF0FF3310E00023009300235F
:105010000193F868B96801220123FFF73BFF0346BB
:10502000002B02DA6FF0010300E00023184610376E
:10503000BD4680BD80B586B002AF78607868FFF766
:105040002FFEF8607868FFF77DFEB860FB68002BE4
:1050500002DBBB68002B02DA4FF0FF3310E00023C5
:10506000009300230193F868B96803220123FFF736
:1050700011FF0346002B02DA6FF0010300E000236A
:1050800018461037BD4680BD80B588B002AF786045
:105090000B46FB707868FFF703FE78617868FFF7CE
:1050A00051FE38617868FFF7A3FEF8607B69002B3A
:1050B00002DB3B69002B02DA4FF0FF3316E00023DE
:1050C0000093002301937869396902220023FFF7D6
:1050D000E1FE084B7A6953F83210FB689AB2FB780C
:1050E000084611461A46FCF7D7F800231846183729
:1050F000BD4680BD201E010880B58AB000AFF860B3
:10510000B9607A60F868FFF7CBFD03467B62F86808
:10511000FFF76EFE03463B62F868FFF737FF7B68D8
:10512000002B05DB7B68DBB2F8681946FFF7ACFFA4
:105130004FF480400121FCF7CFFC7B6ADAB23B6A76
:10514000DBB210461946FCF7B7FE3B6A012202FAB1
:1051500003F3BB6100233B77BB68002B02DA0C230F
:105160007B770AE0BB68002B02D110237B7704E039
:10517000BB68002B01DD08237B770123BB7707F198
:1051800018031846FBF782FD3B6A002B02D1062369
:105190003B7528E03B6A012B02D107233B7522E0D7
:1051A0003B6A022B02D108233B751CE03B6A032BB0
:1051B00002D109233B7516E03B6A042B02D10A2376
:1051C0003B7510E03B6A042B05D93B6A092B02D8DA
:1051D00017233B7507E03B6A092B04D93B6A0F2B69
:1051E00001D828233B7500237B753B6ADBB2BB7576
:1051F0000123FB7507F114031846FBF77DFC3B6A9E
:1052000018462837BD4680BD80B584B000AF7860B1
:1052100039607868FFF744FDF8607868FFF792FD21
:10522000B860FB68002B02DBBB68002B02DA4FF092
:10523000FF3311E00A4BFA6853F83210BB689AB298
:105240003B68002B0CBF00230123DBB2084611464C
:105250001A46FBF7E9FF3B6818461037BD4680BD8C
:10526000201E010880B584B000AF78607868FFF731
:1052700017FDF8607868FFF765FDB860FB68002BE4
:1052800002DBBB68002B02DA4FF0FF330FE00A4B62
:10529000FA6853F83220BB689BB210461946FBF7F8
:1052A00057FF0346012B14BF00230123DBB218462E
:1052B0001037BD4680BD00BF201E010880B588B0F4
:1052C00000AF78607868FFF7EBFCF8617868FFF76B
:1052D0008FFDB861FB69002B02DBFB69082B01DD48
:1052E000002313E0FB69DA000A4B13447B617B69FE
:1052F0001B68143303F140433B613B6903F10473C2
:105300005A01BB699B001344FB60FB6818462037B9
:10531000BD4680BD201E010880B588B000AF786012
:105320007868FFF7BDFCF8617868FFF761FDB86148
:10533000FB69002B02DBFB69082B01DD002313E076
:10534000FB69DA000A4B13447B617B691B681033ED
:1053500003F140433B613B6903F104735A01BB69AC
:105360009B001344FB60FB6818462037BD4680BD98
:10537000201E010880B590B006AF786039603868AB
:10538000FFF78EFC38623868FFF7DCFCF86138689C
:10539000FFF72EFDB8613B6A002BC0F2DE80FB698F
:1053A000002BC0F2DA806E4B3A6A53F832307B61E0
:1053B00000237B6219E03B6A41337A6A91007A6A82
:1053C0009200786902441268386A0090F869019086
:1053D000786A029003910492786862491A46BB6920
:1053E00005F0D4FC7B6A01337B627B6A092BE2DD2A
:1053F000BB69072B0ADC7B6920331A68BB699B00F9
:1054000022FA03F303F00F037B620AE07B69243383
:105410001A68BB69083B9B0022FA03F303F00F03F1
:105420007B62786850497A6A7B6A05F0AFFC7B69D9
:105430001A68BB695B0022FA03F303F003037B6283
:105440004A4B7A6A53F82230786849497A6A05F0FB
:105450009DFC464B7A6A53F822301B783B737B697C
:1054600004331A68FB6913407B627B6A002B0CBF14
:1054700000230123DBB21A463E4B53F822307868F2
:105480003D497A6A05F082FC7B6A002B0CBF002341
:105490000123DBB21A46374B53F822301B787B735B
:1054A0007B6908331A68BB695B0022FA03F303F0D7
:1054B00003037B62314B7A6A53F8223078683049B3
:1054C0007A6A05F063FC2D4B7A6A53F822301B7818
:1054D000BB737B690C331A68BB695B0022FA03F368
:1054E00003F003037B62274B7A6A53F82230786813
:1054F00025497A6A05F04AFC224B7A6A53F8223031
:105500001B78FB7300233B7407F10C0378681F4979
:105510001A4605F03BFC7B6910331A68FB6913409F
:105520007B627B6A002B0CBF00230123DBB278680F
:1055300017491A4605F02AFC7B6914331A68FB697F
:1055400013407B627B6A002B0CBF00230123DBB27C
:10555000786810491A4605F019FC2837BD4680BD09
:10556000201E0108001F0108281F01082C00002030
:105570003C1F01083C0000204C1F01084400002093
:105580005C1F0108540000206C1F01087C1F0108EB
:10559000881F0108941F010880B582B000AF7860B1
:1055A0007B68013B0D2B69D801A252F823F000BFA4
:1055B000E9550008F3550008FD5500080756000896
:1055C000115600081B560008255600082F560008E3
:1055D0003956000845560008515600085D56000827
:1055E000675600087156000801200121FCF774FA83
:1055F00044E001200121FCF751FA3FE002200121A3
:10560000FCF74CFA3AE004200121FCF747FA35E0B8
:1056100008200121FCF742FA30E010200121FCF7BC
:105620003DFA2BE020200121FCF738FA26E0022089
:105630000121FCF751FA21E04FF480300121FCF701
:105640004BFA1BE04FF400300121FCF745FA15E05E
:105650004FF480200121FCF73FFA0FE040200121A8
:10566000FCF71CFA0AE080200121FCF717FA05E09C
:105670004FF480700121FCF711FA00BF0837BD46D6
:1056800080BD00BF80B582B000AF786039607B68B4
:10569000013B0D2B5AD801A252F823F0D556000831
:1056A000DF560008E9560008F3560008FD560008CA
:1056B0004D5700084D5700080757000811570008BC
:1056C0001B570008255700082F57000839570008B6
:1056D0004357000838680121FFF7D6FC36E03868E8
:1056E0000121FFF7D1FC31E038680221FFF7CCFC43
:1056F0002CE038680221FFF7C7FC27E03868022158
:10570000FFF7C2FC22E038680321FFF7BDFC1DE073
:1057100038680321FFF7B8FC18E038680321FFF769
:10572000B3FC13E038680321FFF7AEFC0EE03868E5
:105730000921FFF7A9FC09E038680921FFF7A4FC5B
:1057400004E038680921FFF79FFC00BF0837BD4619
:1057500080BD00BF80B588B000AF786007F10C0352
:105760001846FBF7EFFF7B68012B05D07B68072B02
:105770000FDD7B680B2B0CDCBB69FB610D4B9B6861
:1057800003F40043002B03D0FB695B00FB610BE0DB
:105790000AE07B69FB61074B9B6803F48053002B95
:1057A00002D0FB695B00FB61FB6918462037BD46F0
:1057B00080BD00BF0038024080B58AB000AF78607D
:1057C00039604FF6FF737B627B68122B01DD00238B
:1057D00045E0254B7A6853F822303B623B6A002B48
:1057E00001D100233BE07868FFF7D6FE7868FFF729
:1057F000B1FFF8617B68022B02D07B68052B02D1D8
:105800004FF0FF337B623B68BB61FA69BB69B2FB57
:10581000F3F3013B7B617B69B3F5803F03D34FF624
:10582000FF733B8102E07B699BB23B813B89013383
:10583000FA69B2FBF3F3BB617B6AFB6000237B81F7
:1058400000233B820023BB7407F10803386A194622
:10585000FCF786FC386A0121FCF704FEBB69184698
:105860002837BD4680BD00BFA01F010880B588B0A5
:1058700000AF786039607B68122B01DD002345E0C2
:10588000244B7A6853F82230BB61BB69002B01D1ED
:1058900000233BE07868FFF77FFE7868FFF75AFF48
:1058A00078617B68022B02D07B68052B02D11A4BF2
:1058B000FB6102E04EF66023FB617A69FB69B2FB93
:1058C000F3F39BB2013B9BB23B813B8901337A6985
:1058D000B2FBF3F3FB61FA693B68B2FBF3F3FB60E5
:1058E000FB68FA69B2FBF3F33B6000237B81002382
:1058F0003B820023BB7407F10803B8691946FCF723
:105900002FFCB8690121FCF7ADFD3B681846203734
:10591000BD4680BDA01F010840420F0080B586B083
:1059200000AFF860B9601346FB71FB68122B01DD14
:10593000002321E0124BFA6853F822307B617B6927
:10594000002B01D1002317E0F868B968FFF78EFF3C
:10595000B860FB793B7400237B740023BB74012384
:10596000FB7407F110031846FBF7C6F878690121AC
:105970000122FDF73FFDBB6818461837BD4680BDC4
:10598000A01F010880B483B000AF786087ED000AE3
:10599000284B00221A607B6807EE903AB8EEE77A4F
:1059A000244B1B68013307EE903AF8EEE76AD7ED17
:1059B000007A66EEA77AC7EE277AFDEEE77A17EE51
:1059C000902A1D4B1A601CE01A4B1B685A1C194B7D
:1059D0001A607B6807EE903AB8EEE77A154B1B68C1
:1059E000013307EE903AF8EEE76AD7ED007A66EEFB
:1059F000A77AC7EE277AFDEEE77A17EE902A0E4BCC
:105A00001A600D4B1B68B3F5803F04DB094B1B6824
:105A1000B3F5803FD8DB074B1A684FF6FF739A4205
:105A2000CCBF00230123DBB218460C37BD465DF81E
:105A3000047B7047F80A0020FC0A0020B0B58EB045
:105A400000AFF86087ED020AC7ED010A3960FB6814
:105A5000122B01DD0123CFE0694BFA6853F82230A5
:105A60007B637B6B002B01D10223C5E03B68002BDD
:105A700001D10323C0E0F868FFF76CFE03463B63E7
:105A800097ED027ADFED5F7AB4EEE77AF1EE10FA85
:105A900001DD5D4BBB60386B97ED020AFFF772FFCB
:105AA0000346002B01D10423A6E0F868FFF774FD3C
:105AB000786B0021FCF7D6FC544B1B689BB2BB846F
:105AC0000023FB84524B1B68BB620023BB85002371
:105AD00087F82E3007F12403786B1946FCF740FB5A
:105AE00060233B8201237B820423BB8200233B840F
:105AF00000237B84464B1B68184604F0D9FB044600
:105B00000D46786804F0E6FB02460B46104619463F
:105B10004FF000023F4B04F05BFD02460B4620466F
:105B2000294604F02BFC02460B461046194604F0A9
:105B300037FE0346BB610023BB830023FB833B6826
:105B400003F00103002B0ED007F11003786B194608
:105B5000FCF7A8FC786B0021FCF7B6FF786B0021FE
:105B60000122FDF7DBF93B6803F00203002B0ED0A6
:105B700007F11003786B1946FCF70EFD786B0021D6
:105B8000FCF7BEFF786B04210122FDF7C7F93B68E3
:105B900003F00403002B0ED007F11003786B1946B5
:105BA000FCF782FD786B0021FCF7C8FF786B0821B9
:105BB0000122FDF7B3F93B6803F00803002B0ED078
:105BC00007F11003786B1946FCF7F4FD786B0021A0
:105BD000FCF7D0FF786B0C210122FDF79FF9786B61
:105BE0000121FDF7A1FB786B0121FCF7E3FB786B4A
:105BF0000121FCF737FC002318463837BD46B0BDFD
:105C0000A01F01080000AF440000AF44F80A0020C4
:105C1000FC0A002000005940B0B58CB000AFF8601D
:105C200087ED020AC7ED010A0B46FB70FB68122BD9
:105C300001DD01237BE1084BFA6853F82230FB6257
:105C4000FB6A002B01D1022371E1FB7803F00F0303
:105C5000002B05D103236AE1A01F01080000AF4417
:105C6000F868FFF777FD0346BB6297ED027A5FEDB8
:105C7000057AB4EEE77AF1EE10FA01DDAE4BBB60C7
:105C8000B86A97ED020AFFF77DFE0346002B00F08D
:105C90004D81FB6ADB6A07EE103AF8EE477AC7EDF2
:105CA000097AFB6A5B6B07EE103AF8EE477AC7EDAC
:105CB000087AFB6A9B6B07EE103AF8EE477AC7ED5D
:105CC000077AFB6ADB6B07EE103AF8EE477AC7ED0E
:105CD000067AFB6A1B6C07EE103AF8EE477AC7EDBE
:105CE000057A964B1B689BB2F86A19460122FCF7AD
:105CF000BBFA934B1B68F86A1946FCF7F3FAFB787A
:105D000003F00103002B23D08D4B1B68184604F0D1
:105D1000CFFA04460D46786804F0DCFA02460B46DA
:105D2000104619464FF00002864B04F051FC024623
:105D30000B462046294604F021FB02460B4610463E
:105D4000194604F02DFD0346F86A1946FCF710FECB
:105D5000FB7803F00203002B23D0794B1B68184615
:105D600004F0A6FA04460D46786804F0B3FA024639
:105D70000B46104619464FF00002724B04F028FC07
:105D800002460B462046294604F0F8FA02460B4626
:105D90001046194604F004FD0346F86A1946FCF75C
:105DA000F5FDFB7803F00403002B23D0644B1B6844
:105DB000184604F07DFA04460D46786804F08AFA25
:105DC00002460B46104619464FF000025D4B04F0A8
:105DD000FFFB02460B462046294604F0CFFA024656
:105DE0000B461046194604F0DBFC0346F86A1946D8
:105DF000FCF7DAFDFB7803F00803002B23D0504BAF
:105E00001B68184604F054FA04460D46786804F0FE
:105E100061FA02460B46104619464FF00002494B04
:105E200004F0D6FB02460B462046294604F0A6FAAB
:105E300002460B461046194604F0B2FC0346F86AC7
:105E40001946FCF7BFFDD7ED097AF5EE407AF1EE81
:105E500010FA6BD0FB7803F00103002B15D1384BFF
:105E60001B6807EE903AB8EEE77AD7ED086AD7EDEF
:105E7000097AC6EEA77A67EE277AFCEEE77A17EE84
:105E8000903AF86A1946FCF773FDFB7803F00203B9
:105E9000002B15D12A4B1B6807EE903AB8EEE77A33
:105EA000D7ED076AD7ED097AC6EEA77A67EE277AAB
:105EB000FCEEE77A17EE903AF86A1946FCF766FDB1
:105EC000FB7803F00403002B15D11D4B1B6807EE74
:105ED000903AB8EEE77AD7ED066AD7ED097AC6EEC2
:105EE000A77A67EE277AFCEEE77A17EE903AF86A1F
:105EF0001946FCF759FDFB7803F00803002B15D178
:105F00000F4B1B6807EE903AB8EEE77AD7ED056ABB
:105F1000D7ED097AC6EEA77A67EE277AFCEEE77A24
:105F200017EE903AF86A1946FCF74CFD0023184624
:105F30003037BD46B0BD00BF0000AF44F80A0020B6
:105F4000FC0A00200000594080B487B000AF03462F
:105F5000FB714FF4D8733B614823FB603A69FB68DF
:105F600092FBF3F3BB6000237B6115E010497A6973
:105F70001346DB001344DB000B441B78FA799A428A
:105F800007D17A691346DB001344DB00084A134447
:105F900007E07B6901337B617A69BB689A42E5DB84
:105FA000002318461C37BD465DF8047B704700BFD0
:105FB0006C00002080B584B000AF786039603B6829
:105FC0001B7BDBB2002B30D13B685A683B689B6877
:105FD0009A422AD03B681A683B685B6813441B7876
:105FE000FB733B685B685A1C3B685A603B685A68A5
:105FF0000F4B1340002B03DA013B63F07F030133A7
:106000001A463B685A6001233A68194651733A6848
:106010001373786840F226610122FEF747F9FB7B93
:106020009BB278681946FDF79BFF1037BD4680BDCF
:106030007F00008080B58AB000AFF8600B467A60C0
:10604000FB72FB685B687B62FB6824333B62786AA7
:1060500040F226610022FEF729F93B6A9B68013372
:10606000FB61FA693A4B1340002B03DA013B63F002
:106070007F030133FB613B6A5A68FB699A424CD14A
:106080007B68002B11D03B6A5B680133BB61BA6946
:106090002F4B1340002B03DA013B63F07F030133E6
:1060A000BB613B6ABA695A6037E03B6A1B7BDBB273
:1060B000002B06D0786A40F226610122FEF7F6F83E
:1060C00003E0786A396AFFF775FF786A40F2266163
:1060D0000022FEF7EBF83B6A5B68BB61786A40F22E
:1060E00026610122FEF7E2F8FA69BB699A420AD1F9
:1060F00000237B6102E07B6901337B617A6941F2B5
:1061000087339A42F7DDFA69BB699A42DDD0786A33
:1061100040F226610022FEF7C9F83B6A1A683B6A22
:106120009B681344FA7A1A703B6AFA699A603B6A70
:106130001B7BDBB2002B05D0786A40F2266101227E
:10614000FEF7B4F8FB7A18462837BD4680BD00BF7D
:106150007F00008080B588B000AFF860B9607A60D9
:106160003B60FB68DBB21846FFF7EEFEB861BB6927
:10617000002B02D14FF0FF332AE0BB695B687B61E3
:106180007B69002B02D16FF0010321E03B68002BFB
:106190001CDD0023FB610DE0FB697A6813441B786A
:1061A000FB74FB7CB86919460022FFF743FFFB69CB
:1061B0000133FB61FA693B689A42EDDBBB6924332A
:1061C00078691946FFF7F6FE3B6801E04FF0FF33B0
:1061D00018462037BD4680BD90B58BB000AF7860C3
:1061E0007B68002B00D1E4E07B681B6C7B627B68E2
:1061F0005B68184640F22551FEF7CCF80346002BA9
:106200006BD07B685B681846FDF7BCFE034687F8D9
:1062100023307B6A002B3FD17B683433FB61FB6901
:106220009B680133BB61BA69634B1340002B03DAEF
:10623000013B63F07F030133BB61FB695A68BB69B3
:106240009A424AD0FB691B68002B46D0FB691A684A
:10625000FB699B68134497F823201A70FB69BA699D
:106260009A607B681B6C002B37D07B681B6CDB68EB
:1062700003F00203002B30D097F8233078681946DA
:106280000122FFF7D7FE7B685A687B6824331046EB
:106290001946FFF78FFE20E07B6A03F5E0737B6110
:1062A0007B695B680133BB61BA69434B1340002BC8
:1062B00003DA013B63F07F030133BB617B691A683A
:1062C000BB699A4209D097F82330786A19460022B0
:1062D00001F018FD786800F047FC7B685B681846A1
:1062E00040F22661FEF756F80346002B61D07B682A
:1062F0005B68184640F22661FEF7A4F87B6A002B23
:1063000031D17B6824333B613B699A683B695B68A8
:106310009A420BD17B685B68184640F226610022E6
:10632000FDF7C4FF3B6900221A7342E07B685A689C
:106330003B6919683B695B685C1C386944600B44C5
:106340001B7810461946FDF70BFE3B695A681A4B3D
:106350001340002B03DA013B63F07F0301331A463D
:106360003B695A6025E07B6A03F5E473FB60FB68D8
:106370005A68FB681B689A420CD17B685B681846B8
:1063800040F226610022FDF791FF7B68002283F82E
:1063900044200EE0786A01F0D3FDB860BB68002BA2
:1063A00007DB7B685A68BB689BB210461946FDF74D
:1063B000D7FD2C37BD4690BD7F00008080B500AF73
:1063C0000120FFF7C1FD03461846FFF705FF80BD1A
:1063D00080B500AF0220FFF7B7FD03461846FFF770
:1063E000FBFE80BD80B500AF0320FFF7ADFD034687
:1063F0001846FFF7F1FE80BD80B500AF0420FFF71F
:10640000A3FD03461846FFF7E7FE80BD80B500AF49
:106410000520FFF799FD03461846FFF7DDFE80BD16
:1064200080B500AF0620FFF78FFD03461846FFF743
:10643000D3FE80BD80B58AB000AF78607B685B68B2
:106440003B623B6A002B02D16FF00103D6E0386A51
:106450000021FDF707FD7B689B69002B05D07B6859
:106460009B6918460121FBF719FB7B68DB69002B50
:1064700005D07B68DB6918460121FBF72DFB7B68A3
:106480009B68002B08D07B689A687B6893F8203063
:1064900010461946FEF7F8FD7B68DB68002B0DD02F
:1064A0007B68DB681846FEF771FD7B68DA687B68FD
:1064B00093F8203010461946FEF7E6FD07F10C036D
:1064C0001846FDF773FC7B681B6C002B02D07B68C1
:1064D0001B6C7B62786A01F06BFD0346FB607B6A94
:1064E0009B6803F4E073802B0DD0802B02D8402BE7
:1064F00006D011E0C02B09D0B3F5807F09D00BE0A6
:1065000000233B8208E000233B8205E000233B821E
:1065100002E000233B8200BF7B6A9B6803F0080314
:10652000002B03D04FF400537B8201E000237B82D9
:106530007B6A9B6803F01003002B0DD07B6A9B687D
:1065400003F02003002B03D04FF4C063BB8205E0AF
:106550004FF48063BB8201E00023BB8207F10C0390
:10656000386A1946FDF768FB4FF480400121FBF7BC
:10657000B3FA7B6893F82130DBB23B7700237B775B
:106580000023BB770123FB7707F11C031846FAF7BA
:10659000B3FA7B685B6A002B06D1802005F028F8EF
:1065A00003461A467B685A627B6800229A627B68BF
:1065B0000022DA627B68002283F830207B680022A8
:1065C00083F831207B685B6B002B06D1802005F0BF
:1065D0000FF803461A467B685A637B6800229A6369
:1065E0007B680022DA63386A40F225510122FDF708
:1065F0005DFE386A0121FDF735FC00231846283777
:10660000BD4680BD80B586B000AFF860B9607A60E5
:10661000FB68DBB21846FFF797FC78617B69002BBB
:1066200002D14FF0FF330CE07B695B683B613B6953
:10663000002B02D16FF0010303E07869FFF7FAFE47
:10664000034618461837BD4680BD00BF80B586B0EA
:1066500000AF786039607B68DBB21846FFF774FCE6
:1066600078617B69002B02D14FF0FF3329E07B6911
:106670005B683B613B69002B02D16FF0010320E0B6
:10668000386940F225510022FDF710FE386940F2CA
:1066900026610022FDF70AFE38690021FDF7E2FBC2
:1066A0007B6993F82130DBB23B7300237B730023BB
:1066B000BB730023FB7307F10C031846FAF71CFAAF
:1066C000002318461837BD4680BD00BF80B58CB08A
:1066D00000AFF860B9607A603B60FB68DBB21846D7
:1066E000FFF732FCB862BB6A002B02D14FF0FF33D8
:1066F00053E0BB6A5B687B627B6A002B02D16FF060
:1067000001034AE0BB6A34333B620023FB623FE093
:106710003B6A5B68FB61786A40F225510022FDF715
:10672000C5FD3B6A9B68BB61786A40F22551012236
:10673000FDF7BCFDBA69FB699A4201D1FB6A2CE006
:10674000FB6901337B617A69164B1340002B03DA36
:10675000013B63F07F0301337B61FB6A7A6813447A
:106760003A6A1168FA690A4412781A70786A40F233
:1067700025510022FDF79AFD3B6A7A695A60786AD2
:1067800040F225510122FDF791FDFB6A0133FB62C6
:10679000FA6A3B689A42BBDB3B6818463037BD4615
:1067A00080BD00BF7F00008080B588B000AF7860FA
:1067B00039607B68DBB21846FFF7C6FBF861FB69FE
:1067C000002B01D100232DE0FB695B68BB61BB6935
:1067D000002B01D1002325E0FB6934337B61B869CC
:1067E00040F225510022FDF761FD7B699B683B610A
:1067F0007B695B68FB60B86940F225510122FDF7B7
:1068000055FD3A69FB689A4201D100230AE03A69D2
:10681000FB689A4203DAFA683B69D31A02E03A69E4
:10682000FB68D31A18462037BD4680BD80B58AB0B4
:1068300000AF786039607B68DBB21846FFF784FBF5
:1068400078627B6A002B01D100233AE07B6A5B68A7
:106850003B623B6A002B01D1002332E07B6A243388
:10686000FB61386A40F22661FDF794FD0346BB6187
:10687000386A40F226610022FDF718FDFB699B682B
:106880007B61FB695B683B61BB69DBB2386A40F2E4
:1068900026611A46FDF70AFD7A693B699A4201D1E1
:1068A00080230EE07A693B699A4203DA3A697B6990
:1068B000D31A02E07A693B69D31AFB60FB68C3F123
:1068C000800318462837BD4680BD00BF80B58AB01A
:1068D00000AFF860B9607A603B60FB68DBB21846D5
:1068E000FFF732FBF861FB69002B02D14FF0FF3359
:1068F00082E0FB695B68BB61BB69002B01D10023AF
:106900007AE07B683E4A934273D03E4A934203D07A
:106910003D4A934212D06EE03B681A1D3A601B68F4
:106920007B61FB691B6C002B06D0FB691B6C7869D3
:1069300019465C2205F008F900235DE03B681A1D4A
:106940003A601B687B61FB691B6C002B17D0FB69ED
:106950001B6C9B683B62FB691B6C7A6912681A604E
:10696000FB691B6C7A6952685A60FB691B6C7A6917
:1069700092689A60FB691B6C7A69D268DA600023BE
:106980007B6211E0FB691B6C002B0AD0FB691B6C5E
:106990007A69796A043152F821107A6A043243F82C
:1069A00022107B6A01337B627B6A112BEADD7B69F3
:1069B0009A683B6A9A420AD1FB691B6C002B16D07D
:1069C000FB691B6C9A6D7B699B6D9A420FD0FB69CA
:1069D0001B6C002B08D0FB691B6C1A467B699B6DF6
:1069E0001046194601F018FBF869FFF723FD002354
:1069F00002E0002300E0002318462837BD4680BD92
:106A00000344088002445C8001445C4080B586B049
:106A100000AFF860B9607A60FB68DBB21846FFF738
:106A200093FA78617B69002B02D14FF0FF3316E0B7
:106A30007B691B6C002B0CD14FF4EC7004F0D8FD7B
:106A400003461A467B691A647B691B6C184600F082
:106A50001FFFF868B9687A68FFF7D4FD0346184647
:106A60001837BD4680BD00BF80B584B000AF7860E8
:106A700039607B68DBB21846FFF766FAF860FB689E
:106A8000002B01D1002305E078683968FFF7DEFDAF
:106A9000B860BB6818461037BD4680BD80B588B069
:106AA00000AFF860B9607A603B60FB68DBB2184603
:106AB000FFF74AFAF861FB69002B02D14FF0FF3370
:106AC0001DE0FB695B68BB61BB69002B02D16FF005
:106AD000010314E0B86940F225510022FDF7E6FBFE
:106AE000FB691B6C184679683A6801F085F9786192
:106AF000B86940F225510122FDF7D8FB7B691846A1
:106B00002037BD4680BD00BF80B586B000AF78603D
:106B100039607B68DBB21846FFF716FA78617B694B
:106B2000002B01D100231AE07B695B683B613B6964
:106B3000002B01D1002312E0386940F225510022D8
:106B4000FDF7B4FB7B691B6C184601F039F9F8605E
:106B5000386940F225510122FDF7A8FBFB68184671
:106B60001837BD4680BD00BF80B586B000AF7860E5
:106B70007B685B687B617B681B6C3B613B6903F5F1
:106B8000E473FB607B6893F84430DBB2002B32D1B6
:106B9000FB681A68FB685B689A422CD0FB681B682C
:106BA0003A69134493F8DC30FB72FB681B685A1C8B
:106BB000FB681A60FB681A68104B1340002B03DA5D
:106BC000013B63F07F0301331A46FB681A6001231F
:106BD0007A68194682F845107A6882F84430FB7A60
:106BE0009BB278691946FDF7BBF9786940F22661D6
:106BF0000122FDF75BFB1837BD4680BD7F0000809A
:106C000080B58AB000AFF8600B467A60FB72FB6813
:106C10005B687B62FB681B6C03F5E4733B62786A1C
:106C200040F226610022FDF741FB3B6A5B680133BD
:106C3000FB61FA693B4B1340002B03DA013B63F025
:106C40007F030133FB613B6A1A68FB699A424CD1AE
:106C50007B68002B11D03B6A1B680133BB61BA69AA
:106C6000304B1340002B03DA013B63F07F03013309
:106C7000BB613B6ABA691A6037E0FB6893F844303D
:106C8000DBB2002B06D0786A40F226610122FDF7C4
:106C90000DFB02E0F868FFF767FF786A40F22661B3
:106CA0000022FDF703FB3B6A1B68BB61786A40F278
:106CB00026610122FDF7FAFAFA69BB699A420AD104
:106CC00000237B6102E07B6901337B617A6941F2D9
:106CD00087339A42F7DDFA69BB699A42DDD0786A58
:106CE00040F226610022FDF7E1FAFB681A6C3B6A6C
:106CF0005B681344FA7A83F8DC203B6AFA695A60CD
:106D0000FB6893F84430DBB2002B05D0786A40F280
:106D100026610122FDF7CAFAFB7A18462837BD46DC
:106D200080BD00BF7F00008080B588B000AFF860F4
:106D3000B9607A603B60FB68DBB21846FFF704F984
:106D4000B861BB69002B02D14FF0FF3327E0BB696C
:106D50005B687B617B69002B02D16FF001031EE051
:106D60003B68002B19DD0023FB610DE0FB697A68AD
:106D700013441B78FB74FB7CB86919460022FFF7AB
:106D80003FFFFB690133FB61FA693B689A42EDDB27
:106D9000B869FFF7E9FE3B6801E04FF0FF331846A2
:106DA0002037BD4680BD00BF80B485B000AF78609D
:106DB0007B68002B02D14FF0FF3320E00023FB6003
:106DC00002E0FB680133FB60FB68302B05DC0F4BF6
:106DD000FA6853F82230002BF3D1FB68302B0CDC1F
:106DE0000A4BFA68796843F82210FB685A1C074B73
:106DF000002143F82210002301E06FF00103184640
:106E00001437BD465DF8047B704700BF000B0020BF
:106E100080B485B000AFF860B9607A603B60002351
:106E200018461437BD465DF8047B704780B485B0C2
:106E300000AFF860B9607A603B603B681846143771
:106E4000BD465DF8047B704780B500AF0248FFF790
:106E5000ABFF0346184680BD1420010880B500AF83
:106E60000248FFF7A1FF0023184680BD4820010813
:106E700090B59DB000AFF860B9607A60FB68002BF8
:106E800050D0FB681B78002B4CD0664B1B68002B46
:106E90000ED0654B1B685B68002B06D0624B1B68ED
:106EA0005B68184603F0CCFF02E0002007F084F88E
:106EB000F868002100F0BEF8F866FB6E002B31DDAB
:106EC000FB6E002B2ED0FB6E1A01564B1344554A15
:106ED00014460FCB84E80F00524AFB6E1B0113448B
:106EE00000221A60504B1C680020504903F0D8FF64
:106EF0000346636007F110030020194601F0FCF817
:106F0000FB6943F00203FB6107F1100318464FF4DD
:106F1000E13101F081F807F11003002000211A4649
:106F200001F0FCF8BB68002B4DD0BB681B78002B30
:106F300049D03C4B1B69002B0ED03B4B1B689B6818
:106F4000002B06D0384B1B689B68184603F078FF6F
:106F500002E0012007F030F8B868012100F06AF87B
:106F6000F866FB6E002B2EDDFB6E012B2BD0FB6E2B
:106F70001A012C4B13442B4A02F110040FCB84E866
:106F80000F00284AFB6E1B01134400221A60264B97
:106F90001C680120264903F083FF0346A36007F124
:106FA00010030120194601F0A7F807F11003184655
:106FB0004FF4E13101F030F807F110030120002116
:106FC0001A4601F0ABF87B68002B26D07B681B7853
:106FD000002B22D07868012100F02CF8F866FB6EB7
:106FE000002B1ADDFB6E022B17D0FB6E1A010D4B26
:106FF00013440C4A02F120040FCB84E80F00094A25
:10700000FB6E1B01134400221A60074B1C68022010
:10701000074903F045FF0346E36000231846743731
:10702000BD4690BDDC1000205006002070200108F5
:107030007420010880B588B000AF78603960032300
:10704000FB610AE0684AFB691B0113441B68002BC3
:1070500000D105E0FB690133FB61FB693B2BF1DDEE
:10706000FB693C2B02D14FF0FF33B8E07B68002B6B
:1070700003D07B681B78002B02D16FF00103AEE0D8
:10708000594AFB691B011344083300221A60564A0F
:10709000FB691B011344083300225A60524AFB6902
:1070A0001B0113443A685A604F4AFB691B011344A1
:1070B00001221A600023BB6155E04C4BBA6953F8BA
:1070C00022301B687868194605F02CFB02467B6865
:1070D0009A4245D1454BBA6953F822301B6818468D
:1070E00005F09EF903467A6813443B613F4BBA6949
:1070F00053F822203C49FB691B010B4408331A60FA
:107100003B691B78002B2BD0394B1A683B691B78E5
:10711000013313441B7803F00403002B20D03B6998
:107120001B78002B28D007F10803386919460A227A
:1071300005F0BCFCF860BB681B78002B08D02A4A1D
:10714000FB691B01134400221A606FF0020346E042
:10715000254AFB691B0113440833FA685A600BE0A7
:10716000BB690133BB61BB69312B05DC1F4BBA69BD
:1071700053F82230002BA0D11B4AFB691B0113449A
:1071800008331B68002B29D0174AFB691B011344E5
:1071900008331B689B68002B12D0134AFB691B0144
:1071A000134408331B689B680F49FA6912010A44AB
:1071B000083252681046F9693A689847786101E0E8
:1071C00000237B617B69002B08D0074AFB691B0108
:1071D000134400221A604FF0FF3300E0FB691846A9
:1071E0002037BD4680BD00BFDC100020000B002012
:1071F0002002002090B585B000AFF860B9607A60D9
:10720000FB68002B02DBFB683B2B02DD4FF0FF33FA
:1072100028E0164AFB681B01134408331B68002B47
:107220001ED0124AFB681B01134408331B681B69FC
:10723000002B13D00D4AFB681B01134408331B6855
:107240001C690A4AFB681B01134408335B68184633
:10725000F968BA687B68A047034603E07B6801E0F1
:107260004FF0FF3318461437BD4690BDDC100020A8
:1072700090B585B000AFF860B9607A60FB68002B0C
:1072800002DBFB683B2B02DD4FF0FF3332E01B4A91
:10729000FB681B0113441B68002B02D16FF0010334
:1072A00028E0164AFB681B01134408331B68002BB7
:1072B0001ED0124AFB681B01134408331B68DB68AD
:1072C000002B13D00D4AFB681B01134408331B68C5
:1072D000DC680A4AFB681B01134408335B681846E4
:1072E000F968BA687B68A047034603E0002301E021
:1072F0004FF0FF3318461437BD4690BDDC10002018
:1073000080B584B000AF78607B68002B02DB7B68BF
:107310003B2B02DD4FF0FF3335E01D4A7B681B013C
:1073200013441B68002B02D16FF001032BE0184AB5
:107330007B681B01134408331B68002B1CD0144AC4
:107340007B681B01134408331B689B69002B11D019
:107350000F4A7B681B01134408331B689B690C4967
:107360007A6812010A4408325268104679689847D0
:10737000F86001E00023FB60054A7B681B011344B1
:1073800000221A60FB6818461037BD4680BD00BF5A
:10739000DC10002090B585B000AFF860B9607A606D
:1073A000FB68002B02DBFB683B2B02DD4FF0FF3359
:1073B00032E01B4AFB681B0113441B68002B02D1FF
:1073C0006FF0010328E0164AFB681B0113440833E1
:1073D0001B68002B1ED0124AFB681B0113440833A4
:1073E0001B68DB69002B13D00D4AFB681B0113449B
:1073F00008331B68DC690A4AFB681B011344083325
:107400005B681846F968BA687B68A047034603E0E2
:10741000002301E04FF0FF3318461437BD4690BDFE
:10742000DC10002080B584B000AF78607B68002B52
:1074300002DB7B683B2B01DD002331E01A4A7B68CD
:107440001B0113441B68002B01D1002328E0164ABE
:107450007B681B01134408331B68002B1DD0124AA4
:107460007B681B01134408331B681B6A002B11D077
:107470000D4A7B681B01134408331B681B6A0A49C9
:107480007A6812010A4408325268104679689847AF
:10749000F86004E00023FB6001E00123FB60FB686F
:1074A00018461037BD4680BDDC10002080B584B082
:1074B00000AF78607B68002B02DB7B683B2B01DD33
:1074C000002331E01A4A7B681B0113441B68002B20
:1074D00001D1002328E0164A7B681B0113440833BE
:1074E0001B68002B1DD0124A7B681B011344083314
:1074F0001B685B6A002B11D00D4A7B681B0113448B
:1075000008331B685B6A0A497A6812010A44083228
:107510005268104679689847F86004E00123FB60E0
:1075200001E00123FB60FB6818461037BD4680BDB3
:10753000DC10002090B587B000AFF860B9607A60C9
:10754000FB68002B02DBFB683B2B01DD002337E0EF
:107550001D4AFB681B0113441B68002B01D100234B
:107560002EE0194AFB681B01134408331B68002BEB
:107570001FD0154AFB681B01134408331B685B6965
:10758000002B13D0104AFB681B01134408331B68FF
:107590005C690D4AFB681B01134408335B6818469D
:1075A000F968BA687B68A047786104E000237B61D2
:1075B00001E000237B617B69002BB8BF5B425B422B
:1075C00018461C37BD4690BDDC10002080B483B047
:1075D00000AF78607B68002B02DB7B683B2B01DD12
:1075E000002319E00F4A7B681B0113441B68002B22
:1075F00001D1002310E00B4A7B681B0113440833C0
:107600001B68002B07D0074A7B681B011344083313
:107610001B685B6800E0002318460C37BD465DF828
:10762000047B7047DC10002080B584B002AF786026
:107630007B68002B02DB7B683B2B01DD002331E004
:107640001A4A7B681B0113441B68002B01D10023DD
:1076500028E0164A7B681B01134408331B68002B83
:107660001FD0124A7B681B01134408331B685B68F8
:10767000002B01D1002315E00C4A7B681B01134449
:1076800008331B681B6809497A6812010A440832EA
:107690005268009206486321064A04F019FC044B24
:1076A00000E0002318460837BD4680BDDC100020EE
:1076B000C80B00207820010880B586B002AFF860C2
:1076C000B9607A60FB68002B02DBFB683B2B01DDB5
:1076D000012339E01E4AFB681B0113441B68002B81
:1076E00001D1022330E01A4AFB681B01134408331E
:1076F0001B68002B27D0164AFB681B011344083374
:107700001B685B68002B01D103231DE0BB68002BC5
:1077100001D1042318E07B68013B1A460C49FB6841
:107720001B010B4408331B681B680948F9680901F1
:107730000144083149680091B8681146054A04F0CF
:10774000C7FB002300E0052318461037BD4680BD67
:10775000DC1000207820010880B584B000AF78608C
:1077600039607B683B2B07DD03F024FB03460122D5
:107770001A604FF0FF333FE07B681A01204B13443F
:10778000FB60FB681B68002B07D103F013FB03466B
:1077900002221A604FF0FF332EE03B68002B07D126
:1077A00003F008FB034603221A604FF0FF3323E087
:1077B0003B684FF6FF721A803B6800225A803B6894
:1077C0004FF400525A603B6801221A813B68002244
:1077D0005A813B6800229A813B680022DA813B682B
:1077E0004FF400721A613B684FF40072DA623B6832
:1077F0004FF400721A63002318461037BD4680BD4F
:10780000DC10002080B582B000AF786039607B6802
:10781000002B03D07B681B78002B07D103F0CAFA3A
:10782000034601221A604FF0FF332DE03B68002B26
:1078300007D103F0BFFA034603221A604FF0FF336B
:1078400022E03B6800221A803B6800225A803B6895
:107850004FF400525A603B6801221A813B680022B3
:107860005A813B6800229A813B680022DA813B689A
:107870004FF400721A613B684FF40072DA623B68A1
:107880004FF400721A63002318460837BD4680BDC6
:1078900080B582B000AF78607B68002B00D139E002
:1078A000786800214FF4EC7204F0E8F97B68184620
:1078B0004FF4164100F0B0FB7B68184600F0F0FB77
:1078C0007B6804221A617B687F22DA617B6815225B
:1078D0005A627B680322DA627B681C221A637B6827
:1078E0001A225A637B681122DA637B6813221A64B6
:1078F0007B6812229A627B6817221A627B681622C2
:107900005A647B680F229A647B6800229A617B68C4
:1079100019229A630837BD4680BD00BF80B487B086
:1079200000AFF860B9607A60FB70BB685B680133D8
:107930007A6893FBF2F2796801FB02F29B1A7B6191
:10794000BB681A687B699A4202D14FF0FF3309E0A5
:10795000BB685B68FA681344FA781A70BB687A6986
:107960005A60002318461C37BD465DF8047B7047FB
:1079700080B582B000AF78600B46FB707B6803F186
:107980005C017B6803F5E072FB78084611468022B3
:10799000FFF7C4FF034618460837BD4680BD00BF49
:1079A00080B582B000AF78600B46FB707B6803F156
:1079B000DC017B6803F5E472FB78084611468022FF
:1079C000FFF7ACFF034618460837BD4680BD00BF31
:1079D00080B584B000AF786039600023FB6009E0B7
:1079E0003B681B7878681946FFF7DAFFF8603B6858
:1079F00001333B60FB68002B03D13B681B78002BF5
:107A0000EED1FB6818461037BD4680BD80B582B008
:107A100000AF78600B46FB70FB781F2B06D9FB7814
:107A200078681946FFF7BCFF03460BE078685E21D3
:107A3000FFF7B6FFFB784033DBB278681946FFF7F3
:107A4000AFFF034618460837BD4680BD80B588B0F5
:107A500000AF78600B46FB707B68DB68BB617B68BE
:107A600003F5AE737B617B6810333B617B6803F584
:107A7000E873FB60FB681B68622B02DD4FF0FF338D
:107A80002DE1FA783B6904331B689A4204D13B69C3
:107A900004331B68002B0DD1FA783B6908331B684F
:107AA0009A4204D13B6908331B68002B02D1FB7852
:107AB0000A2B2DD10023FB610AE0FB697A6913448C
:107AC0001B7878681946FFF753FFFB690133FB61A8
:107AD000FB681A68FB699A42EFDCFB787868194604
:107AE000FFF746FF7B6900221A70FB6800225A608C
:107AF000FB685A68FB681A60BB6903F00203002B3D
:107B000004D0FB7878681946FFF74AFF0023E6E0C7
:107B1000FA783B690C331B689A427DD13B690C3380
:107B20001B68002B78D0FB685B68002B01D1002319
:107B3000D5E0FB685B68013B7A6913441B78FB72F4
:107B4000FB685B68FB610BE0FB69013B7A691344EE
:107B5000FA6979690A4412781A70FB690133FB618A
:107B6000FB681A68FB699A42EEDAFB685B685A1E8A
:107B7000FB685A60FB681B685A1EFB681A60BB6989
:107B800003F00203002B45D0FB685A68FB681B68B2
:107B90009A420BD178685449FFF71AFFFB7A1F2BE2
:107BA00038D878685049FFF713FF33E0FB7A1F2B72
:107BB00004D878684D49FFF70BFF03E078684C491B
:107BC000FFF706FF78684B49FFF702FFFB685B6829
:107BD000FB610AE0FB697A6913441B7878681946EF
:107BE000FFF714FFFB690133FB61FB681A68FB694F
:107BF0009A42EFDCFB7A1F2B04D878683E49FFF7E6
:107C0000E7FE03E078682021FFF7CAFE78683B4969
:107C1000FFF7DEFE002362E0FA783B6914331B684D
:107C20009A4219D13B6914331B68002B14D07B692D
:107C300000221A70FB6800225A60FB685A68FB68D1
:107C40001A60BB6903F00203002B03D078682C494B
:107C5000FFF7BEFE002342E0FB681A68FB685B6822
:107C60009A420ED1FB685B68591CFA6851607A69C8
:107C70001344FA781A70FB681B685A1CFB681A6078
:107C800022E0FB681B68FB610BE0FB6901337A694A
:107C90001344FA6979690A4412781A70FB6901334E
:107CA000FB61FB685A68FB699A42EEDDFB685B6822
:107CB000591CFA6851607A691344FA781A70FB68A3
:107CC0001B685A1CFB681A60BB6903F00203002B97
:107CD00004D0FB7878681946FFF798FE0023184611
:107CE0002037BD4680BD00BF8020010884200108E8
:107CF0008C20010894200108982001089C2001088C
:107D0000A020010880B588B000AFF8600B467A600B
:107D1000FB72FB68002B02D14FF0FF334CE0FB6895
:107D2000FB61FB691B68BB61FB69DB687B617B698D
:107D300003F002033B61FB7A0A2B02D00D2B09D022
:107D400018E0BB6903F48073002B02D00D23FB7293
:107D500010E00FE0BB6903F04003002B01D00023CB
:107D60002AE0BB6903F08003002B02D00A23FB72D8
:107D7000FFE700BFBB6903F00803002B03D0FB7AC9
:107D800003F07F03FB727B6903F00103002B05D036
:107D9000FB7AF8681946FFF759FE0CE0FB7AF868A1
:107DA0001946FFF7E5FD3B69002B04D0FB7AF86824
:107DB0001946FFF72BFE002318462037BD4680BD2D
:107DC00080B483B000AF78607B68002B02D14FF0A5
:107DD000FF330AE07B68D3F8C4217B68D3F8C03155
:107DE0009A420CBF00230123DBB218460C37BD4674
:107DF0005DF8047B704700BF80B586B000AFF860C7
:107E0000B9607A60FB68002B02D14FF0FF333FE08E
:107E1000F868FFF7D5FF78617B69002B02DA6FF015
:107E2000010335E07B69002B01D1002330E0FB68C2
:107E300003F5E0733B6100237B611EE07B69BA6858
:107E400013443A691268F9680A4492F85C201A707F
:107E50007B6901337B613B691B685A1C3B691A6073
:107E60003B691A680C4B1340002B03DA013B63F0AB
:107E70007F0301331A463B691A603B695A683B69C4
:107E80001B689A4203D07A697B689A42D6DB7B6989
:107E900018461837BD4680BD7F00008080B586B08B
:107EA00000AFF860B9607A6000233B61FB68002B8B
:107EB00002D14FF0FF3316E000237B610BE07B69BA
:107EC000BA6813441B78F8681946FFF769FD3861F2
:107ED0007B6901337B617A697B689A4202DA3B698C
:107EE000002BECD07B6918461837BD4680BD00BF1B
:107EF00080B485B000AF78607B68002B01D100238F
:107F000015E07B68D3F8CC315A1C0C4B1340002B86
:107F100003DA013B63F07F030133FB607B68D3F836
:107F2000C821FB689A420CBF00230123DBB218462C
:107F30001437BD465DF8047B704700BF7F000080AA
:107F400080B487B000AF78607B68002B02D14FF01F
:107F5000FF3324E07B6803F5E4737B617B695A6837
:107F60007B691B689A4202D16FF0010317E07B68BE
:107F7000D3F8C8315A1C0D4B1340002B03DA013BD8
:107F800063F07F0301333B617B691B687A681344AC
:107F900093F8DC30FB607B693A691A60FB6818462D
:107FA0001C37BD465DF8047B704700BF7F00008032
:107FB00080B483B000AF78607B689B6D18460C3747
:107FC000BD465DF8047B704780B483B000AF786035
:107FD0007B689B6D18460C37BD465DF8047B704787
:107FE00080B582B000AF786039607868396800F099
:107FF00013F8034618460837BD4680BD80B582B0E9
:1080000000AF786039607868396800F005F8034699
:1080100018460837BD4680BD80B485B000AF786093
:1080200039607B689B6843F400727B689A607B6868
:108030009B6823F4F8327B689A607B683A689A659B
:108040000023FB601CE0154AFB68DB0013445B68FF
:108050001A463B689A4210D17B689B6823F40072F1
:108060007B689A607B689A680C4BF96853F83130EA
:108070001A437B689A6000230AE0FB680133FB60C7
:10808000064AFB68DB0013445B68002BDBDA002345
:1080900018461437BD465DF8047B7047AC200108D4
:1080A00080B483B000AF78607B681B6823F4BF6343
:1080B00023F004037A6813607B685B6823F0010295
:1080C0007B685A607B68DB6823F4507323F00303FA
:1080D0007A68D3607B689B6823F4E8727B689A6057
:1080E0007B689B6843F480727B689A600C37BD465E
:1080F0005DF8047B704700BF80B582B000AF786048
:108100003960786804493A68F8F726FA0023184677
:108110000837BD4680BD00BF02445C8080B584B096
:1081200000AFF860B9607A60F86804497A68F8F7D7
:1081300013FA002318461037BD4680BD01445C4049
:1081400080B483B000AF78603960002318460C37E4
:10815000BD465DF8047B704780B483B000AF7860A3
:10816000002318460C37BD465DF8047B704700BFFE
:1081700080B483B000AF78603960002318460C37B4
:10818000BD465DF8047B704780B483B000AF786073
:108190003960002318460C37BD465DF8047B7047F4
:1081A00080B483B000AF7860034B18460C37BD46EF
:1081B0005DF8047B704700BFAC21010880B485B036
:1081C00000AFF860B9607A60BB68064A118892789F
:1081D00019809A70012318461437BD465DF8047B58
:1081E000704700BFAC21010880B58AB000AF78604D
:1081F0003960924BFB613B6800221A703B684FF478
:1082000096425A603B6800225A703B6808229A6086
:108210003B680122DA603B6800229A7001233B62CE
:10822000786803F0F1FE0346BB61B869F96904F0B0
:1082300079FB7862F5E0786A0021002204F036FCD0
:1082400078617B6A1B783B617D4B1A683B6901331F
:1082500013441B7803F00303022B02D13B69203B3C
:1082600000E03B69FB733B6A013B042B00F2D480C6
:1082700001A252F823F000BF8D820008EF820008AF
:10828000CD830008DB830008E98300087B69632B4A
:1082900025DCFB7B323B062B28D801A252F823F0C9
:1082A000BD820008ED820008CD820008C58200086A
:1082B000ED820008ED820008D58200083B680022AC
:1082C0001A700BE03B6801221A7007E03B6802223B
:1082D0001A7003E03B6803221A7000BF06E03B6897
:1082E0007A695A603B6A01333B6295E094E0FB7B1C
:1082F000303B232B66D801A252F823F0BD8300083F
:10830000B5830008C5830008C5830008C58300083D
:10831000C5830008C5830008C5830008C58300081D
:10832000C5830008C5830008C5830008C58300080D
:10833000C5830008C5830008C5830008C5830008FD
:10834000C5830008C5830008C5830008C5830008ED
:108350009D830008C5830008C5830008C583000805
:10836000C5830008C5830008C5830008C5830008CD
:10837000AD8300088D83000895830008C58300083D
:10838000C5830008C5830008A58300083B68002258
:108390005A7017E03B6801225A7013E03B680222D2
:1083A0005A700FE03B6803225A700BE03B680422CE
:1083B0005A7007E03B6805225A7003E03B680622CA
:1083C0005A7000BF3B6A01333B6225E03B687A6923
:1083D0009A603B6A01333B621EE03B687A69DA606F
:1083E0003B6A01333B6217E0FB7B4E2B04D0532BDF
:1083F00006D0482B08D00BE03B6800229A7007E0BB
:108400003B6801229A7003E03B6802229A7000BF29
:108410003B6A01333B6200BF0020F96904F082FA35
:1084200078627B6A002B7FF406AFB86903F0E8F846
:10843000002318462837BD4680BD00BFB021010883
:108440002002002080B59AB000AF786039607A6869
:1084500007F10C0310461946FFF74EFE0346002BAA
:1084600002D04FF0FF3314E007F10C0318463968CF
:1084700000F014F87A6807F10C03104600211A4640
:10848000FFF74CFE0346002B02D06FF0010300E023
:10849000002318466837BD4680BD00BF80B582B056
:1084A00000AF786039603B6878681946FFF7B4FD23
:1084B0000837BD4680BD00BF80B59AB000AF786078
:1084C0007A6807F10C0310461946FFF715FE0346BC
:1084D000002B02D04FF0FF3305E007F10C031846E4
:1084E000FFF766FD034618466837BD4680BD00BFEE
:1084F00080B59AB000AF786039607A6807F10C03F4
:1085000010461946FFF7F8FD0346002B02D04FF046
:10851000FF3314E007F10C031846396800F014F833
:108520007A6807F10C03104600211A46FFF7F6FDA2
:108530000346002B02D06FF0010300E00023184631
:108540006837BD4680BD00BF80B483B000AF78609F
:1085500039607B68002B00D129E07B689B6823F49D
:10856000E0727B689A603B68052B06D17B689B684C
:1085700043F040027B689A6019E03B68062B06D105
:108580007B689B6843F080027B689A600FE03B68E1
:10859000072B06D17B689B6843F0C0027B689A601A
:1085A00005E07B689B6843F480727B689A600C37B7
:1085B000BD465DF8047B704780B59AB000AF786027
:1085C0007A6807F1080310461946FFF795FD034640
:1085D000002B02D04FF0FF331AE03B6903F4E07345
:1085E0007B667B6EB3F5807F01D1082310E07B6E44
:1085F000C02B01D107230BE07B6E802B01D106231A
:1086000006E07B6E402B01D1052301E06FF0620391
:1086100018466837BD4680BD80B59AB000AF786017
:1086200039607A6807F10C0310461946FFF764FDBC
:108630000346002B02D04FF0FF3314E007F10C0388
:108640001846396800F014F87A6807F10C031046F0
:1086500000211A46FFF762FD0346002B02D06FF09F
:10866000010300E0002318466837BD4680BD00BF07
:1086700080B483B000AF786039607B68002B00D194
:108680000FE03B68022B06D17B689B6843F0080231
:108690007B689A6005E07B689B6823F008027B6832
:1086A0009A600C37BD465DF8047B704780B59AB080
:1086B00000AF78607A6807F1080310461946FFF7A3
:1086C0001BFD0346002B02D14FF0FF330AE03B694C
:1086D00003F00803002B02D002237B6601E0012394
:1086E0007B667B6E18466837BD4680BD80B59AB004
:1086F00000AF786039607A6807F10C0310461946BC
:10870000FFF7FAFC0346002B02D04FF0FF3316E0D0
:108710003B68DBB207F10C021046194600F014F872
:108720007A6807F10C03104600211A46FFF7F6FCA1
:108730000346002B02D06FF0010300E0002318462F
:108740006837BD4680BD00BF80B483B000AF78609D
:108750000B46FB707B68002B00D132E07B689B6886
:1087600023F0804323F030037A689360FB78012B79
:1087700006D17B689B6843F030027B689A6020E0FA
:10878000FB78022B06D17B689B6843F010027B6864
:108790009A6016E0FB78032B08D17B689B6843F056
:1087A000804343F010037A6893600AE0FB78042B5F
:1087B00007D17B689B6843F0804343F030037A68BD
:1087C00093600C37BD465DF8047B704780B59AB066
:1087D00000AF78607A6807F1080310461946FFF782
:1087E0008BFC0346002B02D04FF0FF3320E03B69A7
:1087F00003F01003002B18D03B6903F08043002BDB
:1088000009D03B6903F02003002B01D0042300E0D2
:1088100003237B660BE03B6903F02003002B01D0B0
:10882000012300E002237B6601E000237B667B6E70
:1088300018466837BD4680BD80B59AB000AF7860F5
:1088400039607A6807F10C0310461946FFF754FCAB
:108850000346002B02D04FF0FF3316E03B68DBB23B
:1088600007F10C021046194600F014F87A6807F177
:108870000C03104600211A46FFF750FC0346002B5C
:1088800002D04FF0FF3300E0002318466837BD46A2
:1088900080BD00BF80B483B000AF78600B46FB7032
:1088A0007B68002B00D134E0FB78002B0CD17B6877
:1088B0009B6823F400127B689A607B681B6823F432
:1088C00060627B681A6024E0FB78022B0CD17B6825
:1088D0001B6823F460627B681A607B689B6843F4C2
:1088E00000127B689A6014E0FB78012B11D17B6841
:1088F0009B6823F400127B689A607B681B6843F4D2
:1089000060627B681A607B681122DA637B681322DD
:108910001A640C37BD465DF8047B704780B59AB089
:1089200000AF78607A6807F10C0310461946FFF72C
:10893000E3FB0346002B02D04FF0FF330EE07B69D0
:1089400003F40013002B01D0022307E0FB6803F4BB
:10895000C063002B01D0012300E0002318466837D4
:10896000BD4680BD80B584B000AF786039603B689B
:10897000002B02D10023FB600EE03B68012B02D1EB
:108980000123FB6008E03B68022B02D10223FB605D
:1089900002E06FF062030BE07B681846F968FFF7AE
:1089A000E7FB0346002B02D06FF0010300E0002339
:1089B00018461037BD4680BD80B582B000AF7860E4
:1089C0007B68184604214FF4804205F0FDFA083711
:1089D000BD4680BD80B582B000AF78607B68184628
:1089E00005F0EAFA002318460837BD4680BD00BFEF
:1089F00080B5AAB000AF78607B68013B07F16402E4
:108A000010461D491A4603F097FA07F16403184609
:108A100048F2020105F0E0FAC7F8A400D7F8A43044
:108A2000002B01DC002322E0D7F8A4000221FFF78D
:108A30009FFB07F10803D7F8A4001946FFF75CFB7A
:108A400000237B610023FB600023BB604DF2051314
:108A50003B610023FB650023BB6507F10803D7F8E2
:108A6000A40000211A46FFF759FBD7F8A430184696
:108A7000A837BD4680BD00BFB821010880B586B0CB
:108A800000AF7860396007F1080338681946FFF7CE
:108A9000ABFBFB6878681946FFF700FD7B7A7868C6
:108AA0001946FFF751FE3B6978681946FFF74CFD00
:108AB0007B6978681946FFF7DBFDBB7A7868194651
:108AC000FFF7E8FE1837BD4680BD00BF80B59AB0FD
:108AD00000AF7860396007F10C0378681946FFF73A
:108AE0000BFB07F10C0318463968FFF7C7FF07F1C6
:108AF0000C03786800211A46FFF710FB034618465E
:108B00006837BD4680BD00BF90B59DB000AFF8602E
:108B1000B9607A60F86848F2020105F05DFAF8661B
:108B2000FB6E002B08DC424B1B68DB681846414992
:108B3000FA6802F0C3FB76E0F86E0221FFF718FB3B
:108B40000346002B0FDA3A4B1B68DC6802F032F95F
:108B500003461B68184603F059FC03462046364975
:108B60001A4602F0ABFB07F11003F86E1946FFF747
:108B7000C3FA0346002B0FDA2D4B1B68DC6802F0AA
:108B800019F903461B68184603F040FC03462046CB
:108B90002A491A4602F092FB0023FB6100237B6105
:108BA00000233B614DF20513BB617B687B660023AC
:108BB0003B66BB685B6807F1100210461946FFF779
:108BC0006DFCBB685B7807F1100210461946FFF791
:108BD000BBFDBB689B6807F1100210461946FFF702
:108BE000B3FCBB68DB6807F1100210461946FFF7BB
:108BF0003FFDBB689B7807F1100210461946FFF74E
:108C000049FE07F11003F86E00211A46FFF786FAB5
:108C10000346002B07DA064B1B68DB680848012176
:108C2000092202F0D5FCFB6E18467437BD4690BD94
:108C300050060020C4210108D0210108E0210108CC
:108C4000F021010880B586B000AF7860396007F187
:108C5000080338681946FFF7C7FA07F10803786870
:108C600019460022FFF750FF034618461837BD4645
:108C700080BD00BF90B59DB000AFF860B9607A606C
:108C8000F86848F2020105F0A7F9F866FB6E002BC0
:108C900008DC454B1B68DB6818464449FA6802F05B
:108CA0000DFB7BE0F86E0221FFF762FA0346002B12
:108CB0000FDA3D4B1B68DC6802F07CF803461B684A
:108CC000184603F0A3FB0346204639491A4602F032
:108CD000F5FA07F11003F86E1946FFF70DFA03468F
:108CE000002B0FDA304B1B68DC6802F063F8034698
:108CF0001B68184603F08AFB034620462D491A4696
:108D000002F0DCFA7B68002B01D0032300E0012392
:108D1000FB6100237B6140233B614DF20513BB6186
:108D200000237B6600233B66BB685B6807F110028B
:108D300010461946FFF7B2FBBB685B7807F11002DB
:108D400010461946FFF700FDBB689B6807F110024B
:108D500010461946FFF7F8FBBB68DB6807F1100205
:108D600010461946FFF784FCBB689B7807F1100298
:108D700010461946FFF78EFD07F11003F86E00212B
:108D80001A46FFF7CBF90346002B07DA064B1B68A0
:108D9000DB6809480121092202F01AFCFB6E184623
:108DA0007437BD4690BD00BF50060020C4210108A5
:108DB000D0210108E0210108F021010880B586B02A
:108DC00000AF7860396007F1080338681946FFF78B
:108DD0000BFA07F10803786819460022FFF74AFFEB
:108DE000034618461837BD4680BD00BF80B59AB00F
:108DF00000AF7860396007F10C0378681946FFF717
:108E00007BF93B68002B04D0BB6943F00203BB61D4
:108E100003E0BB6923F00203BB6107F10C03786830
:108E200000211A46FFF77AF96837BD4680BD00BFBA
:108E300080B584B000AF78607A6807F10C03104603
:108E400007491A46F7F788FB0346002B02D04FF07C
:108E5000FF3300E0FB6818461037BD4680BD00BFF9
:108E60000344048080B584B000AF78607A6807F16D
:108E70000C03104607491A46F7F76EFB0346002B12
:108E800002D04FF0FF3300E0FB6818461037BD46B4
:108E900080BD00BF0444048080B59AB000AF786004
:108EA00039607A6807F1080310461946FFF724F97C
:108EB0000346002B02D04FF0FF331DE03B68104A01
:108EC00082FB03125211DB17D31A7B667B6E012BD8
:108ED000B8BF0123FB650023BB657A6807F108036F
:108EE000104600211A46FFF719F90346002B02D05D
:108EF0004FF0FF3300E0002318466837BD4680BDC1
:108F00001F85EB5180B59AB000AF786013460A46D2
:108F1000FA70BB707A6807F10C0310461946FFF728
:108F2000EBF80346002B02D04FF0FF3312E0FB7842
:108F3000BB64BB78FB647A6807F10C031046002120
:108F40001A46FFF7EBF80346002B02D04FF0FF3331
:108F500000E0002318466837BD4680BD80B483B06A
:108F600000AF78603960002318460C37BD465DF8C5
:108F7000047B704780B582B000AF78607B6818468C
:108F800044F205410022F7F7E7FA0346002B02D02E
:108F90004FF0FF3300E0002318460837BD4680BD80
:108FA00080B582B000AF78607B68184644F2064115
:108FB0000022F7F7D1FA0346002B02D04FF0FF331F
:108FC00000E0002318460837BD4680BD80B584B058
:108FD00000AF786039603B6800221A607A6807F158
:108FE0000C0310461D491A46F7F7B6FA0346002B44
:108FF00002D04FF0FF332CE0FB6803F00103002B9D
:1090000005D03B681B6843F080023B681A60FB6830
:1090100003F00203002B05D03B681B6843F04002BD
:109020003B681A60FB6803F00403002B05D03B6823
:109030001B6843F020023B681A60FB6803F00803DA
:10904000002B05D03B681B6843F010023B681A6098
:10905000002318461037BD4680BD00BF074404807A
:1090600080B485B000AF7860104B1B680133104AA4
:1090700082FB03129111DA178A1AC82101FB02F24E
:109080009B1AFB600B4B1B68FA689A4200D108E000
:10909000064B1A68084B796843F82210034BFA68AC
:1090A0001A601437BD465DF8047B7047500F0020EE
:1090B0001F85EB51540F0020300C002080B483B08A
:1090C00000AF124B1A68124B53F822307B60114BE1
:1090D0001A680E4B1B689A4201D100230FE00B4B1C
:1090E0001B685A1C0C4B83FB02139911D317CB1A24
:1090F000C82101FB03F3D31A044A13607B681846A6
:109100000C37BD465DF8047B704700BF540F00204C
:10911000300C0020500F00201F85EB5180B588B027
:1091200000AF0346FB71B54B1B781B2B40F0EB8166
:10913000B24803F075F90346BB61B04ABB691344FA
:10914000FA791A70BB690133BB61AC4ABB6913443D
:1091500000221A70BB69022B40F30981A74B9B7850
:109160004D2B40F00481BB69062B40F00081A34BDE
:10917000DB78203B512B00F2DB8001A252F823F078
:10918000C9920008D1920008D992000831930008D2
:10919000319300083193000831930008319300089F
:1091A000F992000801930008099300083193000820
:1091B000319300083193000831930008319300087F
:1091C000E1920008E9920008F1920008319300084A
:1091D000319300083193000831930008319300085F
:1091E000319300083193000831930008319300084F
:1091F000319300083193000831930008319300083F
:10920000319300083193000831930008319300082E
:10921000319300083193000831930008319300081E
:10922000319300083193000831930008319300080E
:1092300031930008319300083193000831930008FE
:1092400031930008319300083193000831930008EE
:1092500031930008319300083193000831930008DE
:1092600031930008319300083193000831930008CE
:1092700031930008319300083193000831930008BE
:1092800011930008199300083193000831930008E6
:10929000319300083193000831930008319300089E
:1092A000319300083193000831930008319300088E
:1092B000319300083193000831930008319300087E
:1092C00021930008299300086FF03103FB612FE020
:1092D0006FF03203FB612BE06FF03303FB6127E09B
:1092E0006FF03403FB6123E06FF03503FB611FE097
:1092F0006FF03603FB611BE06FF03703FB6117E093
:109300006FF03803FB6113E06FF03903FB610FE08E
:109310006FF03A03FB610BE06FF03B03FB6107E08A
:109320006FF03C03FB6103E06FF03D03FB6100BFA6
:10933000FB6923F07F4323F0FF03FB612F4B1B7975
:10934000203BDBB27B612D4B5B79203BDBB23B6189
:109350007B691B04FA691343FB613B691B02FA69D1
:109360001343FB61254B00221A70FB69D7E0234BA6
:109370005B785B2B04D0214B00221A70FB79CEE086
:109380001F4B1A68FB79013313441B7803F0030366
:10939000002B37D0194B00221A70FB79413B072B69
:1093A00000F2BC8001A252F823F000BFCD93000868
:1093B000D3930008D9930008DF930008F1930008C5
:1093C000EB9300081D950008E59300084FF0FF336C
:1093D000A5E06FF00103A2E06FF003039FE06FF0E0
:1093E00002039CE06FF0040399E06FF0050396E040
:1093F000024B00221A70002391E000BF580F00209A
:1094000020020020FB797E2B7BD1474B00221A7073
:1094100046480021002203F049FBF860FB68013B4D
:10942000172B69D801A252F823F000BF8D940008D1
:1094300093940008999400089F940008A59400084C
:10944000AB940008F9940008F9940008F994000816
:10945000F9940008B1940008B7940008BD9400087E
:10946000C3940008C9940008F9940008CF94000838
:10947000D5940008DB940008E1940008E794000804
:10948000F9940008ED940008F39400086FF00403C9
:1094900045E06FF0150342E06FF008033FE06FF026
:1094A00005033CE06FF0060339E06FF0070336E098
:1094B0006FF0090333E06FF00A0330E06FF00B0345
:1094C0002DE06FF00C032AE06FF00D0327E06FF042
:1094D0000E0324E06FF00F0321E06FF010031EE095
:1094E0006FF011031BE06FF0120318E06FF013032D
:1094F00015E06FF0140312E00B4B00221A700023EA
:109500000DE000230BE0FB791B2B07D1064B1B2240
:109510001A70054B00225A70002300E0FB791846B0
:109520002037BD4680BD00BF580F00205A0F0020D5
:1095300080B586B000AF0346FB71994B1B68002BCA
:1095400015D0984B1B68002B0CD0FB791846FFF701
:10955000E5FDB860BB68002B03D0B868FFF780FD5D
:10956000B8E1B7E1FB791846FFF77AFDB2E18E4822
:1095700002F056FF03463B61FB791846FFF7CEFD2C
:10958000B860BB68002B03D0884B1B68002B00D051
:10959000A0E1BB6813F1030F0DD1854B1B68002BB5
:1095A00040F39881824B1B685A1E814B1A60012040
:1095B00000F082FA8EE1BB6813F1040F0FD17C4BEF
:1095C0001B68794AD35C002B00F08481784B1B68C0
:1095D0005A1C774B1A60012000F084FA7AE1BB68CC
:1095E00013F1050F02D0BB68012B0DD1704B1B6826
:1095F000002B08DD6E4B1B68184600F05DFA6C4BC3
:1096000000221A6066E165E1BB6813F1060F02D023
:10961000BB68052B11D1664B1B68634AD35C002BDA
:109620000AD0634B1B683A69D31A184600F05AFAFD
:109630005F4B3A691A604DE14CE1BB68032B02D0E5
:10964000BB68042B03D1594B01221A6042E1BB686D
:109650000A2B02D0BB680D2B14D1544B01221A6087
:1096600000237B6109E0504A7B6913441B7818464C
:10967000FFF7F6FC7B6901337B617A693B699A42AB
:10968000F1DB27E1BB68082B48D1494B1B68002B55
:1096900040F32081464B1B687B610AE07B69013BFC
:1096A00041497A690A4411783F4AD1547B690133B0
:1096B0007B613D4A7B6913441B78002BEED13B69EB
:1096C000013B3B61384A3B69134400221A70384B16
:1096D0001B685A1E364B1A60012000F0EDF900F0AD
:1096E000CBF9334B1B68304AD35C002B0ED0304B88
:1096F0001A682D4B13442F48194602F00DFB2E4BD0
:109700001B689B68184601F093FC04E001202B497C
:10971000012204F081FC00F0BFF9DBE0BB687F2B85
:1097200003D0BB6813F1090F53D1214B1B681E4AAC
:10973000D35C002B4CD01E4B1B6801337B610AE0CD
:109740007B69013B18497A690A441178164AD15459
:109750007B6901337B61144A7B6913441B78002BBE
:10976000EED13B69013B3B610F4A3B691344002248
:109770001A7000F081F90E4B1B680B4AD35C002B6A
:109780001ED00B4B1A68084B13440A48194602F0C6
:10979000C3FA094B1B689B68184601F049FC14E0AA
:1097A0001C0200202C0C0020BC0F00208810002080
:1097B00084100020FC21010850060020002201082E
:1097C00001204649012204F027FC00F065F981E000
:1097D00080E0BB680B2B20D1414B1B68002B04DDC4
:1097E0003F4B1B68184600F067F900F045F904E0AC
:1097F00001203A49012204F00FFC3B695A1E3A61EC
:10980000002BF5D100F048F9354B00221A60344B9B
:109810001B68344A0021D1545CE0BB68002B59DB43
:10982000314B1A68BB68013313441B7803F097036C
:10983000002B4FD03B69C72B4CDC294B1B68294AB6
:10984000D35C002B14D1264B1B68591C244A116091
:10985000BA68D1B2234AD154214B1B68214A002156
:10986000D154FB1D01201946012204F0D5FB31E043
:109870003B69FB600AE0FB6801331A49FA680A4455
:109880001178184AD154FB68013BFB60144B1B68EC
:10989000FA689A42EFDA124B1B68591C104A1160A1
:1098A000BA68D1B20F4AD15400F0E6F80C4B1B68ED
:1098B0005A1E0C4B1A440A4B1B683969CB1A0233E7
:1098C000012011461A4604F0A7FB00F0E5F801203C
:1098D00000F008F91837BD4680BD00BF002201081E
:1098E00084100020BC0F00202002002080B582B030
:1098F00000AF14E01A4B1B685B68184601F0AAFB26
:109900000246FB1C10461946012204F079FB7860E0
:109910007B68002B03DBFB781846FFF709FE104B32
:109920001B685B68184601F095FB03461846FDF777
:1099300079FD0346002BDDD10A4B1B68002B09D0B3
:10994000094B1A68094B1B689A420CBF002301237C
:10995000DBB201E0064B1B6818460837BD4680BDE8
:10996000500600201C020020540F0020500F002041
:109970008810002080B500AFFFF7B8FF054B1B68CB
:10998000002B01D1002302E0FFF798FB03461846A5
:1099900080BD00BF1C02002080B584B000AF78609D
:1099A00039600023BB60FFF7A1FF7B68002B01D16A
:1099B000002333E0FFF782FBF8607B6800221A7017
:1099C00013E0FB68002B0DDDBB687A681344FA686E
:1099D000D2B21A70BB680133BB60BB687A681344AB
:1099E00000221A70FFF76AFBF860FB68002B04D0B6
:1099F0003B685A1EBB689A42E3DCBB68002B03DC61
:109A0000084B1B68002B01D0012300E00023FB6002
:109A1000FB68002B01D000F007F8FB6818461037F0
:109A2000BD4680BD8810002080B400AF084B0022E6
:109A30001A60084B00221A60064B1B68064A002178
:109A4000D154064B00221A60BD465DF8047B704776
:109A50001C02002084100020BC0F00208810002071
:109A600080B400AF034B01221A60BD465DF8047B51
:109A7000704700BF1C02002080B500AF044802F010
:109A80004BF9044B1B689B68184601F0D1FA80BD66
:109A9000042201085006002080B500AF044802F0FF
:109AA0003BF9044B1B689B68184601F0C1FA80BD66
:109AB000082201085006002080B582B000AF78600F
:109AC0000648796802F028F9054B1B689B68184620
:109AD00001F0AEFA0837BD4680BD00BF0C22010878
:109AE0005006002080B582B000AF786006487968E3
:109AF00002F012F9054B1B689B68184601F098FAB2
:109B00000837BD4680BD00BF142201085006002062
:109B100080B582B000AF78600648796802F0FCF842
:109B2000054B1B689B68184601F082FA0837BD4652
:109B300080BD00BF1C2201085006002080B582B005
:109B400000AF78600648796802F0E6F8054B1B68BC
:109B50009B68184601F06CFA0837BD4680BD00BF0F
:109B6000242201085006002080B582B000AF786042
:109B70003960074839687A6802F0CEF8054B1B68EF
:109B80009B68184601F054FA0837BD4680BD00BFF7
:109B90002C2201085006002080B500AF044802F0D6
:109BA000BBF8044B1B689B68184601F041FA80BD66
:109BB000382201085006002080B500AFFFF75CFF97
:109BC000202002F0BDF8FFF767FF80BD80B582B0AE
:109BD00000AF786039607B68002B09DB0F4B7A6837
:109BE0001A600E4B1B6828330D48194602F094F892
:109BF0003B68002B09DB0B4B3A681A60094B1B686A
:109C00001E330748194602F087F8074B1B689B680C
:109C1000184601F00DFA0837BD4680BD8C100020B3
:109C200040220108901000205006002080B500AFAF
:109C3000044802F071F8044B1B689B68184601F059
:109C4000F7F980BD482201085006002080B500AF1A
:109C5000044802F061F8044B1B689B68184601F049
:109C6000E7F980BD502201085006002080B500AF02
:109C7000064802F051F8064802F04EF8054B1B6802
:109C80009B68184601F0D4F980BD00BF5822010836
:109C9000602201085006002080B500AF064802F09F
:109CA0003BF8064802F038F8054B1B689B681846DD
:109CB00001F0BEF980BD00BF6822010870220108D2
:109CC0005006002080B400AF094B1B69DB4303F44E
:109CD0007042084B1A60084B074A128A92B222F06F
:109CE000010292B21A82BD465DF8047B704700BF44
:109CF00000080240941000200048014080B582B066
:109D000000AF7860FDF7AAF8FDF79EF878687968EB
:109D10007A68FDF7ADF800202349FEF7D7FE012051
:109D20002149FEF7D3FE00200021FFF75FF8012054
:109D30000021FFF75BF81D4B1B689B68184600214C
:109D40000222002302F044F81948FBF749F91948A8
:109D5000FBF746F91848FBF743F91848FBF740F9B9
:109D60004FF4807000F044F84FF4007000F040F8B9
:109D70004FF4806000F03CF84FF4006000F038F8D9
:109D80000F48FBF703F90F48FBF700F90E48FBF704
:109D9000FDF80E48FBF7FAF80B2032211A22FBF7E8
:109DA000BDFD0837BD4680BD782201085006002061
:109DB000882201088C2201089022010898220108BB
:109DC000A0220108A8220108B0220108B822010837
:109DD00080B483B000AF0346FB80044BFA881A833B
:109DE0000C37BD465DF8047B704700BF0008024099
:109DF00080B483B000AF0346FB80044BFA885A83DB
:109E00000C37BD465DF8047B704700BF0008024078
:109E100080B483B000AF0346FB80054B044A516910
:109E2000FA884A405A610C37BD465DF8047B70479A
:109E30000008024080B483B000AF03463960FB8065
:109E40003B68002B03D0064BFA881A8302E0044BD0
:109E5000FA885A830C37BD465DF8047B704700BF13
:109E60000008024080B483B000AF0346FB80054B7E
:109E70005A69FB88134018460C37BD465DF8047BD1
:109E8000704700BF0008024080B586B000AF0346AF
:109E900087ED020AC7ED010AFB8100237B61FB8984
:109EA00003F48073002B03D07B6943F004037B61D0
:109EB000FB8903F40073002B01D008237B61FB892D
:109EC00003F44063002B00D03AE0FB8903F44073B5
:109ED000002B00D134E00320FBF75EFB1A4B1B88FC
:109EE0009BB203F00103002B20D1FB8903F48073A4
:109EF000002B06D01548FBF773F803201349FBF736
:109F0000C1FBFB8903F40073002B06D01048FBF75C
:109F100067F803200E49FBF7B5FB032097ED020A13
:109F2000D7ED010A7969FBF789FD09E07B69DBB2AE
:109F3000032097ED020AD7ED010A1946FBF76CFEE4
:109F40001837BD4680BD00BF0004004088220108CC
:109F50008C22010880B483B000AF0346FB80FA88EE
:109F6000064B1B681340002B0CBF00230123DBB200
:109F700018460C37BD465DF8047B704794100020EE
:109F800080B485B000AF0346FB80FA88144B1B6891
:109F90001340FB60FA88134B1B681340BB60FA68E0
:109FA000BB689A4215D0FB68002B06D0FA880D4B8F
:109FB0001B681A430B4B1A6006E0FB88DA43094B17
:109FC0001B681A40074B1A60FB68002B01D0012365
:109FD00000E0002318461437BD465DF8047B704747
:109FE000941000209810002080B582B000AF7860F7
:109FF000F6F7B4FB4FF47A70FAF70CFB7868FFF7CA
:10A000007DFEFFF711FD0837BD4680BD81F00041A0
:10A0100002E000BF83F0004330B54FEA41044FEA4D
:10A02000430594EA050F08BF90EA020F1FBF54EAE8
:10A03000000C55EA020C7FEA645C7FEA655C00F084
:10A04000E2804FEA5454D4EB5555B8BF6D420CDD55
:10A050002C4480EA020281EA030382EA000083EAD8
:10A06000010180EA020281EA0303362D88BF30BD78
:10A0700011F0004F4FEA01314FF4801C4CEA1131CE
:10A0800002D0404261EB410113F0004F4FEA03332D
:10A090004CEA133302D0524263EB430394EA050FB8
:10A0A00000F0A780A4F10104D5F1200E0DDB02FA27
:10A0B0000EFC22FA05F2801841F1000103FA0EF2BB
:10A0C000801843FA05F359410EE0A5F120050EF181
:10A0D000200E012A03FA0EFC28BF4CF0020C43FAB2
:10A0E00005F3C01851EBE37101F0004507D54FF0BF
:10A0F000000EDCF1000C7EEB00006EEB0101B1F50F
:10A10000801F1BD3B1F5001F0CD349085FEA300054
:10A110004FEA3C0C04F101044FEA445212F5800F5F
:10A1200080F09A80BCF1004F08BF5FEA500C50F1FC
:10A13000000041EB045141EA050130BD5FEA4C0CDF
:10A14000404141EB010111F4801FA4F10104E9D168
:10A1500091F0000F04BF01460020B1FA81F308BF5F
:10A160002033A3F10B03B3F120020CDA0C3208DD2B
:10A1700002F1140CC2F10C0201FA0CF021FA02F106
:10A180000CE002F11402D8BFC2F1200C01FA02F176
:10A1900020FA0CFCDCBF41EA0C019040E41AA2BF9B
:10A1A00001EB0451294330BD6FEA04041F3C1CDA63
:10A1B0000C340EDC04F11404C4F1200220FA04F083
:10A1C00001FA02F340EA030021FA04F345EA03012D
:10A1D00030BDC4F10C04C4F1200220FA02F001FAEF
:10A1E00004F340EA0300294630BD21FA04F0294671
:10A1F00030BD94F0000F83F4801306BF81F480110A
:10A200000134013D4EE77FEA645C18BF7FEA655C7C
:10A2100029D094EA050F08BF90EA020F05D054EA4E
:10A22000000C04BF1946104630BD91EA030F1EBF53
:10A230000021002030BD5FEA545C05D14000494157
:10A2400028BF41F0004130BD14F580043CBF01F54A
:10A25000801130BD01F0004545F0FE4141F4700130
:10A260004FF0000030BD7FEA645C1ABF194610460B
:10A270007FEA655C1CBF0B46024650EA013406BF0C
:10A2800052EA033591EA030F41F4002130BD00BFCB
:10A2900090F0000F04BF0021704730B54FF4806488
:10A2A00004F132044FF000054FF0000150E700BF09
:10A2B00090F0000F04BF0021704730B54FF4806468
:10A2C00004F1320410F0004548BF40424FF0000155
:10A2D0003EE700BF42004FEAE2014FEA31014FEA98
:10A2E00002701FBF12F07F4393F07F4F81F06051E7
:10A2F000704792F0000F14BF93F07F4F704730B556
:10A300004FF4607401F0004521F0004120E700BFE8
:10A3100050EA010208BF704730B54FF000050AE06F
:10A3200050EA010208BF704730B511F0004502D570
:10A33000404261EB41014FF4806404F132045FEA72
:10A34000915C3FF4DCAE4FF003025FEADC0C18BF17
:10A3500003325FEADC0C18BF033202EBDC02C2F10D
:10A36000200300FA03FC20FA02F001FA03FE40EA9F
:10A370000E0021FA02F11444C1E600BF70B54FF09F
:10A38000FF0C4CF4E06C1CEA11541DBF1CEA135581
:10A3900094EA0C0F95EA0C0F00F0DEF82C4481EAE9
:10A3A000030621EA4C5123EA4C5350EA013518BF09
:10A3B00052EA033541F4801143F4801338D0A0FBF6
:10A3C00002CE4FF00005E1FB02E506F00042E0FBA3
:10A3D00003E54FF00006E1FB03569CF0000F18BFA9
:10A3E0004EF0010EA4F1FF04B6F5007F64F5407451
:10A3F00004D25FEA4E0E6D4146EB060642EAC621E4
:10A4000041EA55514FEAC52040EA5E504FEACE2E50
:10A41000B4F1FD0C88BFBCF5E06F1ED8BEF1004F53
:10A4200008BF5FEA500E50F1000041EB045170BDCF
:10A4300006F0004646EA010140EA020081EA030113
:10A44000B4EB5C04C2BFD4EB0C0541EA045170BD0F
:10A4500041F480114FF0000E013C00F3AB8014F189
:10A46000360FDEBF002001F0004170BDC4F10004D2
:10A47000203C35DA0C341BDC04F11404C4F1200553
:10A4800000FA05F320FA04F001FA05F240EA0200AE
:10A4900001F0004221F0004110EBD37021FA04F6E4
:10A4A00042EB06015EEA430E08BF20EAD37070BD9E
:10A4B000C4F10C04C4F1200500FA04F320FA05F0FD
:10A4C00001FA04F240EA020001F0004110EBD370FF
:10A4D00041F100015EEA430E08BF20EAD37070BD6F
:10A4E000C4F1200500FA05F24EEA020E20FA04F348
:10A4F00001FA05F243EA020321FA04F001F00041F7
:10A5000021FA04F220EA020000EBD3705EEA430E67
:10A5100008BF20EAD37070BD94F0000F0FD101F096
:10A520000046400041EB010111F4801F08BF013CCF
:10A53000F7D041EA060195F0000F18BF704703F00D
:10A540000046520043EB030313F4801F08BF013D94
:10A55000F7D043EA0603704794EA0C0F0CEA135550
:10A5600018BF95EA0C0F0CD050EA410618BF52EA0A
:10A570004306D1D181EA030101F000414FF0000010
:10A5800070BD50EA410606BF1046194652EA43061E
:10A5900019D094EA0C0F02D150EA013613D195EA92
:10A5A0000C0F05D152EA03361CBF104619460AD1DA
:10A5B00081EA030101F0004141F0FE4141F47001E4
:10A5C0004FF0000070BD41F0FE4141F4780170BDD4
:10A5D00070B54FF0FF0C4CF4E06C1CEA11541DBF39
:10A5E0001CEA135594EA0C0F95EA0C0F00F0A7F83B
:10A5F000A4EB050481EA030E52EA03354FEA013168
:10A6000000F088804FEA03334FF0805545EA13137A
:10A6100043EA12634FEA022245EA111545EA106542
:10A620004FEA00260EF000419D4208BF964244F1D9
:10A63000FD0404F5407402D25B084FEA3202B61AF8
:10A6400065EB03055B084FEA32024FF480104FF4CC
:10A65000002CB6EB020E75EB030E22BFB61A754640
:10A6600040EA0C005B084FEA3202B6EB020E75EBD3
:10A67000030E22BFB61A754640EA5C005B084FEA3B
:10A680003202B6EB020E75EB030E22BFB61A754608
:10A6900040EA9C005B084FEA3202B6EB020E75EB13
:10A6A000030E22BFB61A754640EADC0055EA060ED4
:10A6B00018D04FEA051545EA16754FEA06164FEA17
:10A6C000C30343EA52734FEAC2025FEA1C1CC0D1C3
:10A6D00011F4801F0BD141EA00014FF000004FF050
:10A6E000004CB6E711F4801F04BF01430020B4F111
:10A6F000FD0C88BFBCF5E06F3FF6AFAEB5EB030CC9
:10A7000004BFB6EB020C5FEA500C50F1000041EBC5
:10A71000045170BD0EF0004E4EEA113114EB5C0492
:10A72000C2BFD4EB0C0541EA045170BD41F4801165
:10A730004FF0000E013C90E645EA060E8DE60CEA6D
:10A74000135594EA0C0F08BF95EA0C0F3FF43BAF8A
:10A7500094EA0C0F0AD150EA01347FF434AF95EA41
:10A760000C0F7FF425AF104619462CE795EA0C0F25
:10A7700006D152EA03353FF4FDAE1046194622E7F2
:10A7800050EA410618BF52EA43067FF4C5AE50EACC
:10A7900041047FF40DAF52EA43057FF4EBAE12E7BC
:10A7A0004A0011D212F5001211D20DD56FF4787350
:10A7B000B3EB62520ED44FEAC12343F0004343EAA5
:10A7C000505323FA02F070474FF00000704750EAF0
:10A7D000013002D14FF0FF3070474FF0000070475A
:10A7E0004BB942B9002908BF002802D04FF0FF3111
:10A7F000084600F03BB882B0EC462DE9005000F06E
:10A800001DF8DDF804E002B00CBC70472DE9704380
:10A81000069E14461D468046894600F029F804FB32
:10A8200001F300FB0533A4FB00451D44B8EB040411
:10A8300069EB0505C6E90045BDE870832DE9704365
:10A84000069E1446804689461D4600F05DF900FBD1
:10A8500005F504FB0153A0FB04451D44B8EB0404BB
:10A8600069EB0505C6E90045BDE87083704700BF88
:10A8700000292DE9F00FC0F29F800024002BC0F2C8
:10A880009680154606460F46002B3ED18A4257D980
:10A89000B2FA82F34BB1C3F1200201FA03F720FAB6
:10A8A00002F29D40174300FA03F6290CB7FBF1F2C0
:10A8B000330C01FB127CA8B243EA0C4700FB02F305
:10A8C000BB4209D97F1902F1FF3C80F00181BB42F4
:10A8D00040F2FE80023A2F44FF1AB7FBF1F3B6B202
:10A8E00001FB137146EA014100FB03F0884208D9DD
:10A8F000491903F1FF3780F0ED80884240F2EA8089
:10A90000023B43EA0242002303E08B420AD90023C0
:10A910001A461046194614B1404261EB4101BDE8A8
:10A92000F00F7047B3FA83F8B8F1000F40F084805D
:10A930008B4202D3824200F2DE8000230122E8E74C
:10A9400012B90123B3FBF2F5B5FA85F2002A39D129
:10A950007F1B280C1FFA85FC0123B7FBF0F1320C9A
:10A9600000FB117742EA07470CFB01F2BA4207D914
:10A970007F1901F1FF3802D2BA4200F2C18041468C
:10A98000BF1AB7FBF0F2B6B200FB127046EA004005
:10A990000CFB02FC844507D9401902F1FF3702D2B3
:10A9A000844500F2AB803A4642EA0142B1E7E44313
:10A9B000524263EB430364E7404261EB41014FF0D5
:10A9C000FF345BE79540C2F1200327FA03F1280C1E
:10A9D00026FA03F39740B1FBF0F81F433B0C00FB52
:10A9E00018111FFA85FC43EA01410CFB08F38B4266
:10A9F00006FA02F608D9491908F1FF3279D28B42DA
:10AA000077D9A8F102082944C91AB1FBF0F3BFB203
:10AA100000FB131147EA01470CFB03F2BA4207D9C6
:10AA20007F1903F1FF3160D2BA425ED9023B2F4455
:10AA3000BF1A43EA084390E7C8F1200203FA08FC72
:10AA400025FA02F343EA0C0C4FEA1C4921FA02F3FF
:10AA500001FA08F720FA02F2B3FBF9F1174309FBF8
:10AA600011333A0C1FFA8CFB42EA03430BFB01FA49
:10AA70009A4505FA08F008D913EB0C0301F1FF32EF
:10AA800035D29A4533D902396344CAEB0303B3FB89
:10AA9000F9F209FB1233BFB247EA03470BFB02F995
:10AAA000B94508D917EB0C0702F1FF331BD2B945A2
:10AAB00019D9023A674442EA0145A5FB0001C9EBF6
:10AAC00007078F424FF000030AD305D02A4620E73C
:10AAD000624601E73B4614E706FA08F68642F5D2DD
:10AAE0006A1E002315E71A46E5E70B46A0E7114664
:10AAF000CBE7904688E7434642460AE7023A53E7E7
:10AB000002392F443CE700BF2DE9F00F14460546FB
:10AB10000E46002B43D18A4253D9B2FA82F757B17D
:10AB2000C7F1200620FA06F601FA07F302FA07F445
:10AB30001E4300FA07F5210CB6FBF1F22B0C01FBCA
:10AB40001267A0B243EA074600FB02F3B34209D9F9
:10AB5000361902F1FF3780F0F680B34240F2F380FD
:10AB6000023A2644F61AB6FBF1F3ADB201FB1361CB
:10AB700045EA014100FB03F0884208D9091903F1B5
:10AB8000FF3680F0E280884240F2DF80023B43EAF9
:10AB90000242002310461946BDE8F00F70478B4271
:10ABA0004AD8B3FA83F6002E4DD18B4202D38242AB
:10ABB00000F2D6800023012210461946BDE8F00FAE
:10ABC000704712B90124B4FBF2F4B4FA84F2002AFB
:10ABD0007CD1091B260CA7B20123B1FBF6F02A0C8D
:10ABE00006FB101142EA014107FB00F28A4207D935
:10ABF000091900F1FF3C02D28A4200F2C38060468C
:10AC0000891AB1FBF6F2ADB206FB121145EA014515
:10AC100007FB02F7AF4208D92C1902F1FF3180F08F
:10AC20009680A74240F29380023A42EA00421046E0
:10AC30001946BDE8F00F704700231A461046194622
:10AC4000BDE8F00F7047C6F1200522FA05F4B340C5
:10AC50001C434FEA144821FA05F301FA06F720FADB
:10AC600005F5B3FBF8FC2F4308FB1C333D0C1FFA22
:10AC700084FA45EA03430AFB0CF9994502FA06FBFC
:10AC800004D91B190CF1FF326DD39446C9EB0303B1
:10AC9000B3FBF8F508FB1533BFB247EA03470AFBDD
:10ACA00005F8B84504D93F1905F1FF3361D31D46B6
:10ACB00045EA0C4CACFB0B23C8EB07079F424FF057
:10ACC000000549D345D062462B4663E79440C2F164
:10ACD000200321FA03FC260C20FA03F301FA02F503
:10ACE000BCFBF6F843EA05010B0C06FB18CCA7B237
:10ACF00043EA0C4C07FB08F3634500FA02F509D957
:10AD00001CEB040C08F1FF323AD2634538D9A8F1A4
:10AD10000208A444C3EB0C0CBCFBF6F389B206FB9F
:10AD200013CC41EA0C4107FB03F28A4207D9091907
:10AD300003F1FF3022D28A4220D9023B2144891AF2
:10AD400043EA084349E73A460CE733461FE70A4619
:10AD50006BE7B0409042B6D20CF1FF32002319E706
:10AD60003346324616E799458FD9ACF1020C23449D
:10AD70008CE7B8459BD9023D274499E70346DEE7B7
:10AD80009046C7E7023821443AE700BF0EB410B539
:10AD9000074983B005AB0C6853F8042B01930146B7
:10ADA000204603F047F903B0BDE8104003B07047F8
:10ADB00050060020014B1868704700BF5006002065
:10ADC00070B50C46054631B110B1836B002B2FD006
:10ADD000B4F90C300BB9002070BD2846214600F0B4
:10ADE00067F8E36A064633B12846E16998470028C8
:10ADF000B8BF4FF0FF36A3891B061CD4216B41B1AD
:10AE000004F14003994202D0284600F0B9FA002329
:10AE10002363616C21B1284600F0B2FA0023636419
:10AE200000F010FA0023A38100F00EFA304670BD46
:10AE300000F048F9CCE72846216900F0A1FADDE7E7
:10AE4000024B01461868FFF7BBBF00BF5006002049
:10AE500070B582B00E46114601AA054600F0F6F91B
:10AE6000044690B1284600F0A7F9034658B10848B7
:10AE7000084D0949094A58629C81DE81DB611D62E7
:10AE80009962DA62184602B070BD02B070BD00BFB0
:10AE9000A9BF000885BF0008E1BF000801C0000885
:10AEA000024B0A4601461868FFF7D2BF5006002041
:10AEB0008B899AB22DE9F0410D46110780463CD4AA
:10AEC0006A6843F40063002AAB8159DDAC6A002C48
:10AED0004BD09BB203F48052002192B2D8F80060AC
:10AEE000C8F80010002A4FD02A6D5F0705D56968A1
:10AEF0002B6B521A0BB1EB6BD21A4046E969002357
:10AF0000A047441C4AD0AA892B692B6022F4006315
:10AF10009BB200226A60DA04AB814CD4296BC8F87A
:10AF2000006011B305F14003994202D0404600F0A1
:10AF300027FA00202863BDE8F0812E69AEB12C68A5
:10AF40002E6091070CBF6B690023A41BAB600AE065
:10AF5000324623466F6AE9694046B8470028C0EB8D
:10AF60000404064404DD002CF2DC0020BDE8F0817E
:10AF7000AB8943F04003AB814FF0FF30BDE8F08177
:10AF8000EA6B002AA2DCF0E701234046E969A0470A
:10AF9000431C02461ED0AB89AC6AA6E7D8F8003045
:10AFA0005BB9A9896B6021F400639BB22A69AB810C
:10AFB000DB042A60B2D52865B0E71D2B01D0162B23
:10AFC00019D1AA892B692B6022F400620023AA817F
:10AFD0006B60A3E7D8F80030002BDCD01D2B07D026
:10AFE000162B05D0AB8943F04003AB81BDE8F0815F
:10AFF000C8F80060B9E7AB8943F04003AB81BDE816
:10B00000F08100BF10B5044682B008B1836B53B124
:10B01000B1F90C0008B902B010BD204602B0BDE87D
:10B020001040FFF745BF019100F04CF80199EFE7A0
:10B0300020B1054B01461868FFF7E4BF034B0449F4
:10B04000186800F06BBA00BF50060020C823010842
:10B0500005B0000838B50B4D2B6804460BB19A6B50
:10B060002AB1B4F90C3033B1B4F90E0038BD18462A
:10B0700000F028F8F5E72B6809221A604FF0FF303E
:10B0800038BD00BF50060020014900F047BA00BF9C
:10B09000C1AD000870B54B1E682505FB03F50E46D3
:10B0A00005F1740100F0B4FA044640B100210C30FF
:10B0B000666005F168022160A06000F0DFFD2046B7
:10B0C00070BD00BF2DE9F04F846B83B00746002CA4
:10B0D00065D145683348F8630423032107F53B72C3
:10B0E000C7F8E412C7F8E822C7F8E04205F15C00AF
:10B0F000AB812C606C60AC606C66EC812C616C6127
:10B10000AC612146082200F0B9FDBE68DFF898B0B6
:10B11000DFF898A0DFF89890DFF89880ED610123C0
:10B120000922C5F820B0C5F824A0C5F82890C5F8B4
:10B130002C802146F381B28134607460B4607466FF
:10B1400034617461B461082206F15C00019300F07F
:10B1500095FDFD68F66112200222C6F820B0C6F8FF
:10B1600024A0C6F82890C6F82C802146A881EA8140
:10B170002C606C60AC606C662C616C61AC6105F13C
:10B180005C00082200F07AFD019BED61C5F820B05B
:10B19000C5F824A0C5F82890C5F82C80BB6303B07F
:10B1A000BDE8F08F89B0000885BF0008A9BF00087E
:10B1B000E1BF000801C00008214B70B51D68AB6BF2
:10B1C0000646002B2CD005F538756B68AC68013B42
:10B1D00005D521E0013B5A1C04F168041CD0B4F9E8
:10B1E0000C20002AF6D1002501234FF6FF72E281E0
:10B1F000A38165662560A560656025616561A561BF
:10B20000294604F15C00082200F038FD25636563DF
:10B210006564A564204670BD2B682BB11D46D4E73C
:10B220002846FFF74FFFCEE730460421FFF732FFF5
:10B23000286008B10546C8E70C23336070BD00BF25
:10B24000C8230108704700BF704700BF0B78722BFE
:10B2500030B42ED0772B27D0612B04D01623036077
:10B2600030BC002070474FF4027501244FF4847005
:10B270000CE0782B11D02B2B07D120F01C0024F0F0
:10B28000030440F0100044F0020401314B783BB15C
:10B29000622BEED144F48034F7E744F40064F4E721
:10B2A0002C43146030BC70474FF4C0650124082063
:10B2B000ECE700252C460420E8E700BF0EB410B5EB
:10B2C00083B005AB064C53F8042B0193014620686C
:10B2D00002F0D6FE03B0BDE8104003B0704700BFD7
:10B2E00050060020F8B5234D0F46044600F010FD2F
:10B2F000AB685E6826F00306F11B01F6EF7121F4DE
:10B300007F6121F00F01A1F58057B7F5805F07DB62
:10B310002046002100F04AFDAB683344984204D037
:10B32000204600F0F7FC0020F8BD2046794200F0EE
:10B330003DFD01300DD0104BAA681968F61B46F090
:10B3400001062046C91B5660196000F0E3FC01208D
:10B35000F8BD2046002100F029FDAB68C21A0F2A73
:10B36000DEDD064D04492D6842F00102401B5A60A3
:10B370000860D5E754060020A8100020600A0020CD
:10B380002DE9F0410D460646002955D000F0C0FCDD
:10B3900055F8041CDFF874C121F00103A5F108047D
:10B3A000E218DCF808005768904227F0030769D0DC
:10B3B00011F00101576032D00021D0194068C00758
:10B3C00006D43B44906800294ED0D268C260906099
:10B3D00043F001026260E350E1B9B3F5007F2DD381
:10B3E0005A0A042A6AD89809383041000CEB810CBB
:10B3F0004649DCF80820624566D0516821F0030117
:10B400008B4202D292689445F7D1D368E360A26080
:10B410009C60D4603046BDE8F04100F07BBC55F83C
:10B42000085C641B0CF10808A06840452B4443D01D
:10B43000E568C560A860C0E7BDE8F081DB080CEBFB
:10B44000C3020125DCF804009168A1609B1005FA95
:10B4500003F31843E260CCF8040094603046CC60FB
:10B46000BDE8F04100F056BC294DA842ADD143F0F3
:10B470000102CCF81440CCF81040E060A06062609B
:10B48000E350C7E71F44CB0707D455F8083CE41A3C
:10B490001F44A268E368D3609A601E4B1B6847F0A4
:10B4A00001029F426260CCF80840B3D31A4B304689
:10B4B0001968FFF717FFADE701217EE7142A0CD8C2
:10B4C00002F15B00410091E74B688010012505FA0D
:10B4D00000F003434B60134698E7542A03D8180B37
:10B4E0006E30410082E7B2F5AA7F03D8D80B7730DF
:10B4F00041007BE740F254518A4203D8980C7C30DB
:10B50000410073E7FC217E2070E700BF5406002055
:10B510005C0600205C0A0020A41000202DE9F843FE
:10B5200010F53876804689461BD000277568B468C8
:10B53000013D10D4A389012B05F1FF3507D9B4F9DA
:10B540000E3001332146404601D0C84707436B1CEB
:10B5500004F16804EED13668002EE7D13846BDE824
:10B56000F88337463846BDE8F88300BF2DE9F0413F
:10B5700086B002FB03F51746984601AA0123019104
:10B5800002950595039204930C9C064608B1836BC3
:10B59000D3B1A289930406D4636E42F4005223F41B
:10B5A0000053A28163663046214603AA05F0E4F801
:10B5B00030B10598281AB0FBF7F006B0BDE8F0816D
:10B5C000404606B0BDE8F081FFF77CFDE1E700BF33
:10B5D00030B583B0054C009324680D4613460146F0
:10B5E0002A462046FFF7C2FF03B030BD50060020B8
:10B5F000024B0146186800F00BB800BF500600204F
:10B60000024B01461868FFF7BBBE00BF5006002082
:10B610002DE9F04F01F10B05162D83B0064627D911
:10B6200035F0070527D4A94225D8304600F070FB35
:10B63000B5F5FC7F26D2C14F4FEAD50C07EBCC0302
:10B64000DC689C4200F0D2816368E268A16823F064
:10B650000303234430465D68CA6045F001059160EC
:10B660005D6000F057FB0834204603B0BDE8F08F62
:10B670001025A942D9D900240C232046336003B0F9
:10B68000BDE8F08F5FEA552C00F08A80BCF1040F12
:10B6900000F260814FEA951C0CF1380C4FEA4C0126
:10B6A000A64F07EB8101CC68A14205D10CE0002B2D
:10B6B0007ADAE468A14207D0626822F00302531BE1
:10B6C0000F2BF4DD0CF1FF3C0CF1010C9B4B3C69A2
:10B6D00003F1080E744500F07E81616821F00301DA
:10B6E0004A1B0F2A00F36481002AC3F814E0C3F850
:10B6F00010E06ADAB1F5007F80F03A81C90803EB07
:10B70000C1004FEAA1085A688168A1604FF00109A1
:10B7100009FA08F848EA0202E0605A608460CC60E6
:10B720004FEAAC030120984090425BD8024206D118
:10B730002CF0030C400002420CF1040CFAD007EB91
:10B74000CC084446E146E3689C4207D145E1002A23
:10B7500080F25681DB689C4200F03F81596821F0FD
:10B7600003014A1B0F2AF2DD1C46D3F80CC054F823
:10B77000088F591945F0010942F00105C3F80490FA
:10B780003046C8F80CC0CCF8088079613961C1F83E
:10B790000CE0C1F808E04D608A5000F0BBFA63E7A6
:10B7A0007E214FF03F0C7BE72244E3685068A1689C
:10B7B00040F00105CB6030469960556000F0AAFA70
:10B7C0000834204603B0BDE8F08F214430464B6872
:10B7D00043F001034B6000F09DFA0834204603B0AB
:10B7E000BDE8F08FBC68636823F00309A94504D362
:10B7F000C5EB09030F2B00F39180514B514A196897
:10B800001368013305EB010A04EB090B00F06181B9
:10B810000AF5805A0AF10F0A2AF47F6A2AF00F0A01
:10B8200030465146019200F0C1FAB0F1FF3F804628
:10B83000019A00F00081834500F2FA80DFF810C120
:10B84000DCF80030C3455344CCF8003000F04A81A6
:10B8500012683C4901321BBFCBEB080B5B44C1F8BB
:10B860000080CCF8003018F0070300F01381C3F11A
:10B870000802C3F5805390440833C244CAF30B0A4C
:10B88000CAEB030A51463046CDF804C000F08EFAE8
:10B89000431CDDF804C000F03581C8EB00025244BF
:10B8A00042F00102DCF80030C7F808805344BC4283
:10B8B000C8F80420CCF80030DFF894A015D0B9F116
:10B8C0000F0F40F2EA806168A9F10C0222F0070232
:10B8D00001F0010EA118052042EA0E0E0F2AC4F84D
:10B8E00004E04860886000F21181174ABC68116862
:10B8F0008B4288BF1360154A11688B4288BF136062
:10B90000626822F003029542C5EB020301D80F2BB7
:10B9100004DC304600F0FEF90024A5E6621943F08D
:10B92000010345F0010565603046BA60536000F0E0
:10B93000F1F90834204603B0BDE8F08F540600202A
:10B94000A4100020600A0020A01000209C100020FD
:10B95000A8100020BCF1140F61D9BCF1540F00F203
:10B960008F804FEA153C0CF16E0C4FEA4C0197E6C4
:10B970004B0A042B58D9142B00F2AE8003F15B0262
:10B98000500007EB8000DFF8BC818368834200F041
:10B990008A805A6822F00302914202D29B68984240
:10B9A000F7D1D9687A68E160A3608C60DC60B7E6A3
:10B9B000611942F0010745F00105656030465961A3
:10B9C0001961C1F80CE0C1F808E04F608A500834F2
:10B9D00000F0A0F948E65A68A2E609F1010919F059
:10B9E000030F04F108047FF4AEAE2DE004F1080368
:10B9F0006469A34208BF0CF1020C3FF467AE23E672
:10BA000019441C464868DB6854F8082F40F00105CB
:10BA10004D603046D3609A6000F07CF924E60CF16A
:10BA20005B0C4FEA4C013BE68A0938325000A8E72C
:10BA3000BC423FF403AFBC68626822F0030262E7D5
:10BA4000D8F8008098457BD11CF0030FA8F10803BB
:10BA50000CF1FF3CF4D17B6823EA00037B604000DB
:10BA600098423FF6BFAE00283FF4BCAE0342CC463E
:10BA70007FF465AE400003420CF1040CFAD05EE6A0
:10BA8000BCF5AA7F1AD84FEAD53C0CF1770C4FEAE7
:10BA90004C0105E64FF48053EFE60123C8F804306B
:10BAA000444600222FE791100120D8F8042000FA24
:10BAB00001F10A43C8F80420194674E740F25453D0
:10BAC0009C451BD84FEA954C0CF17C0C4FEA4C017D
:10BAD000E6E50AF1100AA3E6542B1FD80A0B6E32D2
:10BAE00050004EE7CBF30B0100297FF4B1AE0AEB17
:10BAF0000901BA6841F001015160F6E6FC214FF0FE
:10BB00007E0CCDE501224FF0000ACBE604F10801DE
:10BB10003046FFF735FCDAF80030E6E6B3F5AA7FE9
:10BB200003D8CA0B773250002BE740F254529342AD
:10BB300003D88A0C7C32500023E7FC207E2220E7C9
:10BB40007B688CE754060020844641EA000313F02A
:10BB500003036DD1403A41D351F8043B40F8043B14
:10BB600051F8043B40F8043B51F8043B40F8043BD7
:10BB700051F8043B40F8043B51F8043B40F8043BC7
:10BB800051F8043B40F8043B51F8043B40F8043BB7
:10BB900051F8043B40F8043B51F8043B40F8043BA7
:10BBA00051F8043B40F8043B51F8043B40F8043B97
:10BBB00051F8043B40F8043B51F8043B40F8043B87
:10BBC00051F8043B40F8043B51F8043B40F8043B77
:10BBD00051F8043B40F8043B403ABDD2303211D317
:10BBE00051F8043B40F8043B51F8043B40F8043B57
:10BBF00051F8043B40F8043B51F8043B40F8043B47
:10BC0000103AEDD20C3205D351F8043B40F8043B16
:10BC1000043AF9D2043208D0D2071CBF11F8013B14
:10BC200000F8013B01D30B8803806046704700BFDA
:10BC3000082A13D38B078DD010F003038AD0C3F1E9
:10BC40000403D21ADB071CBF11F8013B00F8013BCB
:10BC500080D331F8023B20F8023B7BE7043AD9D38A
:10BC6000013A11F8013B00F8013BF9D20B7803705F
:10BC70004B7843708B78837060467047F0B48407CC
:10BC800043D0541E002A3ED0CDB2034603E0621ECC
:10BC9000002C38D0144603F8015B9A07F7D1032C27
:10BCA0002AD9CDB245EA05250F2C45EA054515D917
:10BCB000A4F110073F0903F1100606EB07161A4618
:10BCC000156055609560D5601032B242F8D104F02D
:10BCD0000F040137032C03EB07130DD91E46224630
:10BCE000043A032A46F8045BFAD8221F22F0030222
:10BCF0000432134404F003042CB1C9B21C4403F809
:10BD0000011BA342FBD1F0BC704714460346C6E7B3
:10BD1000704700BF704700BF0FB400B5074A83B03B
:10BD200004AB106853F8042B8168019302F0A8F962
:10BD300003B05DF804EB04B0704700BF500600206C
:10BD4000034B1B6801469A68184600F003B800BF11
:10BD50005006002070B50D461446064608B1836BA8
:10BD6000D3B1A368013B002BA36006DB23681D70E1
:10BD700023685A1C2260187870BDA26993420EDBBA
:10BD800023681D70236819780A29F2D130462246AB
:10BD9000BDE8704003F050BCFFF794F9E1E730468E
:10BDA00029462246BDE8704003F046BC38B5074C32
:10BDB0000023054608462360F4F718FB431C00D017
:10BDC00038BD2368002BFBD02B6038BD9C140020AD
:10BDD0002DE9F0413C4C25688846044616461F462E
:10BDE00015B1AB6B002B4FD0022E30D8002F2EDBBD
:10BDF00028462146FFF706F9A38900226260A26166
:10BE00001A0628D423F083039BB2022EA3812DD0DF
:10BE1000B8F1000F3CD0012E13D09BB203F0080004
:10BE20002A4AEA6380B2C4F80080C4F810806761CF
:10BE300078B113F0030F18BF0027A7600020BDE8FA
:10BE4000F08143F001037A42A381A261E5E74FF05C
:10BE5000FF30BDE8F08128462169FFF791FAA389F8
:10BE600023F083039BB2022EA381D1D1002004F1E1
:10BE7000430243F0020300250121A381A560226053
:10BE800022616161BDE8F0812846FFF71BF9ABE74D
:10BE9000002F08BF4FF480673846FFF7A9FB8046A4
:10BEA00028B1A38943F080039BB2A381B3E74FF489
:10BEB0008060FFF79DFB804618B9A3894FF0FF30E3
:10BEC000D5E74FF48067ECE75006002089B0000802
:10BED0000CB4F0B5174B0C1E9DB01F6824DB4FF45B
:10BEE000027323AD14BF04F1FF362646029006907C
:10BEF000ADF814304FF6FF7E2B46384602A9229A41
:10BF0000049607960195ADF816E000F0DDFD431CA0
:10BF1000BCBF8B233B6014B1029B00221A701DB082
:10BF2000BDE8F04002B070478B233B604FF0FF301C
:10BF3000F5E700BF500600200EB4F0B59CB021AB71
:10BF40000F4953F8042B019305466FF0004408682D
:10BF500002954FF402774FF6FF7602A90695ADF8E9
:10BF6000147004940794ADF8166000F0ADFD029BC8
:10BF700000221A701CB0BDE8F04003B0704700BF4B
:10BF80005006002010B50C46B1F90E1005F008FA65
:10BF9000002803DB236D0344236510BDA38923F42C
:10BFA0008053A38110BD00BF2DE9F0410C46898963
:10BFB0001D46CB051646074606D5B4F90E100022DD
:10BFC000022304F073FDA18921F48051A181384638
:10BFD000B4F90E1032462B46BDE8F04103F080BBA9
:10BFE00010B50C46B1F90E1004F060FDA389421C97
:10BFF0000EBF23F4805343F480532065A38110BD0A
:10C00000B1F90E1003F0E2BB024B0146186800F0D4
:10C0100003B800BF5006002070B5064608460D461E
:10C0200000F0FEF9441C21463046FFF7F1FA0646BF
:10C0300018B129462246FFF787FD304670BD00BF84
:10C0400010B504468E2900F23181DFE811F091002D
:10C050008F002D012B012901270125012301210139
:10C060001F011D011B011901170115012F011301EA
:10C0700011010F010D010B01090107010501030168
:10C080000101FF00FD00FB00F900F700F500F300DF
:10C09000F100EF00ED00EB002F012F012F012F0128
:10C0A0002F012F012F012F01E900E7002F012F01A0
:10C0B0002F012F012F012F012F012F012F012F0100
:10C0C0002F012F012F01E500E300E100DF002F0128
:10C0D0002F012F01DD002F012F012F01DB002F0188
:10C0E0002F01D9002F012F01D7002F012F012F0180
:10C0F0002F012F012F012F012F012F012F01D5001B
:10C100002F01D300D100CF002F012F01CD002F012F
:10C110002F012F012F012F012F012F012F01CB0004
:10C12000C900C700C500C300C1002F01BF00BD008A
:10C13000BB00B900B700B500B300B100AF00AD005F
:10C14000AB00A900A7002F01A500A300A1009F003C
:10C150002F012F012F012F012F019D002F012F01F2
:10C160002F019B009900970095009300564810BD41
:10C17000564810BD564810BD564810BD564810BD13
:10C18000564810BD564810BD564810BD564810BD03
:10C19000564810BD564810BD564810BD564810BDF3
:10C1A000564810BD564810BD564810BD564810BDE3
:10C1B000564810BD564810BD564810BD564810BDD3
:10C1C000564810BD564810BD564810BD564810BDC3
:10C1D000564810BD564810BD564810BD564810BDB3
:10C1E000564810BD564810BD564810BD564810BDA3
:10C1F000564810BD564810BD564810BD564810BD93
:10C20000564810BD564810BD564810BD564810BD82
:10C21000564810BD564810BD564810BD564810BD72
:10C22000564810BD564810BD564810BD564810BD62
:10C23000564810BD564810BD564810BD564810BD52
:10C24000564810BD564810BD564810BD564810BD42
:10C25000564810BD564810BD564810BD564810BD32
:10C26000564810BD564810BD564810BD564810BD22
:10C27000564810BD564810BD564810BD564810BD12
:10C28000564810BD564810BD564810BD564810BD02
:10C29000564810BD564810BD564810BD564810BDF2
:10C2A000564810BD564810BD564810BD08461146A8
:10C2B000002B14BF1A46224601F0BAFE524B00284A
:10C2C00008BF184610BD00BFD4230108CC230108C5
:10C2D000402A0108282A0108142A0108782A01089E
:10C2E00070270108A8260108E0290108F82901089B
:10C2F000E4250108A429010818280108A02A01083A
:10C30000AC240108742401087C2501087C2601085E
:10C310006C250108B42A0108C025010894270108EA
:10C32000BC2901088C2901085C290108442901085D
:10C330002429010804290108D4280108B02801088B
:10C3400070290108542A0108982801087C2801084E
:10C35000682801084C280108402801082C280108F9
:10C3600008280108F0270108DC270108C427010874
:10C37000CC280108B4270108AC2701088827010848
:10C380005C270108402701082C270108FC2601082A
:10C39000F0260108E0260108C8260108B826010891
:10C3A000902601086C2601085C2601084426010835
:10C3B0002426010804260108AC2501089C25010853
:10C3C0005C2501084C250108382501082C250108A9
:10C3D0001425010808250108F4240108E0240108B7
:10C3E000CC240108A024010890240108602401083D
:10C3F0004C24010830240108242401080C240108DD
:10C40000FC230108E0230108FC2A0108034B002259
:10C41000014618681346FFF713BE00BF5006002000
:10C4200020F0030110F00300C0F1000051F8043BBC
:10C4300000F1040C4FEACC0C6FF000021CBF22FA92
:10C440000CF213434FF0010C4CEA0C2C4CEA0C4C50
:10C45000A3EB0C0222EA030212EACC1204BF51F849
:10C46000043B0430F4D0C2F1000102EA0102B2FA46
:10C4700082F2C2F11F0200EBD20070474FF0010CB4
:10C480002DE9F003644600254FF0FF3663198B4217
:10C4900000EB06070DD23F5D10F80380B8452ED2A1
:10C4A0001D460124C6EB030C63198B4200EB060703
:10C4B000F1D34FF00109C2F800C04C4600254FF0FF
:10C4C000FF376319994200EB070C0ED91CF804C022
:10C4D00010F80380E04519D91D460124C7EB030974
:10C4E0006319994200EB070CF0D8701C01378742A2
:10C4F00024BF3846C2F80090BDE8F00370470CD066
:10C500004FF0010C2E4664466544BFE709D04FF05A
:10C5100001092F464C464D44D3E7644505D001340C
:10C52000B4E74C4504D00134CBE71D460124ADE708
:10C530001D460124C5E700BF2DE9F04FADF21C4DAB
:10C54000164607460D461046194605AA1C46FFF733
:10C5500095FF05AB80460DF2144243F8044F934219
:10C56000FBD15CB104F1FF3E002306A8F25CC3EBF3
:10C570000E010133A34240F82210F7D1059930464D
:10C580003144424604F05EFB00287AD108F1FF3CBA
:10C590000346CDF808C0B4448246CDF8048028464E
:10C5A000CDF80CC01D46A04608E025B1059A93427F
:10C5B00038BFC2EB08039A44002520460AEB080462
:10C5C000221A0021384404F0F5FA002854D1002C36
:10C5D00052D03A1906AB12F8012C53F82230002B36
:10C5E000E3D1019A08F1FF39954228BF2A464A450E
:10C5F00012D207EB0A0316F802C0985C844506EBDA
:10C60000020106D031E011F8010F13F802C0844591
:10C610002BD101324A45F6D3019B02989D4228BF97
:10C6200018461AD2DDF80CC007EB0A039CF800107C
:10C63000DDF808C013F80C2091426ED1039A06EB86
:10C64000050B06E012F8019D13F801C0E14504D185
:10C6500008465A4500F1FF31F4D1013585425ED8D4
:10C66000059DAA44C5EB0805A7E70199C1F101039F
:10C670009A4492440025A0E700200DF21C4DBDE82D
:10C68000F08FC8EB0403434538BF434601332846C7
:10C6900005934FF0000A06EB08094546A3460AEB4E
:10C6A0000B04221A0021384404F084FA0028E3D154
:10C6B000002CE1D03A1906AB12F8012C53F82230C5
:10C6C0001BBB0BF1FF38454507EB0A0012D2435D57
:10C6D00099F800209A4218BF2B4619D14A462B469A
:10C6E00005E012F8011F10F803C08C4510D101338A
:10C6F0004345F6D36B1E1DB9BFE713F1FF33BCD31F
:10C70000F15CC25C9142F8D0059B9A442046C6E792
:10C71000C5F1010292449A44F8E701989DE707EBBE
:10C720000A00AAE72DE9F04F037887B082460E464B
:10C73000002B00F0EF800A789AB1074601310125FD
:10C7400002E011F8012B5AB1934214BF002505F005
:10C75000010517F8013F0C46002BF2D1237823B9CD
:10C760003DB1504607B0BDE8F08F002007B0BDE8EE
:10C77000F08F0AF10100317805F036F8A41B8046ED
:10C780000028F2D0012CEDD0A244504594BFC0EB5C
:10C790000A0501251F2C07D9294632462346FFF7F3
:10C7A000CBFE07B0BDE8F08F214605AA3046FFF763
:10C7B00065FE0599814602463144304604F042FA4E
:10C7C00000285CD1034609F1FF3002903044039009
:10C7D000CDF804909A46284699460AEB04073A1A7F
:10C7E0000021404404F0E6F90028BED1002FBCD05F
:10C7F000019B994528BF4B469C4213D908EB030285
:10C80000F05C12F80A10884206EB03022FD108EB05
:10C810000A0504E012F8011FE85C884227D10133C1
:10C820009C42F7D8019B02994B4576D9039B08EBB4
:10C830000A0C1A781CF801309A426ED1039B06EB61
:10C84000090B06E013F8015D1CF80200854204D1D3
:10C8500011465B4501F1FF32F4D109F10109894527
:10C860005DD8059B9A44C3EB04093846B5E70198A7
:10C87000C0F1010292449A444FF00009F5E7C9EB78
:10C8800004034B4538BF4B460133284605934FF010
:10C89000000B06EB09074D460BEB0409C0EB090240
:10C8A0000021404404F086F900287FF45EAFB9F11E
:10C8B000000F3FF45AAFAC4298BF08EB0B0014D9FD
:10C8C00008EB05033A7813F80B309A421CD13A462C
:10C8D0002B4608EB0B0005E012F8011F10F803C00F
:10C8E0008C4512D101339C42F6D86B1E25B939E72D
:10C8F00013F1FF33FFF436AFF15CC25C9142F7D025
:10C90000059B9B444846C7E72B46C5F1010293446B
:10C910009B44F7E70C46012520E701999DE708EBCA
:10C920000A001FE7024B1A6801235C3200F002B8CC
:10C9300050060020F0B420B307460D4617F8016BEF
:10C9400001E0A64216D015F8014B002CF9D1EEB14A
:10C950003E460C4616F8015B00E073B114F8013B4B
:10C96000AB42FAD15DB100233B70166006463046FB
:10C97000F0BC704763B13846DEE73746E8E72E463D
:10C98000F3E710680028D7D10646F0E71660EEE717
:10C99000176006460370EAE72DE9F00F424C82B0BB
:10C9A000D4F800C001900E4600E02646344614F844
:10C9B000015B0CEB0500407800F0080000F0FF0A76
:10C9C0000028F2D12D2D5BD02B2D04BF7578B41C1F
:10C9D00033F010003CD09946BAF1000F0CBF6FF055
:10C9E000004B4FF0004BBBFBF9F8002709FB18BBCD
:10C9F00038460CE0303DAB4219DD7E1C05D0404589
:10CA000023D820D009FB0050012714F8015B0CEB60
:10CA10000506767816F0040FECD116F0030606D062
:10CA2000012E14BF57263726AD1BAB42E5DC7B1C1D
:10CA300015D0BAF1000F21D10AB1EFB9116002B0DF
:10CA4000BDE8F00F70475D45DCDD4FF0FF37DCE7F8
:10CA5000302D1AD0002BBED10A239946BCE701998C
:10CA6000BAF1000F4FF022030CBF6FF000404FF0FF
:10CA700000400B60002AE2D0611EDFE74042DBE7A6
:10CA8000B41C75784FF0010AA2E7207800F0DF00AF
:10CA9000582803D0002B9ED108239CE710236578EB
:10CAA0009946023498E700BF2002002030B4044CBD
:10CAB0000D46134601462A46206830BCFFF76CBF7E
:10CAC00050060020000000002DE9F04FC5B091464F
:10CAD0000C930891099003F0E5FF00681190FFF7AF
:10CAE0009FFC089C1490A3891A0603D52369002B88
:10CAF00001F092809FED967B8DED127B002334AC8C
:10CB00000D93049429932893169315930A932794CD
:10CB1000264699F80030002B00F0F880252B00F015
:10CB2000F58009F1010201E0252B04D01446013201
:10CB30002378002BF8D1C9EB04057DB1289B299AF5
:10CB4000C6F8009001332A44072B75602992289378
:10CB500000F3C28008360A9828440A902378002BF4
:10CB600000F0C280002394F801808DF87F301A46CF
:10CB70000B93059304F101094FF0FF34069409F17A
:10CB80000109A8F12003582B00F2CC83DFE813F051
:10CB90006F02CA03CA037602CA03CA03CA03CA03DE
:10CBA000CA03CA0319036903CA039D00C000CA036C
:10CBB0007D0284028402840284028402840284024C
:10CBC00084028402CA03CA03CA03CA03CA03CA038B
:10CBD000CA03CA03CA03CA0395027403CA037403CF
:10CBE000CA03CA03CA03CA036D03CA03CA0378008F
:10CBF000CA03CA03CA03CA03CA035900CA03CA0341
:10CC0000B402CA03CA03CA03CA03CA03CA03CA03D3
:10CC1000CA03CA03CA033C034D03740374037403B9
:10CC200004034D03CA03CA030D03CA03CA027C00EE
:10CC30002603AA03CA03DE02CA035F00CA03CA03AB
:10CC4000E400DDF814C04CF0100CCDF814C0059CC5
:10CC5000A20600F15B83059CE30600F1E585DDF8A3
:10CC600014C01CF0400F00F0DF85DDF830C0BCF8C8
:10CC700000400CF1040C00250123CDF830C092E0F7
:10CC8000059D45F010050595DDF814C01CF0200346
:10CC900040F03183DDF814C01CF0100240F0BD8577
:10CCA000DDF814C01CF0400300F0B785DDF830C09B
:10CCB000BCF800400CF1040C13460025CDF830C040
:10CCC00071E00B9C0C9364420B94059D45F00405A8
:10CCD000059599F8008052E70998089927AA04F069
:10CCE000FDFD40B934AE36E7299B23B10998089978
:10CCF00027AA04F0F3FD089C0A98A38913F0400FBB
:10CD000018BF4FF0FF3045B0BDE8F08F4C4625E727
:10CD100099F80080B8F12A0F09F1010001F01B8198
:10CD2000A8F13003092B98BF002101F28B8010F885
:10CD3000018B01EB810103EB4101A8F13003092BC9
:10CD4000F5D941EAE171069181461AE7AFF3008017
:10CD50000000000000000000059DA14C1694AF06E5
:10CD60008DF87F2040F1D081DDF830C00CF1070351
:10CD700023F0070303F108040C94D3E90045DDF820
:10CD800014C01CF0010F00F0638454EA050000F0A9
:10CD90005F8430234CF0020C8DF880308DF8818058
:10CDA000CDF814C002234FF0000A8DF87FA0069939
:10CDB000002905DBDDF814C02CF0800CCDF814C080
:10CDC00054EA050040F0C6820699002940F0C2826C
:10CDD000002B40F03984DDF814C01CF0010F00F086
:10CDE000338444AF302307F8413D049DEC1BDDF84C
:10CDF00018C000256445A8BFA446CDF81CC01095F6
:10CE0000BAF1000F02D0079D01350795059B13F07D
:10CE100002030E9302D0079D02350795DDF814C07A
:10CE20001CF0840CCDF83CC040F091820B9DDDF8E5
:10CE30001CC0CCEB050BBBF1000F40F38882BBF1AB
:10CE4000100F2999289ADFF8A0A12CDD17973046FA
:10CE500057461025CA46089EA146099C06E0ABF13C
:10CE6000100BBBF1100F00F1080017DD013210317B
:10CE7000072A2991289207604560F0DD2046314657
:10CE800027AA04F02BFD00287FF435AFABF1100B7F
:10CE9000BBF1100F2999289A34A8E7DC4C46D146FB
:10CEA000BA46179F064601320BEB010C072ACDF854
:10CEB000A4C0289286E8000C00F31B849DF87FA094
:10CEC0000836BAF1000F0FD0289B01330CF1010C8A
:10CED0000DF17F010122072BCDF8A4C0289386E82D
:10CEE000060000F3998308360E9B73B1289B01332B
:10CEF0000CF1020C20A90222072BCDF8A4C0289324
:10CF000086E8060000F3948308360F9D802D00F01C
:10CF1000CB82069DC4EB050ABAF1000F3BDDBAF1E6
:10CF2000100F289B2F4D2BDD069432464FF0100B2F
:10CF30002E466146099C089D06E0AAF1100ABAF146
:10CF4000100F02F1080217DD01331031072B299170
:10CF5000289382E84008F0DD2046294627AA04F0FD
:10CF6000BDFC00287FF4C7AEAAF1100ABAF1100F79
:10CF70002999289B34AAE7DC069C35468C46164640
:10CF80000133D444072BCDF8A4C0289386E82004AD
:10CF900000F336830836059DED0500F12582289BB8
:10CFA00037600133A444072BCDF8A4C074602893E4
:10CFB00000F310830836059C630748D50B9D07983E
:10CFC0002C1A002C43DD102C289BDFF81CA02ADD36
:10CFD000574610256246DDF82080DDF824A00AE0DF
:10CFE000002B0108202B0108CC2A0108103C102C32
:10CFF00006F1080615DD01331032072B299228931C
:10D0000037607560F2DD5046414627AA04F066FCA1
:10D0100000287FF470AE103C102C299A289B34AE67
:10D02000E9DC9446BA460133A444072BCDF8A4C0EA
:10D030002893C6F800A0746009DD0998089927AA0A
:10D0400004F04CFC00287FF456AEDDF8A4C00A9C26
:10D0500007980B9DA842ACBF241864190A94BCF130
:10D06000000F40F0C3820023289334AE51E599F8B5
:10D070000080002A7FF483AD202280E5059D45F0E5
:10D080000105059599F8008079E5059D45F0800535
:10D09000059599F8008072E50024A8F130030B94FF
:10D0A000214619F8018B01EB810103EB4101A8F145
:10D0B0003003092BF5D90B9163E5DDF814C08DF829
:10D0C0007F204CF0100CCDF814C0059CA30640F155
:10D0D000B2800C9DE91D21F00701D1E90023083140
:10D0E0000C9114461D46002A73F10000C0F28B8398
:10D0F0009DF87FA001235AE6059DB74C8DF87F204F
:10D10000AF0616943FF530AE059DED0640F1608404
:10D11000DDF830C0DCF800400CF1040CCDF830C074
:10D1200000252CE6DDF814C08DF87F201CF0200FC0
:10D1300000F040840C9C21680A9CE5172B460C9D4E
:10D14000224604350C95C1E90023E2E40C9C2768D3
:10D150004FF0000A8DF87FA0251D002F00F0F58507
:10D16000069C002C3846C0F28B855146224603F0BF
:10D1700021FD002800F05A86069C0C95C01BA04299
:10D18000B8BF044624EAE475CDF818A0CDF840A055
:10D1900007959DF87FA033E6DDF814C04CF0400CF5
:10D1A000CDF814C099F80080E9E499F80080B8F14E
:10D1B0006C0F4B4600F08F84059D45F010050595DA
:10D1C000DDE40C9C0C9D24680B94002C05F10403F9
:10D1D000FFF677AD0C9399F80080D0E40C9ADDF857
:10D1E00014C07E48146816903023151D4FF078083F
:10D1F0004CF0020C8DF880300C95CDF814C0002551
:10D200008DF881800223CEE50C9A0C9D12688DF872
:10D21000A8200023012404359A4607940C958DF824
:10D220007F30069310932AAFF0E5059C8DF87F20A0
:10D23000A3063FF54EAFDDF814C01CF0100F40F010
:10D24000D282059C670640F1CE82DDF830C0BCF981
:10D2500000400CF1040CE51722462B46CDF830C0F7
:10D2600041E799F800802B2289E4059D45F00805E7
:10D27000059599F8008082E4059C8DF87F202507AC
:10D2800040F18D830C9DEB1D23F0070393ED007B94
:10D290008DED127B03F1080CCDF830C09DED120B23
:10D2A00004F078FA012840F06183DDE912010022E0
:10D2B000002304F055FD002840F075859DF87FA0FF
:10D2C000DDF814C0464F474B002503242CF0800C9A
:10D2D00007940695CDF814C0B8F1470FD8BF1F4684
:10D2E00010958DE5DDF814C04CF0200CCDF814C07D
:10D2F00099F8008043E40C9CE31D23F0070303F13D
:10D3000008050C95D3E9004500234CE50C9DEB1D69
:10D3100023F0070303F1080CD3E90045CDF830C032
:10D32000012340E58DF87F20B8F1000F3FF4DCAC1D
:10D3300000234FF0010C9A46CDF81CC08DF8A88050
:10D340008DF87F300693109364462AAF5EE5DDF8D2
:10D35000A4C0B6E5012B00F0EC80022B0DF1CF0349
:10D3600018D1DDF858C0194604F00F00220942EA2E
:10D3700005720F462B091CF80010397052EA0300A1
:10D3800014461D4607F1FF31EED1049DCDE91A2365
:10D39000EC1B2CE5E00840EA457004F00702E908C0
:10D3A000303250EA010C1F461A7004460D4603F154
:10D3B000FF33EFD1059CCDE91801E007394640F174
:10D3C000C180302A00F0BE80049D1F463023EC1B34
:10D3D00001F8013C0BE500BFEC2A0108002B010815
:10D3E000E02A0108DC2A0108B8F1650F40F3AD809E
:10D3F000DDE9120100220023CDF80CC004F0A6FCE8
:10D40000DDF80CC0002800F02681289BAA4A326073
:10D4100001330CF1010C0122072BCDF8A4C0289395
:10D42000726000F3FB820836219B0D9CA34203DB54
:10D43000059DEC077FF5BFAD289B149D119C3460C2
:10D440000133AC44072BCDF8A4C07560289300F3DA
:10D450004C8308360D9D6C1E002C7FF7ACAD102C54
:10D46000289B964D40F3978110276246DDF8248073
:10D47000DDF820A004E00836103C102C40F38A812F
:10D4800001331032072B2992289386E8A000F2DDA1
:10D490004046514627AA04F021FA00287FF42BAC1D
:10D4A000299A289B34AEE7E70B9D0798C0EB050A45
:10D4B000BAF1000F7FF72DADBAF1100F289B7F4D09
:10D4C0002BDD0E9432464FF0100B2E466146099C20
:10D4D000089D06E0AAF1100ABAF1100F02F1080245
:10D4E00017DD01331031072B2991289382E840087A
:10D4F000F0DD2046294627AA04F0F0F900287FF441
:10D50000FAABAAF1100ABAF1100F2999289B34AA94
:10D51000E7DC0E9C35468C4616460133D444072B77
:10D52000CDF8A4C0289386E8200400F312820836C0
:10D53000EFE4002D08BF0A2C80F0388144AF30346E
:10D5400007F8414D049DEC1B51E40D9C012C289CD7
:10D5500040F3D58101340CF101030122072C37601F
:10D5600029932894726000F3DB810836DDF850803F
:10D57000119D356001349844149DCDF8A480072C8A
:10D580002894756000F3D8810836DDE91201002285
:10D59000002304F0DBFB0D9D002840F0B9806B1EDA
:10D5A000013401379844072C2894CDF8A4803760C3
:10D5B000736000F3E2800836DDF854C0159D013435
:10D5C000C44423AB072CCDF8A4C0289486E82800D7
:10D5D0007FF7F0AC0998089927AA04F07FF9002892
:10D5E0007FF489ABDDF8A4C034AEE4E4099808996F
:10D5F00027AA04F073F900283FF435ADFFF77BBB91
:10D600000998089927AA04F069F900287FF473ABF8
:10D61000DDF8A4C034AEBEE40998089927AA04F046
:10D620005DF900287FF467ABDDF8A4C034AE5BE49D
:10D630000998089927AA04F051F900287FF45BABF8
:10D64000DDF8A4C034AE60E4069C34AFFFF7CFBB76
:10D650000223FFF7A8BB219B002B40F3EB810D9C1D
:10D66000109DDDF834A0AC42A8BF2C46002CBA4473
:10D670000BDD289B37600133A444072BCDF8A4C0F1
:10D680007460289300F328830836109D24EAE4741C
:10D690002C1B002C40F3DB80102C289B074D40F303
:10D6A000B18106974FF010082F4662462546DDF8F7
:10D6B00024B0089C09E000BF1C2B0108202B0108A6
:10D6C0000836103D102D40F3998101331032072B9D
:10D6D0002992289386E88001F2DD5846214627AA40
:10D6E00004F0FCF800287FF406AB299A289B34AE9E
:10D6F000E7E70998089927AA04F0F0F800287FF4D2
:10D70000FAAA9DF87FA0DDF8A4C034AEFFF7D9BB1C
:10D710006F1E002F7FF750AF102FB54D23DD43460E
:10D720004FF0100ADDF82480DDF820B004E0103F4F
:10D73000102F06F1080615DD01341033072C29934C
:10D74000289486E82004F2DD4046594627AA04F0D2
:10D75000C5F800287FF4CFAA103F102F299B289CE2
:10D7600034AEE9DC98460134B844072CCDF8A480E7
:10D77000289486E8A0007FF71EAF0998089927AA89
:10D7800004F0ACF800287FF4B6AADDF8A480289C49
:10D7900034AE11E794460133A444072BCDF8A4C05E
:10D7A0002893356074607FF705AC13E70DF1CF0B5C
:10D7B000204629460A220023FDF712F830328BF862
:10D7C0000020204629460A220023FDF709F80446D6
:10D7D0000D4654EA050C5F460BF1FF3BE8D1049D72
:10D7E000EC1BFFF704BB0C9DDDF830C02C68E5177F
:10D7F00022462B460CF1040C002A73F10000CDF8F0
:10D8000030C0BFF675AC4FF02D0A644265EB45059C
:10D810008DF87FA00123FFF7CABA0C9D2C68043550
:10D820000C950025FFF7BFBA0C9D2C6804350C95AC
:10D8300001230025FFF7B7BA0998089927AA04F031
:10D840004DF800287FF457AADDF8A4C034AE109D2F
:10D85000219C2F440D9DAC4242DB059DE9073FD43E
:10D860000D98C7EB0A05041BAC42B8BF2546002D36
:10D870000BDD289B37600133AC44072BCDF8A4C0E7
:10D880007560289300F35282083625EAE575641B1B
:10D89000002C7FF790AB102C289B554D7FF77BAF6A
:10D8A00010276246DDF82480DDF820A004E0083669
:10D8B000103C102C7FF76EAF01331032072B2992EA
:10D8C000289386E8A000F2DD4046514627AA04F0DE
:10D8D00005F800287FF40FAA299A289B34AEE7E7C1
:10D8E000289B119D3560149D75600133AC44072B56
:10D8F000CDF8A4C0289300F3FB810836B0E7059D5E
:10D90000EA073FF527AE01340CF101080123072C8B
:10D91000CDF8A4802894376073607FF74CAE2CE775
:10D920000998089927AA03F0D9FF00287FF4E3A9F2
:10D93000299B289C34AE19E60998089927AA03F078
:10D94000CDFF00287FF4D7A9DDF8A480289C34AE51
:10D950001BE60998089927AA03F0C0FF00287FF466
:10D96000CAA9DDF8A4C034AEFFF7D3BA9DED120BFF
:10D9700003F010FF002840F0C480059D1D4F1E4B92
:10D980009DF87FA00690032425F080050794059557
:10D990001090B8F1470FD8BF1F46FFF731BA0C9C63
:10D9A000E31D23F0070393ED007B08338DED127B1D
:10D9B0000C9373E4DDF814C01CF0100F00F05381D9
:10D9C0000C9C0A9D236804340C941D60FFF7A1B8D9
:10D9D000059C640640F14081DDF830C0BCF8004091
:10D9E0000CF1040C0025CDF830C0FFF7C8B900BF1A
:10D9F000202B0108E82A0108E42A01082C463D46AC
:10DA0000069F94460133A444072BCDF8A4C0289365
:10DA1000356074603FF710AF083618E70998089929
:10DA200027AA03F05BFF00287FF465A9DDF8A4C0F6
:10DA300034AEF9E4289AB549316001320CF1010C99
:10DA40000121072ACDF8A4C02892716000F3F48068
:10DA500008361C462CB90D9D1DB9059DE8077FF5BC
:10DA6000AAAA289B1499119D356001336144149D25
:10DA70002991072B7560289300F3E98106F10802CC
:10DA80006442002C40F31781102CA14D40F34481D7
:10DA9000A34610260C46DDF82480DDF820A006E021
:10DAA0000832ABF1100BBBF1100F40F3338101339F
:10DAB0001034072B2994289382E86000F0DD40465B
:10DAC000514627AA03F00AFF00287FF414A9299CD5
:10DAD000289B34AAE5E7059C93F8018044F02004D4
:10DAE00009F101090594FFF74AB80998089927AA8E
:10DAF00003F0F4FE00287FF4FEA8DDF8A4C034AEE5
:10DB0000A8E4069C013428F0200A00F0A280BAF1B3
:10DB1000470F04D1069C002C08BF01240694DDE9C0
:10DB20001223059D002B45F480750E95C0F2A98146
:10DB30009DED127B8DED1C7B4FF0000BB8F1660F55
:10DB400000F03981B8F1460F00F03581BAF1450F88
:10DB50000CBF069C069D099808BF651C22AA25AB30
:10DB60008DE80C009DED1C0B02212A4621AB01F033
:10DB7000D7FEB8F1670F074602D0B8F1470F05D1BD
:10DB8000DDF814C01CF0010F00F09281BAF1460FCD
:10DB900007EB050400F04381DDE91C0100220023AE
:10DBA00004F0D4F8002840F00481259B9C4206D95B
:10DBB00030215A1C25921970259B9C42F9D8DB1BF9
:10DBC000BAF1470F0D9300F0DB80B8F1650F40F319
:10DBD000E181B8F1660F00F05D81219C10940D9CED
:10DBE000109DAC4200F34081DDF814C01CF0010F21
:10DBF00040F08E8125EAE5732C464FF06708BBF1B3
:10DC0000000F40F0C5800E9D07930595CDF818B024
:10DC10009DF87FA0FFF7F4B809984021FDF7F8FCC4
:10DC200020602061002800F0B781DDF820C040238B
:10DC3000CCF81430FEF75EBF0998089927AA03F0C4
:10DC40004DFE00287FF457A8219CDDF8A4C034AE17
:10DC500000E70625069562E70C9D2C6804350C95B7
:10DC60000025FFF78CB8DDF814C01CF0400F7BD006
:10DC70000C9C0A9D236804340C941D80FEF749BF58
:10DC8000CDF818A0FEF7CCFB0C9520EAE07C069DB1
:10DC9000CDF81CC0044610959DF87FA0FFF7B0B8E2
:10DCA0000998089927AA03F019FE00287FF423A8F1
:10DCB0002999289B34AADDF834C00D9C17600133E4
:10DCC0008C44072BCDF8A4C0289354603FF782AC56
:10DCD00002F10806FFF76FB90998089927AA03F01F
:10DCE000FDFD00287FF407A8DDF8A4C034AECCE425
:10DCF0000998089927AA03F0F1FD00287EF4FBAFEC
:10DD0000219CDDF8A4C034AEAAE500BF1C2B01089D
:10DD1000202B010821465C4601332144072B299121
:10DD2000289315605460BBDC0832C4E70998089951
:10DD300027AA03F0D3FD00287EF4DDAF219C0D99C6
:10DD4000DDF8A4C00C1B34AE9FE5069C1097062C92
:10DD500028BF062424EAE47CBA4606970C95CDF841
:10DD60001CC0924FFFF74CB8DDF830C00A9CDCF8BD
:10DD700000300CF1040CCDF830C01C60FEF7C9BEB9
:10DD8000219BDC1C26DB069C9C4223DB109326E7B0
:10DD90000E9D05954FF02D0A002507938DF87FA065
:10DDA0000695FFF730B84FF02D0A8DF87FA0FFF7EA
:10DDB00087BA234603E722AA25AB8DE80C00099811
:10DDC000069A9DED1C0B032121AB01F0A9FD069DD8
:10DDD0000746DBE6A8F10208013B002B2193BABFFE
:10DDE0005B422D222B22092B8DF88C808DF88D2003
:10DDF00060DC303330228DF88F308DF88E2024ABEC
:10DE00000D9D0D9C23AA9A1A012D1592144440F3DE
:10DE1000B2800134002524EAE4731095EFE63B78E4
:10DE2000302B00F08380219D2C44B5E624EAE47C6D
:10DE3000CDF81CC0069C0C95069010909DF87FA014
:10DE4000FEF7DEBF002481460694FEF79ABE0998CD
:10DE5000089927AA03F042FD00287EF44CAF219CCC
:10DE60002999289B34AA0BE6109C0D9D002CD4BF49
:10DE7000C4F1020401242C4424EAE4734FF067083F
:10DE8000BDE6139912981C9001F100411D914FF0CD
:10DE90002D0B53E6219D1095002D069C54DD002C82
:10DEA0003DD1059DE8073AD4109C24EAE473A6E628
:10DEB000259B84E60DF19A003D4DDA1785FB035151
:10DEC000C2EBA10101EB81040246A3EB440303F181
:10DED0003000092910700B4602F1FF30ECDC01F133
:10DEE00030030DF19B04D9B2844202F8011C5AD9C7
:10DEF0000DF18D00134601E013F8011BA34200F859
:10DF0000011FF9D10DF5887CC2EB4C03F63B77E796
:10DF1000109D6C1C24EAE4734FF067086FE6069DC1
:10DF20006C1C109D2C4424EAE47368E6DDE91C01B6
:10DF30000022002303F00AFF00287FF474AFC5F12C
:10DF4000010521952C4427E6FCB9059DE9071CD461
:10DF500001231C4653E60C9DDDF830C02D6899F86E
:10DF6000018006950CF10403002D0C938146BEF64A
:10DF700006AEFEF701BEDDF814C01CF001037FF40D
:10DF800048AF109324EAE47339E6069DAC1C24EAFA
:10DF9000E47334E6219B1FE7099D0C232B604FF0AF
:10DFA000FF30FEF7B0BE0DF18E0329E7142B0108F8
:10DFB00067666666AFF30080024B0146186801F0A1
:10DFC00005BC00BF5006002008B5FCF7F3FE58233F
:10DFD00003604FF0FF3008BD0EB410B583B005A943
:10DFE000064C51F8042B0191069B0146206803F072
:10DFF000C3F903B0BDE8104003B0704750060020DD
:10E0000030B4044C0D46134601462A46206830BC05
:10E0100003F0C6B95006002030B4044C0D46134638
:10E0200001462A46206830BC01F05ABB5006002049
:10E0300000207047F0B5ADF5057D04AD00934FF4B9
:10E04000007413460F4603AA29460394064603F0BC
:10E05000C5FC044680B1394630462246039B01F098
:10E060003FFBAC42039004D030462146FDF788F9CF
:10E0700003980DF5057DF0BD4FF0FF30F9E700BFC7
:10E080002DE9F04FC5B01C4689460692099002F072
:10E0900009FD00681190FEF7C3F9099D14900B94D7
:10E0A0001DB1AB6B002B00F00B81B9F80C2093B2C3
:10E0B00099040AD4D9F8641042F4005321F40051B1
:10E0C000A9F80C30C9F864109BB21A0740F1C2805D
:10E0D000D9F81020002A00F0BD8003F01A030A2BA3
:10E0E00000F0C4809FED7A7B8DED127B002334AC71
:10E0F0000D93049429932893169315930C932794C6
:10E100002646DDF818C09CF80030002B00F0DC80BB
:10E11000252B00F0D9800CF1010202E0252B00F044
:10E120008B80144601322378002BF7D10698251AEC
:10E130007DB1289B299A0698306001332A44072B29
:10E1400075602992289300F3A48008360C9929441D
:10E150000C912378002B00F0A4800023651C94F818
:10E1600001808DF87F304FF0FF341A460A930593F3
:10E17000069507942B460133A8F12001582900F297
:10E18000FE83DFE811F03D02FC03FC030903FC03FE
:10E19000FC03FC03FC03FC03FC0344023902FC0304
:10E1A00060003B03FC037B03820382038203820340
:10E1B00082038203820382038203FC03FC03FC03C9
:10E1C000FC03FC03FC03FC03FC03FC03FC035903FA
:10E1D000A303FC03A303FC03FC03FC03FC03930362
:10E1E000FC03FC03DA03FC03FC03FC03FC03FC0359
:10E1F000A902FC03FC03C902FC03FC03FC03FC03AF
:10E20000FC03FC03FC03FC03FC03FC0310032203DC
:10E21000A303A303A303DF022203FC03FC03E8021E
:10E22000FC03F402100222025102FC035A02FC0316
:10E23000A900FC03FC0381020699651A78E70A9C91
:10E240000B9164420A94059D45F00405059593F8E9
:10E25000008090E70998494601F056FAA0B9B9F84C
:10E260000C3003F01A030A2B7FF43CAFB9F90E30DF
:10E27000002BFFF637AF0998069A4946234601F06E
:10E280009FF945B0BDE8F08F4FF0FF3045B0BDE8D5
:10E29000F08F0998494627AA03F00CFC40B934AE28
:10E2A00054E7299B23B10998494627AA03F002FCA9
:10E2B000B9F80C305B06E7D40C9845B0BDE8F08F98
:10E2C0002846FCF7FFFEF0E6069C42E7AFF300802D
:10E2D0000000000000000000059C0693A20640F12B
:10E2E00006820B9DEB1D23F0070303F1080CD3E915
:10E2F0000045CDF82CC001234FF0000A8DF87FA017
:10E300000799002905DBDDF814C02CF0800CCDF84E
:10E3100014C054EA050040F04B830799002940F0EF
:10E320004783002B40F0BD84DDF814C01CF0010FC2
:10E3300000F0B78444AF302307F8413D049DEC1B47
:10E34000DDF81CC000256445A8BFA446CDF820C058
:10E350001095BAF1000F02D0089D01350895059B74
:10E3600013F002030E9302D0089D02350895DDF8E4
:10E3700014C01CF0840CCDF83CC040F016830A9DFC
:10E38000DDF820C0CCEB050BBBF1000F40F30D8393
:10E39000BBF1100F2999289ADFF828A527DD1797D8
:10E3A00010255746A246099C06E0ABF1100BBBF1C5
:10E3B000100F06F1080617DD01321031072A2991E6
:10E3C000289237607560F0DD2046494627AA03F0A1
:10E3D00071FB00287FF46CAFABF1100BBBF1100F99
:10E3E0002999289A34AEE7DC5446BA46179F013281
:10E3F0000BEB010C072ACDF8A4C0289286E8000C8C
:10E4000000F39E849DF87FA00836BAF1000F0FD06C
:10E41000289B01330CF1010C0DF17F010122072B28
:10E42000CDF8A4C0289386E8060000F320840836BF
:10E430000E9B73B1289B01330CF1020C20A9022220
:10E44000072BCDF8A4C0289386E8060000F31C84AF
:10E4500008360F9D802D00F04C83079A151B002D68
:10E460003DDD102D289BDFF860A42CDD514607947C
:10E47000AA464FF0100B6246099C0D4606E0AAF131
:10E48000100ABAF1100F06F1080617DD0133103239
:10E49000072B2992289386E82008F0DD204649467C
:10E4A00027AA03F007FB00287FF402AFAAF1100AA5
:10E4B000BAF1100F299A289B34AEE7DC9446079CEA
:10E4C0002A46554692460133AC44072BCDF8A4C0EA
:10E4D0002893C6F800A0756000F3BD830836059D3B
:10E4E000EB0500F1A682289B37600133A444072B7B
:10E4F000CDF8A4C07460289300F397830836059C78
:10E50000620740D50A9D08982C1A002C3BDD102C80
:10E51000289BDFF8B0A322DD10256246DDF82480B9
:10E52000574604E0103C102C06F1080615DD0133B7
:10E530001032072B2992289337607560F2DD404630
:10E54000494627AA03F0B6FA00287FF4B1AE103C82
:10E55000102C299A289B34AEE9DC9446BA46013344
:10E56000A444072BCDF8A4C02893C6F800A074607B
:10E5700009DD0998494627AA03F09CFA00287FF490
:10E5800097AEDDF8A4C00C9C08980A9DA842ACBFC9
:10E59000241864190C94BCF1000F40F0528300233E
:10E5A000289334AEADE5DDF814C006931CF02003CB
:10E5B00000F0CE810B9CE31D23F0070303F1080557
:10E5C0000B95D3E90045002396E60B9ADDF814C0BD
:10E5D0000693151D30234FF078084CF0020CB74815
:10E5E0008DF880300B951468CDF814C000258DF897
:10E5F0008180169002237FE693F800802B22BAE5F3
:10E6000093F80080002A7FF4B6AD2022B3E50B9C7E
:10E610000B9D24680A94002C05F10401FFF60FAE4F
:10E620000B9193F80080A6E5DDF814C04CF0200CA7
:10E63000CDF814C093F800809DE50B9C06932768E5
:10E640004FF0000A8DF87FA0251D002F00F079867D
:10E65000079C002C3846C0F22E865146224602F016
:10E66000A9FA002800F0B286079C0B95C01BA042B7
:10E67000B8BF044624EAE475CDF81CA0CDF840A04C
:10E6800008959DF87FA064E6059D8C4C0693AF0627
:10E6900016948DF87F2047D5DDF82CC00CF10703C8
:10E6A00023F0070303F108040B94D3E90045DDF8D8
:10E6B00014C01CF0010F00F0F88254EA050000F0CD
:10E6C000F48230234CF0020C8DF880308DF881807C
:10E6D000CDF814C002230FE6DDF814C006934CF009
:10E6E000100CCDF814C0059CA2063FF5FAAD059CB0
:10E6F000E30600F13483DDF814C01CF0400F00F095
:10E700002E83DDF82CC0BCF800400CF1040C002571
:10E710000123CDF82CC0EFE5059D694C0693AF06AB
:10E720008DF87F201694B7D4059DED0640F1EF8457
:10E73000DDF82CC0DCF800400CF1040CCDF82CC046
:10E740000025B4E7DDF814C04CF0400CCDF814C03F
:10E7500093F800800FE593F80080B8F16C0F19462C
:10E7600000F07B85059D45F01005059503E5DDF876
:10E7700014C006931CF0200F8DF87F2000F0A784B2
:10E780000B9C21680C9CE5172B460B9D22460435FB
:10E790000B95C1E90023B4E4059D45F001050595FD
:10E7A00093F80080E7E40B9A0B9D069312688DF8AE
:10E7B000A8200023012404359A4608940B958DF86F
:10E7C0007F30079310932AAFC9E5059C0693A306F3
:10E7D0008DF87F203CD50B9DE91D21F00701D1E983
:10E7E000002308310B9114461D46002A73F10000E6
:10E7F000C0F2D1839DF87FA0012381E593F80080CA
:10E80000B8F12A0F03F1010000F0B886A8F1300139
:10E81000092998BF002300F2298610F8018B03EB29
:10E82000830301EB4303A8F130010929F5D943EA39
:10E83000E373079303469FE4DDF814C006934CF09E
:10E84000100CCDF814C0059C8DF87F20A306C2D40F
:10E85000DDF814C01CF0100F40F0B382059C670671
:10E8600040F1AF82DDF82CC0BCF900400CF1040C83
:10E87000E51722462B46CDF82CC0B6E7059D45F09E
:10E880008005059593F8008075E40024A8F1300117
:10E890000A94204613F8018B00EB800001EB400046
:10E8A000A8F130010929F5D90A9065E4059D45F0E4
:10E8B0000805059593F800805DE400BF002B010872
:10E8C000EC2A0108402B0108302B0108059C069317
:10E8D00025078DF87F2040F10E840B9DEB1D23F062
:10E8E000070393ED007B8DED127B03F1080CCDF84F
:10E8F0002CC09DED120B02F04DFF012840F0558316
:10E90000DDE912010022002303F02AFA002840F07A
:10E9100033859DF87FA0DDF814C09F4F9F4B0025E5
:10E9200003242CF0800C08940795CDF814C0B8F19E
:10E93000470FD8BF1F4610950BE5059D069345F080
:10E9400010050595DDF814C01CF020037FF432AEED
:10E95000DDF814C01CF0100240F03F82DDF814C056
:10E960001CF0400300F03982DDF82CC0BCF80040F8
:10E970000CF1040C13460025CDF82CC0BCE4069322
:10E980008DF87F20B8F1000F3FF48BAC00234FF0DF
:10E99000010C9A46CDF820C08DF8A8808DF87F3004
:10E9A0000793109364462AAFD9E4DDF8A4C02CE5A0
:10E9B000012B00F0E380022B0DF1CF0318D1DDF81D
:10E9C00058C0194604F00F00220942EA05720F46AA
:10E9D0002B091CF80010397052EA030014461D463A
:10E9E00007F1FF31EED1049DCDE91A23EC1BA7E41A
:10E9F000E00840EA457004F00702E908303250EAC6
:10EA0000010C1F461A7004460D4603F1FF33EFD187
:10EA1000059CCDE91801E007394640F1B880302A5D
:10EA200000F0B580049D1F463023EC1B01F8013C2B
:10EA300086E4B8F1650F40F3B780DDE912010022EA
:10EA40000023CDF80CC003F081F9DDF80CC00028DC
:10EA500000F02E81289B524A326001330CF1010CE8
:10EA60000122072BCDF8A4C02893726000F36F83B6
:10EA70000836219B0D9CA34203DB059DEF077FF524
:10EA80003EAD289B149D119C34600133AC44072B90
:10EA9000CDF8A4C07560289300F3E88308360D9D77
:10EAA0006C1E002C7FF72BAD102C289BDFF8F4A0F8
:10EAB00040F39C8110256246DDF82480574604E02F
:10EAC0000836103C102C40F38F8101331032072B95
:10EAD0002992289337607560F2DD4046494627AA9F
:10EAE00002F0E8FF00287FF4E3AB299A289B34AEBC
:10EAF000E7E70A980899451A002D7FF7AEAC102D6C
:10EB0000289BDFF8A0A02CDD51460E94AA464FF0BA
:10EB1000100B6246099C0D4606E0AAF1100ABAF1F4
:10EB2000100F06F1080617DD01331032072B29926A
:10EB3000289386E82008F0DD2046494627AA02F0FF
:10EB4000B9FF00287FF4B4ABAAF1100ABAF1100F94
:10EB5000299A289B34AEE7DC94460E9C2A465546FB
:10EB600092460133AC44072BCDF8A4C02893C6F8D5
:10EB700000A0756000F3028208366EE4002D08BF25
:10EB80000A2C80F03F8144AF303407F8414D049D9A
:10EB9000EC1BFFF7D5BB00BFE02A0108DC2A010807
:10EBA0001C2B0108302B01080D9C012C289C40F3E4
:10EBB000A78101340CF101050123072C2995289424
:10EBC0003760736000F3B78108361498119931608B
:10EBD00001340544072C29952894706000F3C28104
:10EBE0000836DDE912010022002303F0AFF8002807
:10EBF00040F0BD800D9A0134531E01371D44072C8F
:10EC0000289429953760736000F389810836DDF810
:10EC100054C00134AC44159DCDF8A4C023AB072CDF
:10EC2000289486E828007FF769AC0998494627AA06
:10EC300002F040FF00287FF43BABDDF8A4C034AE07
:10EC40005DE40998494627AA02F034FF00283FF402
:10EC5000A6ACFFF72DBB0998494627AA02F02AFF68
:10EC600000287FF425ABDDF8A4C034AE37E4099862
:10EC7000494627AA02F01EFF00287FF419ABDDF8F1
:10EC8000A4C034AEFFF7D4BB0998494627AA02F0C6
:10EC900011FF00287FF40CABDDF8A4C034AEFFF701
:10ECA000D8BB079C34AFFFF74BBB0223FFF724BB55
:10ECB000219B002B40F357820D9C109DDDF8348082
:10ECC000AC42A8BF2C46002CB8440BDD289B376013
:10ECD0000133A444072BCDF8A4C07460289300F33B
:10ECE000FA820836109D24EAE4742C1B002C40F3B1
:10ECF000B180102C289BDFF80CA740F31B825146F3
:10ED00001025BA466246DDF824B00F4604E0083606
:10ED1000103C102C40F30A8201331032072B299249
:10ED2000289337607560F2DD5846494627AA02F0FD
:10ED3000C1FE00287FF4BCAA299A289B34AEE7E7DD
:10ED40000998494627AA02F0B5FE00287FF4B0AA28
:10ED50009DF87FA0DDF8A4C034AEFFF756BB0B9D35
:10ED60002C6804350B9501230025FFF7C5BA0D9BD0
:10ED70005F1E002F7FF74BAF102FDFF888A640F300
:10ED8000E6804FF01008DDF824B004E00836103FAC
:10ED9000102F40F3DC8001341035072C299528947E
:10EDA000C6F800A0C6F80480F0DD5846494627AAF8
:10EDB00002F080FE00287FF47BAA299D289C34AEB7
:10EDC000E5E70B9DDDF82CC02C680CF1040CE51771
:10EDD000CDF82CC022462B4607E50B9D2C68043548
:10EDE0000B950025FFF788BA9446BA460133A44430
:10EDF000072BCDF8A4C02893C6F800A074607FF755
:10EE00007DAB12E70DF1CF0B204629460A220023E5
:10EE1000FBF7E6FC30328BF80020204629460A2218
:10EE20000023FBF7DDFC04460D4654EA050C5F4663
:10EE30000BF1FF3BE8D1049DEC1BFFF781BA099869
:10EE4000494627AA02F036FE00287FF431AADDF8F1
:10EE5000A4C034AE109D219C2F440D9DAC4240DBDC
:10EE6000059DE8073DD40D98C7EB0805041BAC428F
:10EE7000B8BF2546002D0BDD289B37600133AC441D
:10EE8000072BCDF8A4C07560289300F34B82083699
:10EE900025EAE575641B002C7FF731AB102C289B0D
:10EEA000DFF860A5A2DD10256246DDF82480574614
:10EEB00003E00836103C102C96DD01331032072B8E
:10EEC0002992289337607560F3DD4046494627AAAA
:10EED00002F0F0FD00287FF4EBA9299A289B34AEBC
:10EEE000E8E7289B119D3560149D75600133AC44A3
:10EEF000072BCDF8A4C0289300F307820836B2E7A9
:10EF0000059DE9073FF555AE01340CF101050123DC
:10EF1000072C29952894376073607FF777AE09989E
:10EF2000494627AA02F0C6FD00287FF4C1A9299D01
:10EF3000289C34AE6BE60998494627AA02F0BAFD30
:10EF400000287FF4B5A9299D289C34AE3DE6013404
:10EF50003D44072C29952894C6F800A077607FF7D8
:10EF600055AEDCE70998494627AA02F0A3FD002820
:10EF70007FF49EA9299D289C34AE32E60998494623
:10EF800027AA02F097FD00287FF492A9DDF8A4C01B
:10EF900034AEFFF762BA4FF02D0A644265EB4505C7
:10EFA0008DF87FA00123FFF7ABB99DED120B02F0A6
:10EFB000F1FB002800F02381079C013428F0200A8F
:10EFC00000F06F82BAF1470F04D1079C002C08BFF4
:10EFD00001240794DDE91223059D002B45F480757B
:10EFE0000E95C0F255829DED127B8DED1C7B4FF08E
:10EFF000000BB8F1660F00F0DA81B8F1460F00F0AF
:10F00000D681BAF1450F0CBF079C079D099808BF30
:10F01000651C22AA25AB8DE80C009DED1C0B02217E
:10F020002A4621AB00F07CFCB8F1670F074602D0FE
:10F03000B8F1470F05D1DDF814C01CF0010F00F046
:10F040003382BAF1460F07EB050400F0CB81DDE90E
:10F050001C010022002302F079FE002840F0A58167
:10F06000259B9C4206D930215A1C25921970259B5C
:10F070009C42F9D8DB1BBAF1470F0D9300F08D814C
:10F08000B8F1650F40F39282B8F1660F00F03C8250
:10F09000219C10940D9C109DAC4200F3EC81DDF896
:10F0A00014C01CF0010F40F03C8225EAE5732C46A9
:10F0B0004FF06708BBF1000F40F064810E9D08938C
:10F0C0000595CDF81CB09DF87FA0FFF742B9DDF89B
:10F0D00014C01CF0100F40F0AB80DDF814C01CF021
:10F0E000400F00F03D810B9C0C9D236804340B9471
:10F0F0001D80FFF706B80B9CE31D23F0070393ED7B
:10F10000007B08338DED127B0B93FFF7F2BB059C60
:10F11000640640F18680DDF82CC0BCF800400CF19C
:10F12000040C0025CDF82CC0FFF7C1BA94463A462E
:10F13000574692460133A444072BCDF8A4C0289328
:10F14000C6F800A074603FF77AAE083682E60998E8
:10F15000494627AA02F0AEFC00287FF4A9A8DDF8F2
:10F16000A4C034AE85E4289AA249316001320CF182
:10F17000010C0121072ACDF8A4C0289271605FDC40
:10F1800008361C462CB90D9D1DB9059DED077FF570
:10F19000B6A9289B149A119D356001336244149DD1
:10F1A0002992072B7560289300F353810836644237
:10F1B000002C72DD102CDFF84CA240F39B805146EE
:10F1C0001025BA46DDF824800F4604E00836103CCE
:10F1D000102C40F38C8001331032072B2992289396
:10F1E00037607560F2DD4046494627AA02F062FCAE
:10F1F00000287FF45DA8299A289B34AEE7E7059D97
:10F200007D4F7E4B9DF87FA00790032425F080055D
:10F21000089405951090B8F1470FD8BF1F46FFF727
:10F2200098B80B9D2C6804350B950025FFF73FBA65
:10F230000B9C0C9D236804340B941D60FEF761BF8A
:10F240000998494627AA02F035FC00287FF430A827
:10F25000219CDDF8A4C034AE94E7059C91F80180B0
:10F2600044F0200401330594FEF785BF0998494610
:10F2700027AA02F01FFC00287FF41AA8DDF8A4C01A
:10F2800034AE0CE40998494627AA02F013FC002882
:10F290007FF40EA8299A289B34AEDDF834C00D9C6B
:10F2A000376001339444072BCDF8A4C028937460D1
:10F2B0007FF724A9B9E4CDF81CA0FDF7B1F80B95B0
:10F2C00020EAE07C079DCDF820C0044610959DF80B
:10F2D0007FA0FFF73EB80998494627AA02F0EAFB4B
:10F2E00000287EF4E5AFDDF8A4C034AEFAE4394678
:10F2F00057468A4601332244072B29922893C6F8A1
:10F3000000A07460BEDC0836C7E70998494627AA02
:10F3100002F0D0FB00287EF4CBAF219CDDF8A4C026
:10F3200034AEA0E50998494627AA02F0C3FB00289D
:10F330007EF4BEAF219C0D99DDF8A4C00C1B34AE49
:10F34000A6E5079C1097062C28BF062424EAE47C37
:10F35000BA4607970B95CDF820C0294FFEF7F9BFA5
:10F36000DDF82CC00C9CDCF800300CF1040CCDF85E
:10F370002CC01C60FEF7C5BE4FF02D0A8DF87FA093
:10F38000FFF7C9BA0E9D05954FF02D0A0025089389
:10F390008DF87FA00795FEF7DFBF219BDC1C33DBD8
:10F3A000079C9C4230DB109374E6234662E622AA57
:10F3B00025AB8DE80C000998079A9DED1C0B0321E5
:10F3C00021AB00F0ADFA079D07463AE624EAE47C5B
:10F3D000CDF820C0079C0B95079010909DF87FA05A
:10F3E000FEF7B7BF3B78302B00F0A280219D2C4464
:10F3F0002DE600BF1C2B0108E82A0108E42A0108B9
:10F40000142B0108302B0108A8F10208013B002B46
:10F410002193BABF5B422D222B22092B8DF88C80C1
:10F420008DF88D2042DC303330228DF88F308DF80E
:10F430008E2024AB0D9D0D9C23AA9A1A012D1592A6
:10F44000144440F391800134002524EAE4731095BC
:10F4500030E60998494627AA02F02CFB00287EF4E2
:10F4600027AF219C299A289B34AEA0E600240346AE
:10F470000794FEF781BE109C0D9D002CD4BFC4F1F3
:10F48000020401242C4424EAE4734FF0670811E6D7
:10F49000139912981C9001F100411D914FF02D0B12
:10F4A000A7E50625079595E5259BE3E50DF19A006F
:10F4B000414DDA1785FB0351C2EBA10101EB810439
:10F4C0000246A3EB440303F13000092910700B46F8
:10F4D00002F1FF30ECDC01F130030DF19B04D9B2F5
:10F4E000844202F8011C63D90DF18D00134601E03E
:10F4F00013F8011BA34200F8011FF9D10DF5887C18
:10F50000C2EB4C03F63B95E7219D1095002D079C1F
:10F5100023DDDCB9059DE80718D4109C24EAE473C8
:10F52000C8E5109D6C1C24EAE4734FF06708C1E540
:10F53000DDE91C010022002302F008FC00287FF412
:10F5400055AFC5F1010521952C4480E5079D6C1C44
:10F55000109D2C4424EAE473ACE514BB059DE90737
:10F560001FD401231C46A5E5DDF814C01CF00103DF
:10F570007FF469AF109324EAE4739BE50B9DDDF8FB
:10F580002CC02D6893F8018007950CF10401002D23
:10F590000B910346BEF6EFAD4FF0FF340794FEF734
:10F5A000EABD079DAC1C24EAE47383E5219B2DE7AB
:10F5B0000DF18E033EE700BF67666666AFF300801D
:10F5C0002DE9F0430C46ADF26C4DB1F80C90E769B3
:10F5D000496EB4F80E8019911AAD4FF480664FF061
:10F5E000000E079729F00209676A0095694604959D
:10F5F00002960596ADF80C90ADF80E800997CDF8FF
:10F6000018E00646FEF73CFD051E07DB304669465E
:10F61000FBF7F8FC002818BF4FF0FF35BDF80C30A1
:10F620005B0603D5A38943F04003A38128460DF26E
:10F630006C4DBDE8F08300BFF8B50D461446074693
:10F6400010B1836B002B48D0A289A369A36093B249
:10F65000180738D52669002E35D09904EDB215D596
:10F66000236862699E1B96421CDA0136A268591C07
:10F67000013AA26021601D706369B3421AD0A38968
:10F68000DB0701D50A2D15D02846F8BD636E23F49B
:10F69000005342F4005263662368A28162699E1B94
:10F6A0009642E2DB38462146FBF7ACFC40B92368C2
:10F6B0000126DBE738462146FBF7A4FC0028E3D00F
:10F6C0004FF0FF30F8BD3846214600F01DF8002805
:10F6D000F6D1A289266993B2BFE7FBF7F3FCB3E743
:10F6E00070B5084C06460025084611461A462560A6
:10F6F000F0F71EFF431C00D070BD2368002BFBD029
:10F70000336070BD9C1400202F4B1B6870B50646FB
:10F710000C4613B19A6B002A36D0A589ABB21907F3
:10F720000CD52269AAB113F001011ED06369002132
:10F730005B42A361A160F2B1002070BDDA063BD547
:10F740005B0725D4226945F00803A3819BB2002AF8
:10F75000E9D103F42071B1F5007FE4D030462146B1
:10F7600001F0B8F9A3892269DDE7980758BF6169FC
:10F77000A160002AE0D1A3891A06DDD543F0400339
:10F78000A3814FF0FF3070BD1846FBF79BFCC4E728
:10F79000216B49B104F14003994203D03046FBF795
:10F7A000EFFDA5890023236325F0240500232269AA
:10F7B0006360ADB22260C6E745F0400509233360BF
:10F7C0004FF0FF30A58170BD5006002038B5074CC2
:10F7D0000023054608462360F0F756FE431C00D080
:10F7E00038BD2368002BFBD02B6038BD9C14002053
:10F7F0002DE9F04F03690D699D4283B0834600F304
:10F800008B80013D01F1140400F1140A54F8252005
:10F810005AF825300132B3FBF2F8AA009146009263
:10F820005244A1440192B8F1000F3DD04FF0000EB8
:10F830007046224653468C4652F8046B1968B7B29C
:10F84000360C07FB08EE06FB08F606EB1E461FFA11
:10F850008EF7C71BB0B217FA81F7C0EB114000EB6F
:10F860002740BFB247EA0047914543F8047B4FEA7F
:10F8700020404FEA164EDFD2009A5AF80230614615
:10F8800093B9019A131F9A450CD252F8043C4BB914
:10F89000A2F1080302E01A68043B1AB99A4505F17F
:10F8A000FF35F8D3CBF81050584601F07DFC002806
:10F8B0002EDB08F101085346002254F8046B186847
:10F8C000B1B2521A360C12FA80F1C6EB104202EBBA
:10F8D000214289B241EA0241A14543F8041B4FEAA3
:10F8E0002242EAD25AF825200AEB850382B91A1F70
:10F8F00092450BD253F8042C42B9083B02E01A6837
:10F90000043B1AB99A4505F1FF35F8D3CBF81050EE
:10F91000404603B0BDE8F08F002003B0BDE8F08F93
:10F920002DE9F04F9DB004460491016C269D06928E
:10F9300009935BEC10AB49B1436C4B60012202FAB6
:10F9400003F38B6001F038FA00232364BBF1000F4E
:10F95000D94635DB00232B60A54B1A4609EA030381
:10F96000934216D0002200235046594602F0EEF989
:10F9700056465F46804648B3099E01233360279E62
:10F98000002E00F0C9809B48306001381DB0BDE8F2
:10F99000F08F099E42F20F733360BAF1000F00F04E
:10F9A000A4809548279E002EF0D0C378002B00F04D
:10F9B000B58000F10803279E33601DB0BDE8F08FCD
:10F9C00001232BF000492B60CB46C5E7204647ECCE
:10F9D000106B1BA91AAA01F075FC5FEA19550C906F
:10F9E00040F08C801A9F1B9D6FF482633D449D42C2
:10F9F000C0F297821F3305F212425B1B09FA03F330
:10FA00002AFA02F243EA0200FAF742FC0126013D1B
:10FA1000B846A1F1F87118960022784BFAF7FAFA75
:10FA20006DA3D3E90023FAF7A9FC6DA3D3E9002362
:10FA3000FAF7F2FA064628460F46FAF739FC6AA3A7
:10FA4000D3E90023FAF79AFC02460B4630463946C2
:10FA5000FAF7E2FA06460F4602F0AAF9394608908C
:10FA600000223046002302F07BF9002840F02A8271
:10FA7000089E162E00F22382614B03EBC603D3E9E6
:10FA8000000152465B4602F089F9002800F04E82E0
:10FA9000013E089600261096C5EB0805013D079526
:10FAA00000F12A8200260A96089E002EC0F21882D3
:10FAB000DDF81CE00F96B6440026CDF81CE00E964B
:10FAC000049E092E2CD8052EC4BF043E049604992A
:10FAD000A1F10203CCBF00260126032B22D8DFE8C8
:10FAE00013F0AE03A302B703AB04464A424BC9F37B
:10FAF000130000280CBF1046184653E7CBF313033E
:10FB000043F07F51CDF860805046A5F2FF3541F4B7
:10FB10004011DDF868807FE73B4837E7C31C4AE7C0
:10FB200000260496002565642946204601F01EF94A
:10FB30004FF0FF3901260B9006952064CDF84490D4
:10FB40000D961B9B002BC0F2D180089E0E2E00F359
:10FB5000CD802B4B03EBC60393ED007B069E002E5E
:10FB60008DED047BC0F27783DDE9042359465046CE
:10FB7000FAF72EFD02F01CF90546FAF799FBDDE9CC
:10FB80000423FAF7FBFB0B46024659465046FAF7A8
:10FB900041FADDF82CE005F13003B9F1010F06461A
:10FBA0000F468EF800300EF1010B61D00022174B8A
:10FBB000FAF7E4FB0022002306460F4602F0C6F8DF
:10FBC00000287ED1DDF82C800B9B0694C844DDE92B
:10FBD00004AB03F1020926E061436F63A787D23FBC
:10FBE000B3C8608B288AC63FFB799F501344D33F2C
:10FBF0000000F07F1D2B01085C2B01080000F83F7E
:10FC0000702B0108502B01081C2B01080000244018
:10FC1000FAF7B4FB0022002306460F4602F096F8DE
:10FC2000002840F0D38352465B4630463946FAF707
:10FC3000CFFC02F0BDF80546FAF73AFB52465B46A8
:10FC4000FAF79CFB02460B4630463946FAF7E2F9D2
:10FC500005F1300EC14509F801EC4C4606460F4649
:10FC60004FF00002A94B09F10109D1D1A346069C2E
:10FC700032463B4630463946FAF7CEF906460F463D
:10FC80003246DDE904013B4602F06AF840B9DDE99D
:10FC9000040132463B4602F059F890B1EB0710D50B
:10FCA0001BF8015C0B9A05E09A4200F0318413F8CE
:10FCB000015C9B46392D0BF1FF33F5D06A1CD2B2A3
:10FCC0001A7020460C9901F077F8089E731C099E63
:10FCD00000228BF800203360279E002E00F01E8348
:10FCE0000B98C6F800B01DB0BDE8F08F0D9E002E39
:10FCF00000F00781049E012E40F3D5820E9E09F18B
:10FD0000FF37BE42C0F29B83F71BB9F1000FC0F270
:10FD100092840A9D4B460A9E1E440A96079E2046E0
:10FD20001E440121079601F0EBF8064665B10799DC
:10FD3000002909DD0B460A9AAB42A8BF2B46D21A0E
:10FD4000C91A0A92ED1A07910E9B002B1BDD0D9923
:10FD5000002900F06A83002F11DD31463A46204623
:10FD600001F076F9064631460C9A204601F0D2F8A9
:10FD70000C998046204601F01FF8CDF830800E9B8C
:10FD8000DA1B40F08A820121204601F0B9F80F9970
:10FD90000029804605DD01460F9A204601F058F9FA
:10FDA0008046049A012A40F3CB8200270F9900294C
:10FDB00040F0AA820120079B034413F01F0300F0C8
:10FDC000A780C3F12002042A40F3C9840A9ADDF80F
:10FDD0001CE0C3F11C031A449E440A921D44CDF852
:10FDE0001CE00A9B002B05DD0C991A46204601F009
:10FDF0007DF90C900799002905DD4146079A2046B8
:10FE000001F074F98046109A002A40F06282B9F13C
:10FE1000000F40F3B0820D9A002A40F089800D9DBA
:10FE20000C9FDDF82CB006E0394620460A2200235C
:10FE300000F0CCFF074638464146FFF7D9FC30308A
:10FE40000BF805000135A945EEDCDDF82CB00C9768
:10FE50008246B9F1010FACBFCB440BF1010B002579
:10FE60000C990122204601F041F941460C9001F025
:10FE70009BF9002840F311831BF8012C0B9905E036
:10FE8000994200F09A8213F8012C9B46392A0BF113
:10FE9000FF33F5D001321A704146204600F08CFF46
:10FEA000002E3FF40EAF2DB1B54203D029462046B7
:10FEB00000F082FF3146204600F07EFF01E7012678
:10FEC0001096E9E50898FAF7F3F932463B4601F057
:10FED0003DFF00287FF4CCAD089E013E0896C7E5A3
:10FEE0000A9EDDF820E0CEEB06060A96CEF100066B
:10FEF0000E9600260F96E3E56E420A9600260796B8
:10FF0000D2E50E9F0A9D0D9E10E700BF0000244021
:10FF10001C230A99079A19441A440A911D4407920E
:10FF20005FE74048401B0AFA00F06DE51090B3E52A
:10FF3000002D05DD31462A46204601F0D7F8064659
:10FF4000002F40F0EF8237460B9B0B9A4B440AF090
:10FF500001010A930D91551CDDF830900AE000F084
:10FF600035FF394606460A222046002300F02EFFC0
:10FF70000746013541464846FFF73AFC314683467D
:10FF8000484601F011F93A4606904146204601F0F4
:10FF90002FF9C26805F1FF3E03460BF1300ACDF898
:10FFA0001CE0002A40F0888119464846039301F07E
:10FFB000FBF8039B024619462046039200F0FCFE24
:10FFC000039A2AB9049919B90D9B002B00F0A78355
:10FFD000069B002BC0F2428205D1049919B90D9BF2
:10FFE000002B00F03B82002A00F3B0820A9905F84A
:10FFF00001AC8D42AB4600F0BA8249460A2200238A
:020000040801F1
:10000000204600F0E3FEBE428146314620464FF0D6
:100010000A024FF00003A2D100F0D8FE06460746C0
:10002000A7E700BFEEFBFFFF00210D91069A089B9A
:100030001A4402F10109B9F1000F11924D4640F343
:1000400045810021172D61640AD9012204235B0038
:1000500003F11400A842114602F10102F7D96164CC
:10006000204600F083FE0E2D0B9020643FF669AD14
:10007000002E3FF466AD089E002ECDE914AB40F390
:100080002082A84B06F00F0203EBC2033511D3E91F
:100090000067EB0640F1DB81A34B50465946D3E99C
:1000A0000823FAF795FACDE9120105F00F054FF094
:1000B00003088DB1DFF870A230463946EE0705D54A
:1000C000DAE90023FAF75AF908F101086D100AF18C
:1000D000080AF3D106460F46DDE9120132463B46D7
:1000E000FAF776FA82468B46109E46B1504659463C
:1000F00000228E4B01F034FE002840F0BD824046C5
:10010000FAF7D6F852465B46FAF738F90022884BE0
:10011000F9F782FF0646A1F15077B9F1000F00F020
:10012000688108991991C8460D9A002A00F0288222
:100130007C4B804903EBC80353E902230020FAF704
:1001400047FA32463B46F9F765FFCDE912015946B9
:10015000504601F02DFE0546FAF7AAF802460B4676
:1001600050465946F9F756FF30350B9ECDE9000150
:10017000EDB23570DDE91201DDE9002306F1010B76
:1001800001F00CFE002840F0BF82DDE900230020D2
:100190006649F9F73FFF02460B46DDE9120101F01F
:1001A000FDFD002840F0B682B8F1010F40F38581D3
:1001B000B044CDF85890A246C146DDE90067DDE9BC
:1001C00012450DE000205949F9F724FF22462B463D
:1001D00001F0C6FD002840F09B82CB4500F06A810B
:1001E000204629460022544BFAF7C8F80022524B09
:1001F00004460D4630463946FAF7C0F80F46064623
:1002000001F0D6FD8046FAF753F802460B46304619
:100210003946F9F7FFFE08F130085FFA88F8224600
:100220002B460BF8018B06460F4601F099FD32462E
:100230003B460028C6D0199E0896544641E5002248
:100240000D92069B002B3DDD1D4611939946F8E665
:1002500001230D93F5E7B9F1000F3FF785AC40F0AE
:10026000E0800022354BDDE90401FAF787F85246B9
:100270005B4601F089FDC8464E46002800F091809B
:10028000069BDDF82CB0DB4308934146204600F086
:1002900093FD002E7FF40EAE13E50C99204600F07E
:1002A000D7FE0C906FE5189E002E00F0CA8103F275
:1002B00033430E9F0A9D2EE50146204600F07CFD4B
:1002C000012285E601251195A94606950021616464
:1002D000C6E60C98414600F067FF0028BFF697ADD0
:1002E000DDF820E00C990EF1FF3E20460A220023A3
:1002F000CDF820E000F06AFD0D990C90002940F047
:100300002082DDF8449082E5D8F8103008EB8303B2
:10031000186900F0A7FDC0F120004CE50B98FFF72D
:1003200035BB00BF702B0108382C01080000F03FDE
:1003300000001C400000E03F00002440000014408A
:10034000BAF1000F7FF431ADCBF31303002B40F073
:100350007F812BF000473F0D3F05002F3FF426AD76
:100360000A9BDDF81CE001330EF1010E0A93CDF873
:100370001CE001271AE5049A022A7FF74CADB9F177
:10038000000F7FF47DAF41464B460522204600F02A
:100390001DFD804641460C9800F006FF00287FF7BF
:1003A0006FAFDDF820E00B9931230EF1010ECDF88F
:1003B00020E00B7001F1010B67E7089ADDF82CE0F3
:1003C0003123013208928EF8003065E5A346069C81
:1003D00077E44046F9F76CFF02460B465046594613
:1003E000F9F7CCFF00229E4BF9F716FE0646A1F165
:1003F00050775046594600229A4BF9F70BFE324689
:100400003B4682468B4601F0C9FC002840F0B48090
:10041000324607F100435046594601F0A1FC00283E
:100420004BD04FF0000846462AE70C990E9A20461A
:1004300000F00EFE0C90A6E401210D91F6E50E9E53
:100440000E97BB1B0F9E1E440F9600275DE49DED8B
:10045000147B4FF002088DED127B2AE6002ACDF8BE
:100460003090D94611DD0C990122204600F03EFE65
:1004700041460C9000F098FE002840F35B81BAF1F1
:10048000390F00F0238109F1310A3546079E86F8BD
:1004900000A006F1010B3E46FEE403D11AF0010F65
:1004A0007FF4EAAC5B469B46013B1BF8012C302AEB
:1004B000F9D0F1E4DDF858905446DDE914ABFFF7CC
:1004C00040BB089E7542002D00F0C580664B05F0CC
:1004D0000F0203EBC203D3E90023DDE91401F9F7AE
:1004E0004DFF2D1182468B4600F036815F4E4FF056
:1004F0000208EA0705D5D6E90023F9F73FFF08F11E
:1005000001086D1006F10806F3D182468B46EBE533
:10051000089E013608960B9E3022327031221A70E6
:10052000FFF7CFBB7168204600F020FC33699A1CAE
:100530000546920006F10C010C30FBF705FB204646
:100540002946012200F0D2FD0746FDE4BAF1390F39
:10055000CDF8309000F0BA80DDF81CE00AF101031C
:1005600035468EF800300EF1010B3E4694E43546D8
:10057000CDF830903E4673E44FF00008464610E751
:10058000394908F1FF3E01EBCE0132463B46D1E945
:100590000001CDF848E0F9F7F1FECDE91601594622
:1005A000504601F005FC0546F9F782FE02460B466F
:1005B00050465946F9F72EFD0F460B993035B8F1E4
:1005C000010F06460D7001F1010B21D00B994B1E56
:1005D0000D4603EB080A304639460022244BF9F752
:1005E000CDFE0F46064601F0E3FB8046F9F760FEBC
:1005F00008F1300802460B4630463946F9F70AFD45
:1006000005F8018F5545E8D1129A06460F469344E6
:100610000022184BDDE91601F9F7FEFC32463B4695
:1006200001F09EFB00285BD0199E08961BF8015C28
:100630000B9AFFF73FBB0A9E0023C9EB0605FFF7A5
:100640006ABB1A9B0E9F0A9DC3F13603FFF763BB7B
:100650005746FFF7ABBBDDE914AB4FF0020843E5AB
:1006600000001C4000001440702B0108382C0108C9
:10067000000024400000E03FB9F1000F3FF4A9AEB4
:10068000119E002E7FF719AF0022384B5046594675
:10069000F9F774FE824608F101008B46F9F708FE6F
:1006A00002460B4650465946F9F768FE0022304B89
:1006B000F9F7B2FCDDF820E0DDF844800EF1FF3EF2
:1006C0000646CDF864E0A1F150772DE5079B0B9924
:1006D000392235461A703E4603F1010BFFF7D6BBAF
:1006E000DDE9162300202349F9F794FC32463B4606
:1006F00001F054FB00283FF4E0AE5B469B46013B13
:100700001BF8012C302AF9D0199E0896FFF7D9BAA8
:1007100045465446199E08960B9AFFF7CBBABAF194
:10072000390FCDF83090D946D0D0069B002B3FF73B
:10073000AAAEAAE67FF4A9AE1AF0010F3FF4A5AE67
:100740009DE6314620460A220023DDF8449000F061
:100750003DFB0646FFF75BBB4FF00208C4E43FF4E5
:1007600040ABC3F13C03FFF7D4BB00BF0000244003
:1007700000001C400000E03F2DE9F04F936883B07B
:10078000164681460C462BB38B89190726D522695C
:1007900022B303F0020292B23568002A2CD04FF047
:1007A000000ADFF8E8B2D046D84534BF43465B467E
:1007B00052464846B8F1000F4FD0E169676AB84722
:1007C000002856DDB3681B1A8244C0EB0808B360EA
:1007D000002BE9D1002003B0BDE8F08F4846214648
:1007E000FEF792FF002840F04881A389356803F0A6
:1007F000020292B2002AD2D113F0010A42D1D046AD
:10080000B8F1000F23D09A05A76876D5B845C0F097
:10081000A48013F4906F40F0B2802068BB4651462C
:100820005A4600F043FAA2682168D21B01EB0B0381
:10083000A26023604246B3689B1A9244C2EB080848
:10084000B360002BC6D0A389B8F1000FDBD1D5F877
:1008500000A0D5F804800835D2E7D5F800A0D5F877
:1008600004800835A0E748462146FAF7CBFB00286C
:1008700059D0A38943F040034FF0FF30A38103B068
:10088000BDE8F08F9246019293469046B8F1000F72
:100890002BD0019F002F64D020682169D4F808C0B4
:1008A0006269C24534BF5346434688421F4603D956
:1008B0009444634500F3AE80934236DB1346676A87
:1008C000E16948465A46B847071ED2DDBAEB070A27
:1008D0003AD0B368DB1BBB44C7EB0808B360002BFE
:1008E0003FF478AFB8F1000FD3D10027D5F800B0AE
:1008F000D5F8048001970835C8E720682369984235
:1009000002D86369984572D2B84538BF47463A461F
:10091000514600F0CBF9A3682268DB1B3A44A36080
:100920002260002B9FD03A4685E71A46594600932D
:1009300000F0BCF9009BA1682268C91ABAEB070A4B
:100940001344A1602360C4D148462146FAF75AFBFC
:1009500000288ED1CDF804A0BBE720684746C346E7
:100960005DE758460A21424600F024F900287FD06E
:1009700000F1010A0127CBEB0A0A01978CE72268F4
:1009800021696769C1EB020C07EB47070CF1010213
:1009900007EBD77742447F10974234BF17463A4659
:1009A0005B054FD511464846CDF800C0FAF730FE3A
:1009B000DDF800C08346002862D062462169CDF888
:1009C00000C0FBF7C1F8A289DDF800C022F49062F4
:1009D00042F08002A2810BEB0C00CCEB0702C4F8C2
:1009E00010B067612060A2604746C34617E76FF00A
:1009F0000042904538BF424692FBF3F202FB03F3FC
:100A0000676AE16948465246B84700287FF731AF28
:100A1000024610E762465946CDF800C000F046F99C
:100A2000DDF800C023686344236048462146CDF8C2
:100A300000C0FAF7E7FADDF800C000287FF419AF2C
:100A4000674643E74846CDF800C000F0BDFCDDF83E
:100A500000C083460028BED148462169FAF790FCC1
:100A6000A3890C2223F080039BB2C9F8002001E780
:100A7000012708F1010A01970EE74FF0FF30AAE6BF
:100A80000C23C9F80030A389F4E600BF00FCFF7F07
:100A9000004870479C0A0020014B1868704700BF4F
:100AA000BC0A002000487047640A002070B5084C5A
:100AB00006460025084611461A462560EFF718FD40
:100AC000431C00D070BD2368002BFBD0336070BD89
:100AD0009C140020F0B58B899AB2960791B00C4611
:100AE000054637D4B1F90E10002917DB01AA01F031
:100AF0007BF8002810DB029B03F47043B3F5005130
:100B00004F424F41B3F5004F2CD0A38943F400630B
:100B1000A3814FF480660BE0A3899AB212F0800F94
:100B200043F40063A38114BF40264FF4806600277E
:100B300028463146FAF76CFDA389002829D01B4AC4
:100B4000EA6343F08003A381206020616661A7B956
:100B500011B0F0BD01F1430301220B600B614A614A
:100B600011B0F0BD124AA36A9342CED1A3894FF4CB
:100B700080663343A381E664DAE72846B4F90E10B1
:100B800001F046F80028E3D0A38943F00103A381D4
:100B9000DEE79A05DCD404F1430243F002030121AD
:100BA000A381226022616161D2E700BF89B00008A1
:100BB000E1BF0008830770B4C9B23FD0541E2AB306
:100BC00003788B4223D0431C04E0FCB104788C42B0
:100BD0001DD0144613F0030F184604F1FF3203F141
:100BE0000103F2D1032C14D8651E4CB303788B4259
:100BF0000DD0421C002302E004788C4207D0AB42A7
:100C0000104603F1010302F10102F5D1002070BC8E
:100C1000704741EA0126034646EA06461846043371
:100C200002687240A2F1013525EA020212F0803F0B
:100C3000DAD1043C032C1846F0D8D5E71446D1E7A6
:100C40002046E4E7032A70B428D940EA01039B0751
:100C500013D005780C78A54224D1013A002305E091
:100C600010F8015F11F8014FA5421BD1934203F127
:100C70000103F5D1002070BC70470C46034625687F
:100C80001E68AE422146184604F1040403F1040331
:100C900004D1043A032A18462146F0D8002AD8D1B4
:100CA0001046E8E7281B70BC704700BF8842F0B4CC
:100CB00010D98C18A0420DD28518531E42B121467E
:100CC0002A4611F8014D02F8014D013B5C1CF8D198
:100CD000F0BC70470F2A3FD940EA01039B073FD180
:100CE000A2F110073F0900EB071610360C46034629
:100CF00025681D6065685D60A5689D60E568DD60CC
:100D00001033B34204F11004F2D17B1C02F00F0C3B
:100D10001B01BCF1030F1944034423D90E461D46A1
:100D20006446043C56F8047B45F8047B032CF8D851
:100D3000ACF1040424F00304043402F0030223445D
:100D40002144002AC4D01A4411F8014B03F8014B86
:100D50009342F9D1F0BC70470346002AF3D1B7E7BC
:100D60000346F0E76246002AEDD1B1E7C26C70B5E8
:100D700005460C464AB152F8240080B1016842F899
:100D8000241000220261C26070BD2122042100F003
:100D90009DFEE86402460028EDD1002070BD0121CF
:100DA00001FA04F6721D2846920000F08FFE00281A
:100DB000F3D044608660E4E731B1C36C4A6853F80D
:100DC0002200086043F82210704700BF2DE9F04769
:100DD000D1F8108082B08946824601F114050024C2
:100DE0002F68BEB23F0C02FB063602FB07F303EB93
:100DF00016430134B6B206EB0346A04545F8046B32
:100E00004FEA1343ECDC53B1D9F8082090450ADAD5
:100E100009EB880108F101024B61C9F8102048462E
:100E200002B0BDE8F087D9F80410019301315046B3
:100E3000FFF79CFFD9F81020023209F10C0104469B
:100E400092000C30FAF780FEDAF84C20D9F8041042
:100E5000019B52F82100C9F8000042F82190A146F8
:100E6000D6E700BF030C1B04B3B90004102310F035
:100E70007F4F04BF0002083310F0704F04BF000121
:100E8000043310F0404F04BF80000233002807DB1A
:100E9000420003D4202070470023E8E7581C704725
:100EA00018467047036813F0070207D0D90720D40B
:100EB0009A0720D49B0803600220704799B209B9B1
:100EC0001B0C102213F0FF0F04BF1B0A0832190776
:100ED00004BF1B090432990704BF9B080232D907DB
:100EE00004D45B0801D12020704701320360104612
:100EF0007047002070475B0803600120704700BF07
:100F000010B50C460121FFF731FF01224461026157
:100F100010BD00BF2DE9F04F0D69D2F810904D457E
:100F200085B00C46924604DA2A4654464D468A4617
:100F30009146A368616805EB09079F42C8BF01316C
:100F4000FFF714FF00F1140606EB870846450190F1
:100F500005D23346002043F8040B9845FBD80AF12C
:100F6000140C0CEB89091434CC45009404EB850572
:100F70005BD2CDF808800397C8465CF8043B9CB26E
:100F800024B3009A33464FF0000900E00B4652F8B4
:100F9000047B19681FFA87FB1FFA81FA380C090CC9
:100FA00004FB0BA7B94404FB001000EB19401946E1
:100FB0001FFA89F949EA004795424FEA104941F87A
:100FC000047BE3D8C3F804905CF8043C5FEA13495F
:100FD00024D0D6F800A0009B504631464FF0000BBD
:100FE00000E011461A88000C09FB020083441FFA36
:100FF0008AFA0A464AEA0B4042F8040B53F8047B8B
:1010000048684FEA174A84B209FB0A4A0AEB1B4AAE
:101010009D424FEA1A4BE4D8C1F804A0E04506F11E
:101020000406AAD8DDF80880039F002F0ADD58F8CF
:10103000043CA8F104081BB104E058F8043D0BB9C6
:10104000013FFAD1019B18461F6105B0BDE8F08F42
:1010500012F003032DE9F041144607460E462CD149
:10106000A4101CD0BD6C002D30D04FF0000804E05F
:10107000641014D02868A8B10546E307F8D53846AF
:1010800031462A46FFF746FFAEB17268FB6C64102A
:1010900053F82210316043F822600646EAD1304608
:1010A000BDE8F081384629462A46FFF733FF28601D
:1010B000C0F80080E0E70646DAE75D1E0A4A002332
:1010C00052F82520FFF782FE0646C9E7012138467F
:1010D000FFF74CFE40F271210122002341610261C1
:1010E0000546B8640360C0E7602C01082DE9F84F9D
:1010F00093460A698B684FEA6B1A0AEB020909F1F9
:1011000001069E420F468046496804DD5B009E4210
:1011100001F10101FADC4046FFF728FEBAF1000FA9
:1011200000F1140409DD00231A4625460133534516
:1011300045F8042BFAD104EB83043A6907F1140350
:101140001BF01F0B03EB820C21D0CBF1200A0022F5
:1011500000E02C461968254601FA0BF10A4345F8D0
:10116000042B53F8042B634522FA0AF2F1D3626090
:101170000AB109F10206D8F84C307A68013E53F8FA
:1011800022100661396043F82270BDE8F88F53F8E9
:10119000042B44F8042B9C45EDD953F8042B44F858
:1011A000042B9C45F3D8E6E702690B69D21A10B408
:1011B00015D19B00143014311944034401E09842C6
:1011C00011D253F8042D51F8044DA242F7D09442A5
:1011D00094BF01204FF0FF305DF8044B704710467C
:1011E0005DF8044B704700205DF8044B704700BF6A
:1011F0002DE9F0470D460446114628461646FFF7EE
:10120000D3FF071E55D04EDB4FF00008696820461B
:10121000FFF7ACFD2F693269C0F80C801435143625
:1012200000F1140305EB870C06EB8208002156F849
:10123000042B55F8044B1FFA82F911FA84FA110CA9
:10124000C1EB1441C9EB0A0201EB224192B242EA1E
:101250000142B04543F8042B4FEA21412C46E6D821
:10126000AC45984615D954F8046B11FA86F1360C42
:1012700006EB214689B241EA0642A44543F8042B15
:101280004FEA2641EFD8EB43634423F003030433D2
:101290004344043B22B953F8042D013F002AFAD0FD
:1012A0000761BDE8F0872B464FF0010835461E4622
:1012B000ACE720463946FFF759FD0123476103613A
:1012C000BDE8F0872DE9F043894683B0012155EC54
:1012D000104B9046FFF74AFDC5F30A570646C5F383
:1012E00013030FB143F48013019314B302A840F821
:1012F000084D6846FFF7D6FD002831D19DE80C0067
:101300007261002B0CBF01240224B3613461D7B990
:1013100006EB8403A0F23240C9F800001869FFF719
:10132000A1FDC0EB4410C8F80000304603B0BDE892
:10133000F08301A8FFF7B6FD0124019B7361203003
:101340003461002FE4D0A7F233470744C0F13500E1
:10135000C9F80070C8F80000304603B0BDE8F0835B
:101360009DE80C00C0F1200103FA01F10A43C340DB
:1013700001937261C5E700BF70B5084C06460025B1
:10138000084611461A462560EFF78AF8431C00D03C
:1013900070BD2368002BFBD0336070BD9C1400200F
:1013A00070B5084C06460025084611461A462560C9
:1013B000EFF7AEF8431C00D070BD2368002BFBD0C4
:1013C000336070BD9C1400202DE9F04F0C4683B0B3
:1013D00090468146002900F0E280FAF799FC08F176
:1013E0000B0654F8043C162E23F00305A4F108075D
:1013F0004BD810210E46B0454CD88D4278DADFF834
:1014000090B3DBF808E07819864500F0CE8042689A
:1014100022F0010C8444DCF804C01CF0010F7AD0E7
:1014200000221046DB0700F1928054F8083CC3EB21
:10143000070ADAF8043023F003032B4488B370451D
:1014400000F0ED8002EB030E8E452ADBC368826854
:101450005746D3609A6057F8081FDAF80C30CB6013
:101460002A1F242A996000F22681132A40F2B380B1
:101470002368CAF808306368CAF80C301B2A00F2E7
:10148000308108340AF11003A6E026F00706002E8A
:101490003146B0DA0C230020C9F8003003B0BDE8B3
:1014A000F08F8B4253DB5746DAF80C1057F8080FD1
:1014B0002A1F242AC160886000F20981132A40F2A1
:1014C00004812168CAF808106168CAF80C101B2A48
:1014D00000F21C8108340AF1100221681160616871
:1014E0005160A16891601D46DAF804303C465746C9
:1014F000AA1B0F2A03F0010319D82B433D447B603C
:101500006B6843F001036B604846FAF703FC204622
:1015100003B0BDE8F08F22F0030202EB050C8C450E
:1015200080DBC26881686546CA609160E0E7B919EE
:1015300042F001001E430A447E604860536843F055
:101540000103083153604846F9F71AFFDCE74146CA
:101550004846FAF75DF88046D0B154F8043C23F0D1
:1015600001023A44A0F10801914200F09E802A1F36
:10157000242A50D8132A23D803462246116819601A
:101580005168596092689A6021464846F9F7F8FE1A
:101590004846FAF7BFFB404603B0BDE8F08F11465E
:1015A00003B0BDE8F04FFAF733B8DEF8042022F0BC
:1015B0000302501906F1100C604519DA704631E744
:1015C00023680360636843601B2A63D800F1080343
:1015D00004F10802D2E73B4622681A6062685A604A
:1015E000A2689A603C467546DAF8043057467FE7B1
:1015F0003744831B43F00103CBF808707B6054F839
:10160000043C03F001031E43484644F8046CFAF717
:1016100081FB20467CE72146FFF748FBB4E702EB5D
:10162000030C06F110029445FFF63BAF5746DAF87B
:101630000C3057F8081F2A1F242ACB60996000F24B
:101640008780132A78D92368CAF808306368CAF8F3
:101650000C301B2A00F2858008340AF1100322683E
:101660001A6062685A60A2689A600AEB0603C6EBC9
:101670000C0242F00102CBF808305A60DAF804306C
:1016800003F001031E434846CAF80460FAF742FB20
:1016900038463DE7A3688360E368C360242A2CD002
:1016A00000F1100304F1100268E750F8042C22F056
:1016B000030215441CE72146384675463C46FFF7B1
:1016C000F5FA5746DAF8043012E73A4605E72146BC
:1016D00038461D463C46FFF7E9FA5746DAF804302B
:1016E00006E7A368CAF81030E368CAF81430242A61
:1016F00018D010340AF118036EE723690361636997
:10170000436104F1180200F1180337E7A168CAF831
:101710001010E168CAF81410242A0FD010340AF10E
:101720001802DAE62369CAF818306369CAF81C306F
:1017300018340AF120034FE73B4690E72269CAF8C4
:1017400018206269CAF81C2018340AF12002C4E685
:1017500021463846CDF804C0FFF7A8FADDF804C0EA
:1017600083E7A368CAF81030E368CAF81430242A63
:1017700003D010340AF1180371E72369CAF818304E
:101780006369CAF81C3018340AF1200367E700BF08
:101790005406002053EC102B33F0004110B408D055
:1017A0000F48A1F5801484420AD804205DF8044B48
:1017B0007047002A0CBF022003205DF8044B7047DD
:1017C000B1F5801F01D20320F7E70648814201D01E
:1017D0000020F2E7D2F1010038BF0020EDE700BFA2
:1017E000FFFFDF7F0000F07FC9B2F0B4002947D0CF
:1017F00085070FD00278002A3FD091423ED0431C8B
:1018000005E013F8012B002A37D0914236D09A0711
:101810001846F6D1036841EA012747EA074783EAF9
:101820000702A2F10135A3F1013425EA020224EAFC
:101830000303134313F0803F11D1021D104652F8E9
:10184000043B83EA0704A4F10136A3F1013526EA3B
:10185000040425EA0303234313F0803FEED003780A
:10186000002B39D0994209D0431C01E0914205D0A8
:10187000184613F8012B002AF8D11046F0BC704727
:1018800084070BD00378002BF8D0431C03E00278C8
:101890000133002AF2D099071846F8D10368A3F162
:1018A000013222EA030313F0803F0AD1031D1846D8
:1018B00053F8042BA2F1013121EA020212F0803F19
:1018C000F5D00378002BD9D0431C18460133027899
:1018D000002AFAD1F0BC70471846CFE72DE9F04F47
:1018E0009368166883B0924680460D46002B6FD0F1
:1018F0004FF0000B08688B685C46002C43D09C427C
:101900001F4645D3AB8913F4906F44D06F692969A2
:1019100007EB470707EBD777C1EB0009621C7F1085
:101920004A44974234BF17463A465B0535D51146BF
:101930004046F9F76DFE002839D0296901904A46E2
:10194000FAF702F9AA89019B22F4906242F0800220
:10195000AA81C9EB070203EB09006F612B612860C4
:10196000AA602746A1464A465946FFF79FF9DAF88A
:101970000820AB682868DB1B4844141BAB60286058
:10198000CAF8084024B3D6F800B074680836B4E743
:101990002746A146E7E7B946E5E74046FFF714FDCD
:1019A00003460028D5D140462969F9F7E9FCAA8900
:1019B0000C23C8F8003042F0400200234FF0FF3003
:1019C000AA81CAF80830CAF8043003B0BDE8F08F25
:1019D0000020CAF8040003B0BDE8F08F70B51446CB
:1019E0009AB0156809B1002D1AD100254FF4227262
:1019F000ADF80C20009504951A464FF6FF7669461F
:101A00001E9B02950595ADF80E60FBF75DF800286A
:101A100011DB009B206000221A7004981AB070BD80
:101A20004FF4C16200910491ADF80C20E4DA8B23ED
:101A300003600020F2E70020F0E700BF4B6E2DE9C5
:101A4000F0479C040E46804691462AD5936812685A
:101A500002F1080A1BB31AE9A000BF0817D0043D21
:101A6000002401E0A74210D0404655F8041F32463A
:101A700000F05CF8431C04F10104F3D10023C9F821
:101A80000830C9F80430BDE8F087D9F80830A3EB76
:101A90008703C9F808300AF1080A002BDBD10020BF
:101AA000ECE7FEF769FE0023C9F80830C9F80430F6
:101AB000BDE8F087936810B41BB15DF8044BFFF7E5
:101AC000BDBF184653605DF8044B704710B502FB6C
:101AD00001F1F9F79DFD044668B150F8042C22F09D
:101AE0000302043A242A18D8132A06D803460022EF
:101AF0001A605A609A60204610BD00231B2A0360BA
:101B000043600FD9242A8360C36005BF036143612A
:101B100000F1100300F11803E9E70021FAF7AEF82D
:101B2000204610BD00F10803E1E700BF2DE9F041B8
:101B300093890F46990482B01446804606D4526EAB
:101B400043F4005342F40052A3816266FEF7A4FFFF
:101B500001283DD03A46404601A904F15C0300F05B
:101B600069F8421C06462CD0002839D09DF8041094
:101B7000002509E0236819702368013323600135CB
:101B8000B5422DD201ABE95CA368013B002BA360F9
:101B9000F0DAA269934205DB23681970236819788B
:101BA0000A29EAD140462246FDF746FDB0F1FF334F
:101BB000584258410028E2D04FF0FF3002B0BDE853
:101BC000F081A38943F04003A38102B0BDE8F08116
:101BD0007B1EFE2BBED8F9B206468DF80410C7E76F
:101BE000384602B0BDE8F08138B5084C0023054600
:101BF000084611462360F5F7AFFD431C00D038BD01
